:020000040000FA
:1000000000040020810A000015070000610A0000BA
:100010001F07000029070000330700000000000050
:10002000000000000000000000000000A50A000021
:100030003D070000000000004707000051070000D6
:100040005B070000650700006F07000079070000EC
:10005000830700008D07000097070000A10700003C
:10006000AB070000B5070000BF070000C90700008C
:10007000D3070000DD070000E7070000F1070000DC
:10008000FB070000050800000F0800001908000029
:10009000230800002D080000370800004108000078
:1000A0004B080000550800005F08000069080000C8
:1000B000730800007D080000870800009108000018
:1000C0009B080000A5080000AF080000B908000068
:1000D000C3080000CD080000D7080000E1080000B8
:1000E000EB080000F5080000FF0800000909000007
:1000F000130900001D090000270900003109000054
:100100003B0900001FB500F003F88DE80F001FBD8C
:1001100000F0ACBC40F6FC7108684FF01022401CA7
:1001200008D00868401C09D00868401C04D0086842
:1001300000F037BA9069F5E79069F9E7704770B554
:100140000B46010B184400F6FF70040B4FF0805073
:100150000022090303692403406943431D1B104621
:1001600000F048FA29462046BDE8704000F042BA47
:10017000F0B54FF6FF734FF4B4751A466E1E11E0DA
:10018000A94201D3344600E00C46091B30F8027B3B
:10019000641E3B441A44F9D19CB204EB134394B25D
:1001A00004EB12420029EBD198B200EB134002EBB2
:1001B000124140EA0140F0BDF34992B00446D1E952
:1001C0000001CDE91001FF224021684600F0F4FB58
:1001D00094E80F008DE80F00684610A902E004C8FB
:1001E00041F8042D8842FAD110216846FFF7C0FF7C
:1001F0001090AA208DF8440000F099F9FFF78AFFCB
:1002000040F6FC7420684FF01025401C0FD0206889
:1002100010226946803000F078F92068401C08D030
:100220002068082210A900F070F900F061F9A869AF
:10023000EEE7A869F5E74FF080500369406940F6A2
:10024000FC71434308684FF01022401C06D0086838
:1002500000F58050834203D2092070479069F7E788
:100260000868401C04D00868401C03D00020704778
:100270009069F9E70420704770B504460068C34DE3
:10028000072876D2DFE800F033041929631E250021
:10029000D4E9026564682946304600F062F92A46CE
:1002A0002146304600F031F9AA002146304600F0E0
:1002B00057FB002800D0032070BD00F009FC4FF46C
:1002C000805007E0201D00F040F90028F4D100F034
:1002D000FFFB60682860002070BD241D94E80700C3
:1002E000920000F03DFB0028F6D00E2070BDFFF715
:1002F000A2FF0028FAD1D4E901034FF0805100EBAE
:10030000830208694D69684382420ED840F6F8704E
:1003100005684FF010226D1C09D0056805EB8305B8
:100320000B6949694B439D4203D9092070BD55694A
:10033000F4E70168491C03D00068401C02D003E0C8
:100340005069FAE70F2070BD2046FFF735FFFFF731
:1003500072FF0028F7D1201D00F0F7F80028F2D135
:1003600060680028F0D100F0E2F8FFF7D3FE00F05B
:10037000BFF8072070BD10B50C46182802D0012028
:10038000086010BD2068FFF777FF206010BD41684E
:10039000054609B1012700E0002740F6F8742068FF
:1003A0004FF01026401C2BD02068AA68920000F065
:1003B000D7FA38B3A86881002068401C27D020688D
:1003C000FFF7BDFED7B12068401C22D026684FF051
:1003D0008050AC686D68016942695143A9420DD9EA
:1003E000016940694143A14208D92146304600F0E5
:1003F000B8F822462946304600F087F800F078F831
:100400007069D2E700F093F8FFF784FEF6E77069B1
:10041000D6E77669DBE740F6FC7420684FF01026DB
:10042000401C23D02068401C0CD02068401C1FD0EA
:100430002568206805F18005401C1BD027683879A5
:10044000AA2819D040F6F8700168491C42D001680A
:10045000491C45D00168491C3ED001680968491C07
:100460003ED00168491C39D000683EE0B069DAE747
:10047000B569DEE7B769E2E710212846FFF778FEA5
:100480003968814222D12068401C05D0D4F8001080
:1004900001F18002C03107E0B169F9E730B108CA63
:1004A00051F8040D984201D1012000E000208A4259
:1004B000F4D158B1286810B1042803D0FEE72846CB
:1004C000FFF765FF3149686808600EE0FFF722FE1C
:1004D00000F00EF87169BBE77169BFE7706904E06D
:1004E0004FF480500168491C01D000F0CBFAFEE7C0
:1004F000BFF34F8F26480168264A01F4E06111439B
:100500000160BFF34F8F00BFFDE72DE9F0411746B3
:100510000D460646002406E03046296800F054F8EF
:10052000641C2D1D361DBC42F6D3BDE8F08140F69B
:10053000FC700168491C04D0D0F800004FF48051D1
:10054000FDE54FF010208069F8E74FF080510A690F
:10055000496900684A43824201D810207047002050
:10056000704770B50C4605464FF4806608E0284693
:1005700000F017F8B44205D3A4F5806405F5805562
:10058000002CF4D170BD0000F40A0000000000202F
:100590000CED00E00400FA05144801680029FCD0C5
:1005A0007047134A0221116010490B68002BFCD0E0
:1005B0000F4B1B1D186008680028FCD0002010603D
:1005C00008680028FCD07047094B10B501221A605A
:1005D000064A1468002CFCD0016010680028FCD08A
:1005E0000020186010680028FCD010BD00E4014015
:1005F00004E5014070B50C46054600F073F810B9EB
:1006000000F07EF828B121462846BDE8704000F091
:1006100007B821462846BDE8704000F037B8000012
:100620007FB5002200920192029203920A0B000B06
:100630006946012302440AE0440900F01F0651F80C
:10064000245003FA06F6354341F82450401C8242F8
:10065000F2D80D490868009A10430860081D016827
:10066000019A1143016000F03DF800280AD00649C4
:1006700010310868029A10430860091D0868039A3F
:10068000104308607FBD00000006004030B50F4CED
:10069000002200BF04EB0213D3F800582DB9D3F8A1
:1006A000045815B9D3F808581DB1521C082AF1D3C3
:1006B00030BD082AFCD204EB0212C2F80008C3F8CD
:1006C00004180220C3F8080830BD000000E0014013
:1006D0004FF08050D0F83001082801D0002070473A
:1006E000012070474FF08050D0F83011062905D016
:1006F000D0F83001401C01D0002070470120704725
:100700004FF08050D0F830010A2801D00020704707
:100710000120704708208F490968095808471020B0
:100720008C4909680958084714208A4909680958FA
:100730000847182087490968095808473020854923
:100740000968095808473820824909680958084744
:100750003C20804909680958084740207D490968BC
:100760000958084744207B49096809580847482028
:1007700078490968095808474C207649096809589A
:10078000084750207349096809580847542071499F
:1007900009680958084758206E49096809580847E8
:1007A0005C206C4909680958084760206949096854
:1007B00009580847642067490968095808476820AC
:1007C00064490968095808476C2062490968095852
:1007D000084770205F4909680958084774205D4937
:1007E00009680958084778205A490968095808478C
:1007F0007C205849096809580847802055490968EC
:10080000095808478420534909680958084788202F
:1008100050490968095808478C204E490968095809
:10082000084790204B4909680958084794204949CE
:10083000096809580847982046490968095808472F
:100840009C204449096809580847A0204149096883
:1008500009580847A4203F49096809580847A820B3
:100860003C49096809580847AC203A4909680958C1
:100870000847B0203749096809580847B420354966
:10088000096809580847B8203249096809580847D3
:10089000BC203049096809580847C0202D4909681B
:1008A00009580847C4202B49096809580847C82037
:1008B0002849096809580847CC2026490968095879
:1008C0000847D0202349096809580847D4202149FE
:1008D000096809580847D8201E4909680958084777
:1008E000DC201C49096809580847E02019490968B3
:1008F00009580847E4201749096809580847E820BB
:100900001449096809580847EC2012490968095830
:100910000847F0200F49096809580847F4200D4995
:10092000096809580847F8200A490968095808471A
:10093000FC2008490968095808475FF48070054998
:10094000096809580847000003480449024A034B54
:100950007047000000000020000B0000000B0000AA
:1009600040EA010310B59B070FD1042A0DD310C82C
:1009700008C9121F9C42F8D020BA19BA884201D97E
:10098000012010BD4FF0FF3010BD1AB1D30703D0C6
:10099000521C07E0002010BD10F8013B11F8014B7C
:1009A0001B1B07D110F8013B11F8014B1B1B01D198
:1009B000921EF1D1184610BD02F0FF0343EA032254
:1009C00042EA024200F005B87047704770474FF0A6
:1009D00000020429C0F0128010F0030C00F01B800C
:1009E000CCF1040CBCF1020F18BF00F8012BA8BF1A
:1009F00020F8022BA1EB0C0100F00DB85FEAC17CDE
:100A000024BF00F8012B00F8012B48BF00F8012B90
:100A100070474FF0000200B51346944696462039C1
:100A200022BFA0E80C50A0E80C50B1F12001BFF4A7
:100A3000F7AF090728BFA0E80C5048BF0CC05DF80D
:100A400004EB890028BF40F8042B08BF704748BF5B
:100A500020F8022B11F0804F18BF00F8012B7047CF
:100A6000014B1B68DB6818470000002009480A4951
:100A70007047FFF7FBFFFFF745FB00BD20BFFDE719
:100A8000064B1847064A1060016881F308884068E1
:100A900000470000000B0000000B000017040000DE
:100AA000000000201EF0040F0CBFEFF30881EFF3ED
:100AB0000981886902380078182803D100E0000015
:100AC000074A1047074A12682C3212681047000084
:100AD00000B5054B1B68054A9B58984700BD0000B0
:100AE0007703000000000020F00A0000040000006E
:100AF000001000000000000000FFFFFF0090D00386
:10100000B813002065520200F1C00000CB5102006D
:10101000F1C00000F1C00000F1C0000000000000BD
:10102000000000000000000000000000F15202007B
:10103000F1C0000000000000F1C00000F1C000009D
:10104000595302005F530200F1C00000F1C00000DC
:10105000F1C00000F1C00000F1C00000F1C00000CC
:1010600065530200F1C00000F1C000006B530200A4
:10107000F1C0000071530200775302007D5302005B
:10108000F1C00000F1C00000F1C00000F1C000009C
:10109000F1C00000F1C00000F1C00000F1C000008C
:1010A000F1C0000083530200F1C00000F1C0000055
:1010B000F1C00000F1C00000F1C00000F1C000006C
:1010C00089530200F1C00000F1C00000F1C000002F
:1010D000F1C00000F1C00000F1C00000F1C000004C
:1010E000F1C00000F1C00000F1C00000F1C000003C
:1010F000F1C00000F1C00000F1C00000F1C000002C
:10110000F1C00000F1C0000000F002F824F099F8EE
:101110000AA090E8000C82448344AAF10107DA4552
:1011200001D124F08EF8AFF2090EBAE80F0013F0E7
:10113000010F18BFFB1A43F00103184730470200A4
:10114000504702000A444FF0000C10F8013B13F026
:10115000070408BF10F8014B1D1108BF10F8015B10
:10116000641E05D010F8016B641E01F8016BF9D103
:1011700013F0080F1EBF10F8014BAD1C0C1B09D15A
:101180006D1E58BF01F801CBFAD505E014F8016BCC
:1011900001F8016B6D1EF9D59142D6D3704700005E
:1011A0000023002400250026103A28BF78C1FBD870
:1011B000520728BF30C148BF0B6070471FB500F011
:1011C00003F88DE80F001FBD24F038B870B51A4C35
:1011D00005460A202070A01C00F0D5F85920A080F8
:1011E00029462046BDE8704008F08EB908F097B94E
:1011F00070B50C461149097829B1A0F160015E294A
:1012000008D3012013E0602804D0692802D043F2FB
:1012100001000CE020CC0A4E94E80E0006EB8000A2
:10122000A0F58050241FD0F8806E2846B04720607B
:1012300070BD012070470000080000201800002049
:10124000D45302003249884201D201207047002065
:10125000704770B50446A0F500002E4EB0F1786FCF
:1012600002D23444A4F500042948844201D2012565
:1012700000E0002500F043F848B125B9B44204D39A
:101280002548006808E0012070BD002070BD002DD9
:10129000F9D1B442F9D321488442F6D2F3E710B52C
:1012A0000446A0F50000B0F1786F03D21948044459
:1012B000A4F5000400F023F84FF0804130B1164847
:1012C000006804E08C4204D2012003E01348844209
:1012D000F8D2002080F0010010BD10B520B1FFF75A
:1012E000DEFF08B1012010BD002010BD10B520B1F7
:1012F000FFF7AFFF08B1012010BD002010BD084866
:1013000008490068884201D10120704700207047D9
:1013100000600200000000201C00002008000020E7
:1013200058000020BEBAFECA10B5044600210120B4
:1013300000F041F800210B2000F03DF800210820CA
:1013400000F039F80421192000F035F804210D20AF
:1013500000F031F804210E2000F02DF804210F20B8
:1013600000F029F80421C84300F025F806211620D2
:1013700000F021F80621152000F01DF82046FFF7A7
:1013800025FF002010BDCB2101807047FFF72EBF45
:101390001148704710487047104A10B514680F4B39
:1013A0000F4A08331A60FFF723FF0C48001D046042
:1013B00010BD704770474907090E002804DB00F193
:1013C000E02080F80014704700F00F0000F1E020EA
:1013D00080F8141D7047000003F900421005024018
:1013E00001000001FD48002101604160018170475A
:1013F0002DE9FF4F93B09B46209F160004460DD069
:101400001046FFF726FF18B1102017B0BDE8F08F87
:101410003146012001F0D3FE0028F6D101258DF8D8
:1014200042504FF4C050ADF84000002210A92846A9
:1014300006F0CCFC0028E8D18DF84250A8464FF4C5
:1014400028500025ADF840001C2229466846079523
:101450000CF0D3FF9DF81C000DF11C0A20F00F00CA
:10146000401C20F0F00010308DF81C0020788DF822
:101470001D0061789DF81E000DF1400961F34200E6
:1014800040F001008DF81E009DF8000008AA40F011
:1014900002008DF800002089ADF83000ADF8325020
:1014A0006089ADF83400CDF82CA060680E900AA9D0
:1014B000CDF82890684606F07EFA0028A5D160682D
:1014C000FFF70BFF40B16068FFF710FF20B96078AD
:1014D00000F00300022801D0012000E00020BF4CF2
:1014E00008AA0AA92072BDF8200020808DF8428049
:1014F00042F60120ADF840009DF81E0020F00600E5
:10150000801C20F001008DF81E000220ADF8300094
:10151000ADF8340014A80E90684606F04CFA002886
:1015200089D1BDF82000608036B1211D304600F021
:101530005FF90028C2D109E0BBF1000F05D00CF023
:10154000D7FCE8BB0CF0D4FCD0BBA58017B1012FB1
:1015500043D04AE08DF8428042F6A620ADF8400024
:1015600046461C220021684607950CF046FF9DF870
:101570001C00ADF8346020F00F00401C20F0F0009B
:1015800010308DF81C009DF81D0020F0FF008DF834
:101590001D009DF81E0020F0060040F00100801C98
:1015A0008DF81E009DF800008DF8446040F00200A8
:1015B0008DF80000CDE90A9AADF8306011A800E07E
:1015C00011E00E9008AA0AA9684606F0F4F900286E
:1015D000A6D1BDF82000E08008E00CF089FC10B92D
:1015E0000CF086FC08B103200FE7E58000200CE733
:1015F0003EB50446794D0820ADF80000A88828B112
:101600002046FFF726FE18B110203EBD06203EBD45
:101610002146012001F0D3FD0028F8D12088ADF843
:1016200004006088ADF80600A088ADF80800E088E6
:10163000ADF80A00A88801AB6A46002106F0C2FD99
:10164000BDF800100829E2D003203EBD7FB5634DF0
:101650000446A88868B1002002900820ADF8080070
:10166000CDF80CD02046FFF7F4FD20B1102004B0D7
:1016700070BD0620FBE7A98802AA4FF6FF7006F0AE
:10168000E3FF0028F3D1BDF80810082901D003209A
:10169000EDE7BDF800102180BDF802106180BDF8B3
:1016A0000410A180BDF80610E180E0E701B582B02A
:1016B0000220ADF80000494802AB6A46408800218C
:1016C00006F080FDBDF80010022900D003200EBDF9
:1016D0001CB5002100910221ADF800100190FFF728
:1016E000DEFD08B110201CBD3C486A4641884FF61B
:1016F000FF7006F0A9FFBDF800100229F3D0032007
:101700001CBDFEB5354C06461546207A0F46C0076F
:1017100005D00846FFF79DFD18B11020FEBD0F2033
:10172000FEBDF82D01D90C20FEBD3046FFF791FD1E
:1017300018BB208801A905F040FE0028F4D13078BC
:101740008DF80500208801A906F01AFD0028EBD1CC
:1017500000909DF800009DF8051040F002008DF803
:101760000000090703D040F008008DF80000208831
:10177000694606F0A2FC0028D6D1ADF808502088B2
:101780003B4602AA002106F01DFDBDF80810A94243
:10179000CAD00320FEBD7CB5054600200090019014
:1017A0000888ADF800000C4628460195FFF795FD26
:1017B00018B92046FFF773FD08B110207CBD15B1A4
:1017C000BDF8000060B105486A4601884FF6FF7019
:1017D00006F03AFFBDF8001021807CBD28020020F1
:1017E0000C20FAE72F48C088002800D0012070475D
:1017F00030B5044693B000200D46014600901422F7
:1018000001A80CF0FAFD1C22002108A80CF0F5FD3F
:101810009DF80000CDF808D020F00F00401C20F00B
:10182000F00010308DF800009DF8010006AA20F0AD
:10183000FF008DF801009DF8200001A940F0020092
:101840008DF8200001208DF8460042F60420ADF806
:10185000440011A801902088ADF83C006088ADF8E4
:101860003E00A088ADF84000E088ADF842009DF849
:10187000020020F00600801C20F001008DF802001C
:101880000820ADF80C00ADF810000FA8059008A8CE
:1018900006F091F8002803D1BDF818002880002038
:1018A00013B030BD28020020F0B5007B059F1E4616
:1018B00014460D46012800D0FFDF0C2030803A206E
:1018C0003880002C08D0287A032806D0287B0128ED
:1018D00000D0FFDF17206081F0BDA889FBE72DE96C
:1018E000F04786B0144691F80C900E9A0D46B9F167
:1018F000010F0BD01021007B2E8A8846052807D0C7
:10190000062833D0FFDF06B0BDE8F0870221F2E7FA
:10191000E8890C2100EB400001EB400018803320E7
:101920001080002CEFD0E889608100271AE0009633
:10193000688808F1020301AA696900F086FF06EBD6
:101940000800801C07EB470186B204EB4102BDF89A
:10195000040090810DF1060140460E3212F0C6FEE1
:101960007F1CBFB26089B842E1D8CCE73420108038
:10197000E889B9F1010F11D0122148430E301880C7
:10198000002CC0D0E88960814846B9F1010F00D031
:101990000220207300270DF1040A1FE00621ECE766
:1019A0000096688808F1020301AA696900F04DFFFA
:1019B00006EB0800801C86B2B9F1010F12D007EBCC
:1019C000C70004EB4000BDF80410C18110220AF1E9
:1019D000020110300CF0E7FC7F1CBFB26089B842F6
:1019E000DED890E707EB470104EB4102BDF80400A5
:1019F000D0810AF102014046103212F077FEEBE787
:101A00002DE9F0470E4688B090F80CC096F80C808F
:101A1000378AF5890C20109902F10C044FF0000A66
:101A2000BCF1030F08D0BCF1040F3FD0BCF1070F8D
:101A30007ED0FFDF08B067E705EB850C00EB4C00BC
:101A4000188031200880002AF4D0A8F1060000F0A8
:101A5000FF09558126E01622002101A80CF0CDFCDB
:101A600000977088434601AA716900F0EEFEBDF848
:101A700004002080BDF80600E080BDF80800208149
:101A8000A21C0DF10A01484612F030FEB9F1000F18
:101A900000D018B184F804A0A4F802A007EB080055
:101AA00087B20A346D1EADB2D5D2C3E705EB850C03
:101AB00000EB4C00188032200880002ABAD0A8F130
:101AC000050000F0FF09558137E000977088434614
:101AD00001AA716900F0B9FE9DF80600BDF8041076
:101AE000E1802179420860F3000162F3410182083C
:101AF00062F38201C20862F3C301020962F30411B6
:101B0000420962F34511820962F386112171C0090D
:101B10006071BDF80700208122460DF10901484699
:101B200012F0E4FD18B184F802A0A4F800A000E0CF
:101B300007E007EB080087B20A346D1EADB2C4D2CD
:101B400078E7A8F1020084B205FB08F000F10E0C62
:101B5000A3F800C035230B80002AA6D055819481BC
:101B6000009783B270880E32716900F06EFE61E7F3
:101B70002DE9F84F1E460A9D0C4681462AB1607A2F
:101B800000F58070D080E089108199F80C000C2756
:101B90004FF000084FF00E0A0D2872D2DFE800F077
:101BA0009D070E1B272F374554697272720021461C
:101BB00048460095FFF778FEBDE8F88F207B9146F8
:101BC000082802D0032800D0FFDF3780302009E04A
:101BD000A9F80A80F0E7207B9146042800D0FFDFB7
:101BE000378031202880B9F1000FF1D1E4E7207B64
:101BF0009146042800D0FFDF37803220F2E7207BB7
:101C00009146022800D0FFDF37803320EAE7207BAF
:101C10001746022800D0FFDF3420A6F800A0288055
:101C2000002FC9D0A7F80A80C6E7207B17460428F2
:101C300000D0FFDF3520A6F800A02880002FBBD001
:101C40004046A7F80A8012E0207B1746052802D0FC
:101C5000062800D0FFDF1020308036202880002F9B
:101C6000AAD0E0897881A7F80E80B9F80E00B88173
:101C7000A2E7207B9146072800D0FFDF378037207E
:101C8000B0E72AE04FF0120018804FF0380017003C
:101C9000288091D0E0897881A7F80E80A7F810807D
:101CA00099F80C000A2805D00B2809D00C280DD073
:101CB000FFDF81E7207B0A2800D0FFDF01200AE058
:101CC000207B0B2800D0FFDF042004E0207B0C28C1
:101CD00000D0FFDF052038736EE7FFDF6CE770B5DB
:101CE0000C46054601F0AFFB20B10078222804D253
:101CF000082070BD43F2020070BD0521284610F097
:101D00005DFF206008B1002070BD032070BD30B4BD
:101D10004880087820F00F00C01C20F0F0009030C0
:101D200001F8080B1DCA81E81D0030BC07F06DBC2E
:101D30002DE9FF4784B00027824602970798904616
:101D4000894612300AF025FA401D20F00306079854
:101D500028B907A95046FFF7C2FF002854D1B9F1AE
:101D6000000F05D00798017B19BB052504681BE00F
:101D700098F80000092803D00D2812D0FFDF46E0B4
:101D8000079903254868B0B3497B42887143914263
:101D900039D98AB2B3B2011D10F083FD0446078021
:101DA00002E0079C042508340CB1208810B1032DF3
:101DB00029D02CE00798012112300AF01CFAADF866
:101DC0000C00024602AB2946504608F0A4FA070070
:101DD00001D1A01C029007983A461230C8F80400BE
:101DE000A8F802A003A94046029B0AF011FAD8B154
:101DF0000A2817D200E006E0DFE800F00709141413
:101E0000100B0D141412132014E6002012E61120FA
:101E100010E608200EE643F203000BE6072009E671
:101E20000D2007E6032005E6BDF80C002346CDE9AA
:101E300000702A465046079900F017FD57B9032D48
:101E400008D10798B3B2417B406871438AB2011D43
:101E500010F03BFDB9F1000FD7D0079981F80C9035
:101E6000D3E72DE9FE4F91461A881C468A468046E4
:101E7000FAB102AB494608F04EFA050019D04046C7
:101E8000A61C278810F0DFFF3246072629463B466E
:101E9000009610F0ECFB20882346CDE900504A461E
:101EA0005146404600F0E1FC002020800120BDE8C2
:101EB000FE8F0020FBE710B586B01C46AAB10423B4
:101EC0008DF800301388ADF808305288ADF80A203C
:101ED0008A788DF80E200988ADF80C1000236A4628
:101EE0002146FFF725FF06B010BD1020FBE770B5B7
:101EF0000D46052110F062FE040000D1FFDF2946E7
:101F000004F11200BDE870400AF05EB92DE9F84313
:101F10000D468046002607F075FB044628781028F9
:101F200078D2DFE800F0773B345331311231313170
:101F30000831313131312879001FC0B2022801D077
:101F4000102810D114BBFFDF35E004B9FFDF0521F5
:101F5000404610F033FE007B032806D004280BD047
:101F6000072828D0FFDF072655E02879801FC0B258
:101F7000022820D050B1F6E72879401FC0B20228CD
:101F800019D0102817D0EEE704B9FFDF13E004B929
:101F9000FFDF287901280ED1172137E005214046BF
:101FA00010F00CFE070000D1FFDF07F112014046E0
:101FB0000AF0E7F82CB12A4621464046FFF7A7FE73
:101FC00029E01321404602F01DFD24E004B9FFDFA3
:101FD0000521404610F0F2FD060000D1FFDF694602
:101FE00006F112000AF0D7F8060000D0FFDFA9883A
:101FF000172901D2172200E00A46BDF800008242EC
:1020000002D9014602E005E01729C5D3404600F099
:102010003CFCD0E7FFDF3046BDE8F883401D20F0F0
:10202000030219B102FB01F0001D00E00020104482
:10203000704713B5009848B10024684610F0DBFBE8
:10204000002C02D1F74A009911601CBD0124002028
:10205000F4E72DE9F0470C461546242200212046DE
:102060000CF0CBF905B9FFDFA87860732888DFF89A
:10207000B4A3401D20F00301AF788946DAF80000D0
:1020800010F0D7FB060000D1FFDF4FF000082660FC
:10209000A6F8008077B109FB07F1091D0AD0DAF82C
:1020A000000010F0C6FB060000D1FFDF6660C6F836
:1020B000008001E0C4F80480298804F11200BDE822
:1020C000F0470AF04FB82DE9F047804601F11200C1
:1020D0000D4681460AF05DF8401DD24F20F0030204
:1020E0006E7B14462968386810F0CEFB3EB104FBC5
:1020F00006F2121D03D06968386810F0C5FB052090
:1021000010F004FD0446052010F008FD201A0128F7
:1021100002D1386810F082FB49464046BDE8F047DE
:102120000AF036B870B50546052110F047FD0400E9
:1021300000D1FFDF04F112012846BDE870400AF02B
:1021400020B82DE9F04F91B04FF0000BADF834B04E
:10215000ADF804B047880C4605469246052138463E
:1021600010F02CFD060000D1FFDF24B1A780A4F8F9
:1021700006B0A4F808B0297809220B20B2EB111F91
:102180007ED12A7A04F1100138274FF00C084FF065
:1021900001090391102A74D2DFE802F073F3F2F11F
:1021A0008008D3898EA03DDCF4EFB7B7307B0228DE
:1021B00000D0FFDFA88908EBC001ADF80410302182
:1021C000ADF83410002C25D06081B5F80E900027B2
:1021D0001DE004EBC708317C88F80E10F189A8F8DF
:1021E0000C10CDF800906888042304AA296900F037
:1021F0002CFBBDF81010A8F8101009F10400BDF870
:1022000012107F1C1FFA80F9A8F81210BFB2608963
:10221000B842DED80EE1307B022800D0FFDFE9892A
:1022200008EBC100ADF804003020ADF83400287B85
:102230000A90001FC0B20F90002CEBD06181B5F85E
:102240001090002726E000BFCDF8009068886969EB
:1022500003AA0A9B00F0F9FA0A9804EBC70848445D
:102260001FFA80F908F10C0204A90F9812F03EFA47
:1022700018B188F80EB0A8F80CB0BDF80C1001E049
:10228000D4E0D1E0A8F81010BDF80E107F1CA8F81B
:102290001210BFB26089B842D6D8CBE00DA800902A
:1022A00001AB224629463046FFF719FBC2E0307BDE
:1022B000082805D0FFDF03E0307B082800D0FFDFCF
:1022C000E8891030ADF804003620ADF83400002C59
:1022D0003FD0A9896181F189A18127E0307B09285C
:1022E00000D0FFDFA88900F10C01ADF80410372100
:1022F000ADF83410002C2CD06081E8890090AB89B7
:10230000688804F10C02296956E0E8893921103007
:1023100080B2ADF80400ADF83410002C74D0A98957
:102320006181287A0E280AD002212173E989E1818E
:10233000288A0090EB8968886969039A3CE001214A
:10234000F3E70DA8009001AB224629463046FFF77F
:1023500057FB6FE0307B0A2800D0FFDF1220ADF87A
:102360000400ADF834704CB3A9896181A4F810B0B1
:10237000A4F80EB084F80C905CE020E002E031E0BC
:1023800039E042E0307B0B2800D0FFDF288AADF82F
:1023900034701230ADF8040084B104212173A9898E
:1023A0006181E989E181298A2182688A00902B8AEA
:1023B000688804F11202696900F047FA3AE0307B5C
:1023C0000C2800D0FFDF1220ADF80400ADF8347007
:1023D0003CB305212173A4F80AB0A4F80EB0A4F808
:1023E00010B027E00DA8009001AB224629463046E8
:1023F000FFF75AFA1EE00DA8009001AB22462946CD
:102400003046FFF7B5FB15E034E03B21ADF80400A2
:10241000ADF8341074B3A4F80690A4F808B084F8AA
:102420000AB007E010000020FFDF03E0297A01294D
:1024300017D0FFDFBDF80400AAF800006CB1BDF8AA
:1024400034002080BDF804006080BDF834003928D5
:1024500003D03C2801D086F80CB011B00020BDE8B4
:10246000F08F3C21ADF80400ADF8341014B1697A56
:10247000A172DFE7AAF80000EFE72DE9F8435688DC
:102480000F46804615460521304610F097FB0400A4
:1024900000D1FFDF123400943B46414630466A6863
:1024A00009F0EAFFB8E570B50D46052110F086FB8E
:1024B000040000D1FFDF294604F11200BDE870409E
:1024C00009F074BE70B50D46052110F077FB0400CD
:1024D00000D1FFDF294604F11200BDE8704009F089
:1024E00092BE70B50546052110F068FB040000D1CE
:1024F000FFDF04F1080321462846BDE870400422AE
:10250000AFE470B50546052110F058FB040000D17A
:10251000FFDF214628462368BDE870400522A0E47D
:1025200070B50646052110F049FB040000D1FFDF1D
:1025300004F1120009F02DFE401D20F0030511E00A
:10254000011D00880322431821463046FFF789FC0D
:1025500000280BD0607BABB2684382B26068011D7B
:1025600010F0E9F9606841880029E9D170BD70B5C3
:102570000E46054607F046F8040000D1FFDF0120B3
:10258000207266726580207820F00F00C01C20F059
:10259000F00030302070BDE8704007F036B82DE90B
:1025A000F0438BB00D461446814606A9FFF797FB12
:1025B000002814D14FF6FF7601274FF420588CB134
:1025C00003208DF800001020ADF8100007A805903A
:1025D00007AA204604A912F0A8F878B107200BB08A
:1025E000BDE8F0830820ADF808508DF80E708DF826
:1025F0000000ADF80A60ADF80C800CE00698A178F8
:1026000001742188C1818DF80E70ADF80850ADF8C5
:102610000C80ADF80A606A4602214846069BFFF727
:1026200087FBDCE708B501228DF8022042F60202A2
:10263000ADF800200A4603236946FFF73CFC08BDBD
:1026400008B501228DF8022042F60302ADF8002001
:102650000A4604236946FFF72EFC08BD00B587B083
:1026600079B102228DF800200A88ADF80820498847
:10267000ADF80A1000236A460521FFF759FB07B0A1
:1026800000BD1020FBE709B1072314E407207047C1
:1026900070B588B00D461446064606A9FFF71FFB25
:1026A00000280ED17CB10620ADF808508DF800004E
:1026B000ADF80A40069B6A460821DC813046FFF7E8
:1026C00037FB08B070BD05208DF80000ADF808504C
:1026D000F0E700B587B059B107238DF80030ADF8A9
:1026E0000820039100236A460921FFF721FBC6E772
:1026F0001020C4E770B588B00C460646002506A930
:10270000FFF7EDFA0028DCD106980121123009F01C
:1027100072FD9CB12178062921D2DFE801F0200565
:1027200005160318801E80B2C01EE28880B20AB16E
:10273000A3681BB1824203D90C20C2E71020C0E776
:10274000042904D0A08850B901E00620B9E7012986
:1027500013D0022905D004291CD005292AD007202E
:10276000AFE709208DF800006088ADF80800E08828
:10277000ADF80A00A068039023E00A208DF800005D
:102780006088ADF80800E088ADF80A00A0680A2566
:10279000039016E00B208DF800006088ADF808006B
:1027A000A088ADF80A00E088ADF80C00A0680B2501
:1027B000049006E00C208DF8000060788DF8080089
:1027C0000C256A4629463046069BFFF7B1FA78E7A2
:1027D00000B587B00D228DF80020ADF80810002359
:1027E0006A461946FFF7A4FA49E700B587B071B108
:1027F00002228DF800200A88ADF808204988ADF83B
:102800000A1000236A460621FFF792FA37E71020E4
:1028100035E770B586B0064601200D46ADF80810C4
:102820008DF80000014600236A463046FFF780FA23
:10283000040008D12946304605F0DEFC0021304670
:1028400005F0F8FC204606B070BDF8B51C461546EC
:102850000E46069F10F0E5FA2346FF1DBCB2314636
:102860002A4600940FF0CFFEF8BD30B41146DDE9E2
:1028700002423CB1032903D0002330BC08F029BE3A
:102880000123FAE71A8030BC704770B50C46054644
:10289000FFF72DFB2146284605F0BDFC2846BDE884
:1028A0007040012105F0C6BC4FF0E0224FF400401B
:1028B0000021C2F88001BFF34F8FBFF36F8F17481D
:1028C000016001601649900208607047134900B525
:1028D00000220A600A60124B4FF060721A600028F2
:1028E00008BF00BD0F4A104BDFF840C001280CD0D4
:1028F00002281CBFFFDF00BD032008601A604FF4F0
:10290000000000BFCCF8000000BD022008601A6083
:102910004FF04070F6E700B5FFDF00BD00F5004066
:1029200008F50140A802002014F5004004F501401C
:1029300070B50B2000F0BDF9082000F0BAF90021B5
:102940000B2000F0D4F90021082000F0D0F9F44C5D
:1029500001256560A5600020C4F84001C4F8440169
:10296000C4F848010B2000F0B5F9082000F0B2F9D6
:102970000B2000F091F9256070BD10B50B2000F020
:1029800098F9082000F095F9E5480121416081603F
:10299000E4490A68002AFCD10021C0F84011C0F8BF
:1029A0004411C0F848110B2000F094F9BDE8104024
:1029B000082000F08FB910B50B2000F08BF9BDE8AE
:1029C0001040082000F086B900B530B1012806D0CB
:1029D000022806D0FFDF002000BDD34800BDD34849
:1029E00000BDD248001D00BD70B5D1494FF0004078
:1029F0000860D04DC00BC5F80803CF480024046020
:102A0000C5F840410820C43500F053F9C5F83C41F1
:102A1000CA48047070BD08B5C14A002128B1012818
:102A200011D002281CD0FFDF08BD4FF48030C2F85F
:102A30000803C2F84803BB483C300160C2F84011AB
:102A4000BDE80840D0E74FF40030C2F80803C2F8F0
:102A50004803B44840300160C2F84411B3480CE068
:102A60004FF48020C2F80803C2F84803AD48443050
:102A70000160C2F84811AD48001D0068009008BD13
:102A800070B516460D460446022800D9FFDF002225
:102A9000A348012304F110018B4000EB8401C1F82D
:102AA000405526B1C1F84021C0F8043303E0C0F816
:102AB0000833C1F84021C0F8443370BD2DE9F0411E
:102AC0001D46144630B1012833D0022838D0FFDF2C
:102AD000BDE8F081891E002221F07F411046FFF7FA
:102AE000CFFF012D23D00020944D924F0126687016
:102AF0003E61914900203C3908600220091D0860B0
:102B00008D490420303908608B483D34046008202A
:102B10006C6000F0DFF83004C7F80403082000F010
:102B2000BBF88349F007091F08602E70D0E7012029
:102B3000DAE7012B02D00022012005E00122FBE7A9
:102B4000012B04D000220220BDE8F04198E70122C9
:102B5000F9E774480068704770B500F0D8F8704C19
:102B60000546D4F840010026012809D1D4F808030D
:102B7000C00305D54FF48030C4F80803C4F84061A1
:102B8000D4F8440101280CD1D4F80803800308D5F7
:102B90004FF40030C4F80803C4F84461012012F077
:102BA0008BFDD4F8480101280CD1D4F80803400368
:102BB00008D54FF48020C4F80803C4F84861022007
:102BC00012F07AFD5E48056070BD70B500F09FF8A8
:102BD0005A4D0446287850B1FFF706FF687818B1BF
:102BE0000020687012F068FD5548046070BD032035
:102BF000F8E74FF0E0214FF40010C1F800027047F1
:102C0000152000F067B84B4901200861082000F04A
:102C100061B848494FF47C10C1F80803002002460F
:102C200001EB8003C3F84025C3F84021401CC0B22B
:102C30000628F5D37047410A43F609525143C0F3C1
:102C4000080010FB02F000F5807001EB5020704787
:102C500010B5430B48F2376463431B0C5C020C60F5
:102C6000384C03FB0400384B4CF2F72443435B0D14
:102C700013FB04F404EB402000F580704012107048
:102C800008681844086010BD2C48406870472949FE
:102C90000120C1F800027047002809DB00F01F0284
:102CA000012191404009800000F1E020C0F80011AE
:102CB000704700280DDB00F01F0201219140400900
:102CC000800000F1E020C0F88011BFF34F8FBFF308
:102CD0006F8F7047002809DB00F01F02012191402F
:102CE0004009800000F1E020C0F8801270474907D9
:102CF000090E002804DB00F1E02080F80014704782
:102D000000F00F0000F1E02080F8141D70470C481F
:102D1000001F00680A4A0D49121D1160704700002B
:102D200000B0004004B500404081004044B1004084
:102D300008F5014000800040408500403800002038
:102D400014050240F7C2FFFF6F0C010001000001F3
:102D50000A4810B50468094909480831086012F0AA
:102D60003FFD0648001D046010BD064900200860B4
:102D70004FF0E0210220C1F88002704710050240A8
:102D800001000001FC1F0040374901200860704726
:102D900070B50D2000F049F8344C0020C4F8000153
:102DA0000125C4F804530D2000F050F825604FF0C1
:102DB000E0216014C1F8000170BD10B50D2000F0D5
:102DC00034F82A48012141600021C0F80011BDE813
:102DD00010400D2000F03AB8254810B50468244989
:102DE0002448083108602149D1F80001012804D0A5
:102DF000FFDF1F48001D046010BD1B48001D006858
:102E00000022C0B2C1F8002113F0A3F9F1E710B518
:102E1000164800BFD0F800110029FBD0FFF7DCFFF7
:102E2000BDE810400D2000F011B800280DDB00F0C7
:102E30001F02012191404009800000F1E020C0F80C
:102E40008011BFF34F8FBFF36F8F7047002809DBEE
:102E500000F01F02012191404009800000F1E020B4
:102E6000C0F880127047000004D5004000D0004038
:102E700010050240010000014FF0E0214FF000700A
:102E8000C1F8800101F5C071BFF34F8FBFF36F8FA1
:102E9000C1F80001394B802283F8002441F8800CEE
:102EA000704700B502460420354903E001EBC0033A
:102EB0001B792BB1401EC0B2F8D2FFDFFF2000BD4E
:102EC00041F8302001EBC00100224A718A710122D1
:102ED0000A7100BD2A4A002102EBC000017170474F
:102EE00010B50446042800D3FFDF254800EBC404D6
:102EF0002079012800D0FFDF6079A179401CC0B2A1
:102F0000814200D060714FF0E0214FF00070C1F8B5
:102F1000000210BD70B50425194E1A4C16E0217838
:102F200006EBC1000279012A08D1427983799A42DD
:102F300004D04279827156F8310080472078401CD5
:102F4000C0B22070042801D3002020706D1EEDB2A5
:102F5000E5D270BD0C4810B504680B490B48083128
:102F60000860064890F800044009042800D0FFDFFC
:102F7000FFF7D0FF0448001D046010BD19E000E019
:102F8000E00500205400002010050240010000016F
:102F90000548064A0168914201D1002101600449B7
:102FA000012008607047000058000020BEBAFECA29
:102FB00040E5014070B50C46054609F0F9FB214695
:102FC0002846BDE870400AF0DABC002A14BF4FF46E
:102FD00029614FF4A471002B14BF4FF429624FF400
:102FE000A47200280CBF0120002011449831002851
:102FF00018BF0420084470477047704770470000AE
:103000002CFFFFFFDBE5B15100600200CB00FFFFAA
:1030100084000000C1CF6A00FEA0D9111C1006C3B5
:1030200089CCFC7A7B3B49141906A8C030B5F84D11
:103030000446062CA9780ED2DFE804F0030E0E0E2B
:103040000509FFDF08E0022906D0FFDF04E00329BD
:1030500002D0FFDF00E0FFDFAC7030BD30B50446CA
:103060001038EB4D07280CD2DFE800F0040C060CFA
:103070000C0C0C00FFDF05E0287E112802D0FFDFDA
:1030800000E0FFDF2C7630BD2DE9F04111F0B8FCF7
:10309000044612F0EBFE201AC5B206200FF036FDF2
:1030A000044606200FF03AFD211AD94C207E122842
:1030B00018D000200F1807200FF028FD0646072023
:1030C0000FF02CFD301A3918207E13280CD0002068
:1030D0000144A078042809D000200844281AC0B26E
:1030E000BDE8F0810120E5E70120F1E70120F4E7E8
:1030F000C74810B590F825004108C54800F12600E2
:1031000005D00DF017FEBDE8104006F09DB80DF09B
:10311000F2FDF8E730B50446A1F120000D460A287B
:103120004AD2DFE800F005070C1C2328353A3F445B
:10313000FFDF42E0207820283FD1FFDF3DE0B448A8
:103140008178052939D0007E122836D020782428AD
:1031500033D0252831D023282FD0FFDF2DE0207851
:1031600022282AD0232828D8FFDF26E0207822280A
:1031700023D0FFDF21E0207822281ED024281CD075
:1031800026281AD0272818D0292816D0FFDF14E0C7
:103190002078252811D0FFDF0FE0207825280CD0DB
:1031A000FFDF0AE02078252807D0FFDF05E0207840
:1031B000282802D0FFDF00E0FFDF257030BD1FB5FB
:1031C00004466A46002001F09DFEB4B1BDF802201D
:1031D0004FF6FF700621824201D1ADF80210BDF812
:1031E0000420824201D1ADF80410BDF808108142DC
:1031F00003D14FF44860ADF8080068460EF07EF940
:1032000006F022F804B010BD70B514460D4606460F
:10321000FEF71FF858B90DB1A54201D90C2070BDB9
:10322000002408E056F82400FEF713F808B1102037
:1032300070BD641CE4B2AC42F4D3002070BD2DE933
:10324000F04105461F4690460E4600240068FEF7F2
:103250004DF830B9A98828680844401EFEF746F8A2
:1032600008B110203CE728680028A88802D0B8429E
:1032700002D850E00028F5D0092031E72968085D20
:10328000B8B1671CCA5D152A2ED03CDC152A3AD28B
:10329000DFE802F03912222228282A2A313139396E
:1032A00039393939393939392200085D30BB641C64
:1032B000A4B2A242F9D833E00228DDD1A01C085CF8
:1032C00088F80000072801D2400701D40A2007E748
:1032D000307840F0010015E0C143C90707E001283C
:1032E00007D010E00620FBE60107A1F1805100297C
:1032F000F5D01846F4E63078810701D50B20EFE6CB
:1033000040F0020030702868005D384484B2A8881C
:10331000A04202D2B0E74FF4485382B2A242ADD8E5
:103320000020DDE610B5027843F2022354080122A2
:10333000022C12D003DC3CB1012C16D106E0032C88
:1033400010D07F2C11D112E0002011E080790324ED
:10335000B4EB901F09D10A700BE08079B2EB901F9B
:1033600003D1F8E780798009F5D0184610BDFF2019
:103370000870002010BD08B500208DF8000024481A
:1033800090F82E1049B190F82F0002280ED0032893
:103390000ED0FFDF9DF8000008BD1D4869462530AE
:1033A00001F0FFFD0028F5D0FFDFF3E7032000E088
:1033B00001208DF80000EDE738B50C46054669465A
:1033C00001F0EFFD00280DD19DF80010207861F389
:1033D0004700207055F8010FC4F80100A888A4F830
:1033E0000500002038BD38B51378A8B1022813D0E5
:1033F000FF281AD007A46D46246800944C7905EB89
:103400009414247864F347031370032809D00FE061
:10341000F40100200302FF0123F0FE0313700228D1
:10342000F3D1D8B240F0010005E043F0FE00107087
:10343000107820F0010010700868C2F80100888838
:10344000A2F8050038BD02210FF0B8BB38B50C4614
:103450000978222901D2082038BDADF800008DF886
:10346000022068460DF0A8FC05F0EEFE050003D131
:1034700021212046FFF74EFE284638BD1CB500200E
:103480008DF80000CDF80100ADF80500FE4890F879
:103490002E00022801D0012000E000208DF8070056
:1034A00068460DF00FFD002800D0FFDF1CBD002294
:1034B0000A80437892B263F3451222F040020A80F8
:1034C00000780C282BD2DFE800F02A06090E11162E
:1034D000191C1F220C2742F0110009E042F01D00C8
:1034E00008800020704742F0110012E042F0100006
:1034F00040F00200F4E742F01000F1E742F0010072
:10350000EEE742F0010004E042F00200E8E742F09A
:10351000020040F00400E3E742F00400E0E7072087
:1035200070472DE9FF478AB00025BDF82C60824620
:103530001C4690468DF81C50700703D56068FDF757
:1035400088FE68B9D04F4FF0010997F82E0058B1A6
:1035500097F82F00022807D16068FDF7C7FE18B161
:1035600010200EB0BDE8F087300702D5A089802872
:1035700016D8700705D4B8F1000F02D097F82400D0
:1035800070B1E07DC0F300108DF81B00617D072055
:1035900041B1012906D00229E3D00429E1D12CE070
:1035A0000720DEE749468DF81790F00609D4A27D82
:1035B000072032B1012A04D0022A05D0042AD0D132
:1035C0001BE08DF8191002E002208DF819008DF82B
:1035D00015806068B0B107A9FFF7A4FE0028C0D12C
:1035E0009DF81C00FF280AD0606850F8011FCDF834
:1035F0000F108088ADF8130008E00620B1E743F211
:103600000220AEE7CDF80F50ADF81350E07B002854
:10361000F3D1207C0028F0D1607C0028EDD1A07C83
:103620000028EAD1E07CC006E7D18DF800A0BDF803
:103630002C00ADF80200A0680190A068029004F18F
:103640000F0001F0A2FC8DF80C00FFF794FE8DF83E
:103650000D009DF81C008DF80E008DF816508DF8A9
:103660001850E07D08A900F00F008DF81A00684698
:103670000EF08CF805F0E8FD73E7F0B58FB000258B
:103680008DF830508DF814508DF8345006468DF872
:103690002850019502950395049519B10FC901AC05
:1036A00084E80F00784CA078052801D004280CD1BC
:1036B00001986168884200D120B90398E168884286
:1036C00003D110B108200FB0F0BD207DC00601D598
:1036D0001F2700E0FF273B460DAA05A903A8FFF717
:1036E000AEFD0028EFD1A08AC10702D0C00600D4E9
:1036F000EE273B460AAA0CA901A8FFF7A0FD002867
:10370000E1D19DF81400C00701D00A20DBE7A08AB0
:10371000410708D4A17D31B19DF82810890702D056
:1037200043F20120CFE79DF82810C90709D04007D0
:1037300007D4208818B144F25061884201D907208B
:10374000C1E78DF818508DF81960BDF80800ADF884
:103750001A000198079006A80EF024F805F074FDF1
:103760000028B0D18DF820508DF82160BDF81000F0
:10377000ADF822000398099008A80EF035F805F07E
:1037800063FD00289FD101AD241D95E80F0084E85A
:103790000F00002097E770B586B00D46040005D0F5
:1037A000FDF7A4FD20B1102006B070BD0820FBE796
:1037B0002078C107A98802D0FF2902D303E01F297E
:1037C00001D20920F0E780073BD4FFF75DFC38B158
:1037D0002178C1F3C100012804D0032802D005E0FC
:1037E0001320E1E7284890F82400C8B1C8074FF03B
:1037F00001064FF0000502D08DF80F6001E08DF852
:103800000F50FFF7B8FD8DF8000020786946C0F32F
:10381000C1008DF8010060788DF80250C20801D017
:103820000720C1E778B1C20701D08DF80260820796
:1038300005D59DF8022042F002028DF802204007D3
:1038400003D50620B0E78DF80260002022780B181F
:10385000C2F38002DA7001EB40026388D380401C1F
:10386000A388C0B253810228F0D3207A0028E8D17F
:10387000607A0028E5D1A07A0028E2D1E07A002819
:10388000DFD1207BC00601E0F4010020D9D104F192
:10389000080001F07AFB8DF80E0068460DF0DFFBA2
:1038A00005F0D2FC00288DD18DF810608DF81150F4
:1038B000E088ADF81200ADF8145004A80DF022FC19
:1038C00005F0C2FC00288CD12078C00701D015205B
:1038D00000E01320FFF7C2FB002065E72DE9FF475A
:1038E0000220FD4E8DF804000027708EADF8060012
:1038F000B84643F202094CE001A80FF0C6F80500F3
:1039000006D0708EA8B3A6F83280ADF806803EE0EF
:10391000039CA07F01072DD504F124000090A28E06
:10392000BDF80800214604F1360301F0C5FC05008E
:1039300005D04D452AD0112D3CD0FFDF3AE0A07FC5
:1039400020F00801E07F420862F3C711A1778108E7
:1039500061F30000E07794F8210000F01F0084F884
:1039600020002078282826D129212046FFF7D2FBE5
:1039700021E014E040070AD5BDF8080004F10E016B
:1039800001F019FB05000DD04D4510D100257F1C1D
:10399000FFB202200FF0BAF8401CB842ACD8052D97
:1039A00011D008E0A07F20F00400A07703E0112DE3
:1039B00000D0FFDF0025BDF806007086052D04D07D
:1039C000284604B0CEE5A6F832800020F9E770B5AD
:1039D0000646FFF738FD054605F014FE040000D149
:1039E000FFDF6680207820F00F00801C20F0F000C0
:1039F000203020700320207295F83E006072BDE8F0
:103A0000704005F002BE2DE9F04786B0040000D1F9
:103A1000FFDF2078B04D20F00F00801C20F0F00078
:103A20007030207060680178491F1B2933D2DFE8AD
:103A300001F0FC32323255FB320EFBFB42FA3232DD
:103A40003278FAFAF9F832FAFAF7F6FAFA00C68892
:103A50003046FFF7F8FC0546304607F030FCE0B191
:103A60006068007A85F83E0021212846FFF752FB66
:103A70003046FEF757FB304603F0E2FE31460120A8
:103A800012F02CFEA87F20F01000A877FFF726FF89
:103A9000002800D0FFDF06B064E5207820F0F000B9
:103AA000203020700320207266806068007A607287
:103AB00005F0ABFDD8E7C5882846FFF7C4FC00B980
:103AC000FFDF60680079012800D0FFDF6068017ABD
:103AD00006B02846BDE8F04707F0D6BDC688304698
:103AE000FFF7B1FC050000D1FFDF05F08EFD606837
:103AF00031460089288160684089688160688089D2
:103B0000A881012012F0EAFD0020A875A87F00F02E
:103B100003000228BFD1FFF7E1FE0028BBD0FFDF82
:103B2000B9E7007928B10228B5D03C28B3D0FFDF2F
:103B3000B1E705F06AFD6668B6F806A0307A361D72
:103B4000012806D0687E814605F0EAFA070003D115
:103B500001E0E878F7E7FFDF0022022150460FF08E
:103B600024F8040000D1FFDF22212046FFF7D2FA1B
:103B70003079012800D00220A17F804668F301013E
:103B8000A177308B2081708B6081B08BA08184F80D
:103B900022908DF80880B8680090F86801906A4615
:103BA000032150460FF001F800B9FFDFB888ADF8E7
:103BB0001000B8788DF8120004AA052150460EF0C6
:103BC000F4FF00B9FFDFB888ADF80C00F8788DF885
:103BD0000E0003AA042150460EF0E7FF00B9FFDFF4
:103BE000062106F1120001F004FA40B37079800753
:103BF00000D5FFDF7179E07D61F34700E075D6F80D
:103C00000600A0617089A083062106F10C0001F076
:103C1000F0F9F0B195F825004108607806E043E03E
:103C20003BE072E05AE04FE031E045E061F34700ED
:103C30006070D5F82600C4F80200688D12E0E07DBF
:103C400020F0FE00801CE075D6F81200A061F08A1A
:103C5000D9E7607820F0FE00801C6070F068C4F83E
:103C60000200308AE080B8F1010F04D0B8F1020FF1
:103C700005D0FFDF0FE70320FFF7D8F90BE7287E19
:103C8000122800D0FFDF1120FFF7E8F903E706B0A4
:103C90002046BDE8F04701F09BBD05F0B6FC15F8E5
:103CA000300F40F0020005E005F0AFFC15F8300FD2
:103CB00040F004002870EEE6287E132809D015286D
:103CC000D8D11620FFF7CAF906B0BDE8F04705F0D5
:103CD0009CBC1420F6E70000F4010020A978052917
:103CE00009D00429C6D105F090FC022006B0BDE839
:103CF000F047FFF79BB900790028BBD0E87801F0C6
:103D00002BF905F082FC0320F0E7287E122802D16F
:103D1000687E01F021F91120D4E72DE9F05F054616
:103D200000784FF000080009DFF8B4A891460C466F
:103D3000464601286ED002286DD007280BD00A28ED
:103D40006AD0FFDFA9F8006014B1A4F80080668093
:103D50000020BDE8F09F6968012704F108000B7896
:103D60004FF0020B5B1F4FF6FF721B2B7ED2DFE87A
:103D700003F0647D7D7D0E7D7D7D7D7D7D217D7D5E
:103D80007D2BFDFCFBFA7D14D2F9E7F8F700C8881B
:103D90004FF01208102621469AE14FF01C080A261F
:103DA000BCB38888A0806868807920726868C07910
:103DB0006072C7E74FF01B08142654B3032020722B
:103DC00068688088A080BDE70A793C2ABAD00D1DBA
:103DD0004FF010082C26E4B16988A180298B6182FC
:103DE000298B2182698BA182A98BE1826B790246A2
:103DF000A91D1846FFF7F7FA2979002001290CD0F0
:103E000084F80FB0FF212176E06120626062A06239
:103E100098E70FE03BE15EE199E1E77320760AF174
:103E2000040090E80E00DAF81000C4E90930C4E993
:103E3000071287E7A9F800608AE72C264FF01D08D3
:103E4000002CF7D0A28005460F1D897B008861F306
:103E500000002880B97A490861F341002880B97AC6
:103E6000890861F382002880B97A00E00CE1C90872
:103E700061F3C3002880B97AAA1C0911491C61F3B7
:103E8000041000F07F0028807878B91CFFF7ABFAA7
:103E9000387D05F1090207F11501FFF7A4FA387B17
:103EA00001F0B6F82874787B01F0B2F86874F87EF7
:103EB000A874787AE874387F2875B87B6875388A72
:103EC000E882DAF81C10A961B97A504697F808A080
:103ED000C1F34111012904D0008C504503D2824620
:103EE00009E0FFDF10E0022903D0288820F06000FD
:103EF00009E0504504D1288820F06000403002E0FD
:103F0000288840F060002880A4F824A0524607F1D9
:103F10001D01A8699BE011264FF02008002C89D0D4
:103F2000A280686804F10A02007920726868007B48
:103F3000607269688B1D48791946FFF754FA01E7EA
:103F40000A264FF02108002CE9D08888A0806868F4
:103F5000807920726868C07960729AF8301006E043
:103F600078E06BE052E07FE019E003E03AE021F016
:103F70000401A6E00B264FF02208002CCFD0C88801
:103F8000A0806868007920726868007A01F040F8C3
:103F900060726868407A01F03BF8A072D2E61C2695
:103FA0004FF02608002CBAD0A28068684079607271
:103FB0006868007AA0720AF1040090E80E00DAF84E
:103FC0001000C4E90530C4E90312686800793C2890
:103FD00003D0432803D0FFDFB4E62772B2E684F8AB
:103FE00008B0AFE610264FF02408002C97D0888840
:103FF000A0806868807920816868807A60816868BC
:104000000089A08168688089E0819BE610264FF0D6
:104010002308002C98D08888A0806868C0882081F8
:1040200068680089608168684089A08168688089C3
:10403000E0819AF8301021F0020142E030264FF082
:104040002508002C9AD0A2806968282249680AF0C5
:10405000AAF977E62A264FF02F08002C8ED0A280EE
:1040600069682222091DF2E714264FF01B08002C74
:1040700084D0A280686800790128B0D02772DAE97C
:104080000710C4E903105DE64A46214660E0287A3D
:10409000012803D0022817D0FFDF53E610264FF087
:1040A0001F08002CA2D06888A080A8892081E889F8
:1040B0006081288AA081688AE0819AF8301021F016
:1040C00001018AF830103DE64FF01208102668888A
:1040D00000F07CFF36E6287AC8B3012838D00228E1
:1040E00036D0032801D0FFDF2CE609264FF0110857
:1040F000002C8FD06F883846FFF7A5F990F822A0E2
:10410000A780687A2072042138460EF069FD0521E7
:1041100038460EF065FD002138460EF061FD0121A4
:1041200038460EF05DFD032138460EF059FD0221A0
:1041300038460EF055FD062138460EF051FD072198
:1041400038460EF04DFD504600F006FFFAE5FFE759
:104150002846BDE8F05F01F0C5BC70B5012803D06A
:10416000052800D0FFDF70BD8DB22846FFF76BF940
:10417000040000D1FFDF20782128F4D005F042FAB6
:1041800080B1017821F00F01891C21F0F00110317C
:1041900001700221017245800020A075BDE87040C9
:1041A00005F033BA21462846BDE870401322FFF7D8
:1041B0004DB92DE9F04116460C00804600D1FFDFD5
:1041C000307820F00F00801C20F0F00010303070AC
:1041D0002078012804D0022818D0FFDFBDE8F08144
:1041E0004046FFF730F9050000D1FFDF0320A87536
:1041F00005F00BFA94E80F00083686E80F00F8483F
:1042000010F8301F41F001010170E7E74046FFF769
:104210001AF9050000D1FFDFA1884FF6FF700027D3
:10422000814202D1E288824203D0814201D1E088FA
:1042300040B105F0EAF994E80F00083686E80F006F
:10424000AF75CBE7A87D0128C8D17823002241466D
:1042500012F09AF90220A875C0E738B505460C4659
:104260000846FCF7F6FF70BB232D4AD006DC202D54
:104270000DD0212D23D0222D06D13DE0242D46D076
:10428000252D32D03F2D47D00725284638BD0021A7
:10429000052012F0F9F908B1112038BDA01C0DF06D
:1042A00080F904F0D1FF0500EFD100220823114668
:1042B000052012F069F90528E7D0FFDFE5E760681F
:1042C000FDF70BF808B1102038BD618820886A46D8
:1042D0000DF01BFC04F0B8FF0500D6D16068002883
:1042E000D3D0BDF800100180CFE7A07800F0010125
:1042F00020880DF03BFC17E0206801F09FFE05468A
:10430000C3E7207800F001000CF0E8FC0CE06188C5
:1043100020880DF076FB07E0207800F001008DF892
:10432000000068460CF0A5FF04F08EFFE7E770B5CB
:1043300005460C460846FCF7B2FF08B1102070BDD8
:10434000202D07D0212D0DD0222D0BD0252D09D0C9
:10435000072070BD2088A11C0CF092FDBDE87040C4
:1043600004F072BF062070BD9D482530704708B527
:10437000342200219A480AF040F80120FEF756FE48
:104380001120FEF76BFE96496846263105F0D0F8FD
:1043900093489DF8002010F8251F62F3470121F093
:1043A00001010170002141724FF46171A0F8071002
:1043B00002218172FEF79CFE00B1FFDFFDF712F8CB
:1043C00001F0CFF908BD10B50C464022002120466F
:1043D0000AF013F8A07F20F00300A07720202070BF
:1043E0000020A07584F8230010BD70472DE9FC4122
:1043F0000746FCF72EFF10B11020BDE8FC81784E77
:1044000006F12501D6F825000090B6F82950ADF840
:10441000045096F82B408DF806403846FEF7CCFF46
:104420000028EAD1FEF764FE0028E6D0009946F89D
:10443000251FB580B471E0E710B50446FCF72FFFE7
:1044400008B1102010BD66486549224690F8250045
:1044500026314008FEF7C7FF002010BD3EB50446D8
:104460000D460846FCF71BFF08B110203EBD14B1F5
:1044700043F204003EBD5A488078052803D0042842
:1044800001D008203EBD694602A80AF0BEFB2A46BC
:1044900069469DF80800FEF7A6FF00203EBDFEB568
:1044A0000D4604004FF0000711D00822FEF7ACFEC5
:1044B000002811D1002608E054F826006946FEF7CE
:1044C00031FF002808D1761CF6B2AE42F4D30CF0CE
:1044D0004FFB10B143F20320FEBD414E86F824701D
:1044E0000CB300271BE000BF54F8270002A9FEF719
:1044F00019FF00B1FFDF9DF808008DF8000054F8A7
:10450000270050F8011FCDF801108088ADF8050094
:1045100068460CF052FB00B1FFDF7F1CFFB2AF42D8
:10452000E2D386F824500020FEBD2DE9F0478AB082
:104530001546894604001FD00F4608222946FEF77B
:1045400063FE002811D1002614E000BF54F82600B5
:104550006946103000F025FD002806D147B157F814
:104560002600FCF776FE18B110200AB0BDE8F087EF
:10457000761CF6B2AE42E9D30026A5F101081BE095
:1045800006F1010A0AF0FF0712E000BF54F8260006
:10459000017C4A0854F827100B7CB2EB530F05D16D
:1045A00006221130113109F0D1FE58B17F1CFFB243
:1045B000AF42EBD30AF0FF064645E1DB4E4624B19D
:1045C000012003E043F20520CFE700200CF01AFBA6
:1045D00010B90CF023FB28B143F20420C5E700001A
:1045E000F401002064B300270DF1170826E000BF96
:1045F00054F827006946103000F0D3FC00B1FFDF0B
:1046000054F82700102250F8111FCDF801108088AF
:10461000ADF8050054F827100DF1070009F0C3FEAE
:1046200096B156F827101022404609F0BCFE6846A5
:104630000CF0A8FA00B1FFDF7F1CFFB2AF42D7D366
:10464000FEF71CFF002090E7404601F0EBFCEEE790
:1046500030B585B00446FDF7C5F830B906200EF038
:1046600055FA10B1062005B030BD2046FCF7F1FD2B
:1046700018B96068FCF73AFE08B11020F3E76088CB
:104680004AF2B811884206D82078F94D28B101289D
:1046900006D0022804D00720E5E7FEF729FD18E040
:1046A0006078022804D0032802D043F20220DAE71F
:1046B00085F82F00C1B200200090ADF80400022957
:1046C0002CD0032927D0FFDF68460CF033FB04F021
:1046D000BBFD0028C7D1606801F097FC207858B175
:1046E00001208DF800000DF1010001F09BFC6846EF
:1046F0000DF0A1FA00B1FFDF207885F82E00FEF75B
:10470000BDFE608860B1A88580B20CF073FA00B17C
:10471000FFDF0020A7E78DF80500D5E74020FAE786
:104720004FF46170EFE710B50446FCF7B8FD20B90F
:10473000606838B1FCF7D1FD08B1102010BD606889
:1047400001F070FCCA4830F82C1F6180C17861709C
:1047500080782070002010BD2DE9F843144689466A
:104760000646FCF79CFDA0B94846FCF7BFFD80B9A2
:104770002046FCF7BBFD60B9BD4DA878012800D1EB
:104780003CB13178FF2906D049B143F20400BDE8BD
:10479000F8831020FBE7012801D00420F7E7CCB311
:1047A000052811D004280FD069462046FEF77FFE69
:1047B0000028ECD1217D49B1012909D0022909D075
:1047C000032909D00720E2E70820E0E7024604E0D9
:1047D000012202E0022200E003228046234617461F
:1047E00000200099FEF79DFE0028D0D1A0892880E6
:1047F000A07BE875BDF80000A882AF75BDF8001079
:10480000090701D5A18931B1A1892980C00704D048
:10481000032003E006E08021F7E70220FEF706FC14
:1048200086F800804946BDE8F8430020FEF725BF22
:104830007CB58F4C05460E46A078022803D003288D
:1048400001D008207CBD15B143F204007CBD0720D7
:104850000EF064F910B9A078032806D0FEF714FC16
:1048600028B1A078032804D009E012207CBD1320D1
:104870007CBD304600F053FB0028F9D1E670FEF70E
:104880007AFD0AF0FFF801208DF800008DF8010094
:104890008DF802502088ADF80400E07D8DF8060008
:1048A00068460DF071F804F0CFFC0028E0D1A07844
:1048B000032805D05FF00400FEF7B8FB00207CBDA4
:1048C000E07800F03CFB0520F6E71CB510B143F2A0
:1048D00004001CBD664CA078042803D0052801D034
:1048E00008201CBD00208DF8000001218DF801106A
:1048F0008DF8020068460DF047F804F0A5FC00288A
:10490000EFD1A078052805D05FF00200FEF78EFBFE
:1049100000201CBDE07800F01FFB0320F6E72DE926
:10492000FC4180460E4603250846FCF7DFFC0028C4
:1049300066D14046FEF787FD040004D02078222887
:1049400004D2082059E543F2020056E5A07F00F0AA
:1049500003073EB1012F0CD000203146FEF72FFC9B
:104960000500EFD1012F06D0022F1AD0FFDF284615
:1049700043E50120F1E7A07D3146022801D011B1C5
:1049800007E0112039E56846FCF760FE0028D9D120
:104990006946404606F03BFE0500E8D10120A075BF
:1049A000E5E7A07D032804D1314890F83000C00726
:1049B00001D02EB30EE026B1A07F40071ED4002107
:1049C00000E00121404606F042FE0500CFD1A0756F
:1049D000002ECCD03146404600F0EDFA05461128B5
:1049E000C5D1A07F4107C2D4316844F80E1F716859
:1049F000616040F0040020740025B8E71125B6E797
:104A00001020FAE470B50C460546FEF71CFD0100C7
:104A100005D022462846BDE87040FEF717BD43F298
:104A2000020070BD10B5012807D1114B9B78012BF6
:104A300000D011B143F2040010BD0CF00DF9BDE837
:104A4000104004F001BC012300F090BA00231A4684
:104A5000194600F08BBA70B506460C460846FCF7BE
:104A6000F8FB18B92068FCF71AFC18B1102070BDCB
:104A7000F4010020F84D2A7E112A04D0132A00D315
:104A80003EB10820F3E721463046FEF784FE60B1D0
:104A9000EDE70920132A0DD0142A0BD0A188FF2995
:104AA000E5D31520FEF7DAFA0020D4E90012C5E9B3
:104AB0000712DCE7A1881F29D9D31320F2E71CB520
:104AC000E548007E132801D208201CBD00208DF887
:104AD000000068460CF016FB04F0B6FB0028F4D189
:104AE0001120FEF7BBFA00201CBD2DE9F04FDFF8C6
:104AF00068A3814691B09AF818009B4615460C466B
:104B0000132803D3FFF7DBFF00281FD12046FCF753
:104B1000A0FB78BB2846FCF79CFB58BB20784FF0E5
:104B20000107C0074FF0000102D08DF83A7001E094
:104B30008DF83A1020788846C0F3C1008DF8000047
:104B400060788DF80910C10803D0072011B0BDE8C6
:104B5000F08F80B1C10701D08DF80970810705D5AC
:104B60009DF8091041F002018DF80910400704D5A5
:104B70000620EBE720E08DF809709DF80900810719
:104B800003D540F001008DF8090000206E4606EBC9
:104B9000400162884A81401CA288C0B20A82032870
:104BA000F5D32078C0F3C100012821D003281FD0FD
:104BB0004846FCF74EFB08B11020C7E799F8000003
:104BC000400808D0012809D0022807D0032805D0C2
:104BD00043F20220BAE78DF8028001E08DF80270FE
:104BE000484650F8011FCDF803108088ADF8070043
:104BF000FEF7C1FB8DF801000020424606EB4001A4
:104C00002B88CB826B888B83AB884B84EB880B859E
:104C1000401CCA85C0B28A860328EFD3E088ADF86D
:104C20003C0068460CF01BFB00288ED19AF8180057
:104C30005546112801D0082088E706200DF06EFFA8
:104C400038B12078C0F3C100012804D0032802D075
:104C500006E012207AE795F8240000283FF475AFAB
:104C6000FEF712FA022801D213206FE7584600F02F
:104C700056F90028A1D185F819B068460CF018FC47
:104C800004F0E2FA040098D1687E00F058F912208E
:104C9000FEF7E4F9204659E770B56F4D287E1228DB
:104CA00001D00820E3E60CF006FC04F0CDFA040085
:104CB00005D1687E00F050F91120FEF7CFF92046AB
:104CC000D5E670B5064615460C460846FCF7E7FAE9
:104CD00018B92846FCF7E3FA08B11020C7E62A46BF
:104CE000214630460CF0F1FE04F0AEFA0028F5D172
:104CF00021787F29F2D10520B9E67CB505460C461E
:104D00000846FCF7A6FA08B110207CBD2846FEF73D
:104D10009AFB20B10078222804D208207CBD43F2FF
:104D200002007CBD4C4890F83000400701D51120AE
:104D30007CBD2178C80802D16078C20801D0072064
:104D40007CBD890801D1800801D006207CBDADF86A
:104D5000005020788DF8020060788DF80300022062
:104D6000ADF8040068460BF06CFD04F06DFA7CBDF4
:104D700070B586B014460D460646FEF764FB28B1B2
:104D80000078222805D2082006B070E643F202001F
:104D9000FAE72846FCF7AAFA20B944B12046FCF706
:104DA0009CFA08B11020EFE700202060A0802A487C
:104DB00090F83000800701D51120E5E703A93046BF
:104DC0000BF07CFD18B100BF04F03EFADCE7ADF853
:104DD0000060BDF81400ADF80200BDF81600ADF893
:104DE0000400BDF81000BDF81210ADF80600ADF8D3
:104DF00008107DB1298809B1ADF80610698809B19C
:104E0000ADF80210A98809B1ADF80810E98809B118
:104E1000ADF80410DCB1BDF80610814201D9081AC2
:104E20002080BDF80210BDF81400814201D9081A93
:104E30006080BDF80800BDF80410BDF816200144DC
:104E4000BDF812001044814201D9081AA0806846BA
:104E50000BF002FEB8E70000F40100201CB5724917
:104E60000968CDE9001068460CF0FBF904F0ECF994
:104E70001CBD1CB500200090019068460CF0F1F9B3
:104E800004F0E2F91CBD70B505460C460846FCF777
:104E900006FA08B11020EAE5214628460CF03AF857
:104EA000BDE8704004F0D0B93EB505460C46084652
:104EB000FCF7F5F908B110203EBD002000900190EC
:104EC0000290ADF800502089ADF8080020788DF8E8
:104ED0000200606801902089ADF808006089ADF893
:104EE0000A0068460CF028F804F0AEF93EBD0EB595
:104EF000ADF800000020019068460CF01DF804F0A9
:104F0000A3F90EBD10800888508048889080C8881A
:104F100010818888D080002050819081704710B522
:104F2000044604F0FDF830B1407830B1204604F07A
:104F300010FC002010BD052010BD122010BD10B5C2
:104F400004F0EEF8040000D1FFDF607800B9FFDF65
:104F50006078401E607010BD10B504F0E1F80400E8
:104F600000D1FFDF6078401C607010BD1CB5ADF84B
:104F700000008DF802308DF803108DF8042068468B
:104F80000CF066FD04F060F91CBD0CB527A2D2E957
:104F90000012CDE900120079694601EB501000784B
:104FA0000CBD0278520804D0012A02D043F202203C
:104FB0007047FEF7B7B91FB56A46FFF7A3FF68460B
:104FC0000CF0ACFA04F040F904B010BD70B50C0060
:104FD00006460DD0FEF737FA050000D1FFDFA680A8
:104FE00028892081288960816889A081A889E08139
:104FF0003DE510B500231A4603E0845C2343521CB0
:10500000D2B28A42F9D30BB1002010BD012010BDED
:1050100000B530B1012803D0022801D0FFDF002005
:1050200000BDFF2000BD0000485502000706050432
:105030000302010010B50446FCF70BF908B110207B
:1050400010BD2078C0F30210042807D86078072824
:1050500004D3A178102901D8814201D2072010BDC4
:10506000E078410706D421794A0703D4000701D428
:10507000080701D5062010BD002010BD10B513781B
:105080005C08837F64F3C713837713789C08C37F1E
:1050900064F30003C3771078C309487863F34100D1
:1050A000487013781C090B7864F347130B7013785E
:1050B000DB0863F3000048705078487110BD10B5EC
:1050C000C4780B7864F300030B70C478640864F34D
:1050D00041030B70C478A40864F382030B70C47896
:1050E000E40864F3C3030B700379117863F30001E0
:1050F000117003795B0863F34101117003799B0818
:1051000063F3820111700079C00860F3C30111706C
:1051100010BD70B514460D46064604F073FA80B112
:105120000178182221F00F01891C21F0F001A03133
:1051300000F8081B214609F036F9BDE8704004F07C
:1051400064BA29463046BDE870401322FEF77EB9A6
:105150002DE9F047064608A8904690E830048946B5
:105160001F4614220021284609F047F90021CAF8F9
:105170000010B8F1000F03D0B9F1000F03D114E013
:105180003878C00711D02068FCF789F8C0BBB8F1A7
:10519000000F07D120681230286020681430686042
:1051A0002068A8602168CAF800103878800724D5E4
:1051B0006068FCF792F818BBB9F1000F21D0FFF737
:1051C000D3F80168C6F868118188A6F86C11807957
:1051D00086F86E0101F015FDF94FEF60626862B16B
:1051E00096F8680106F2691140081032FEF7FBF8E4
:1051F00010223946606809F0D6F80020BDE8F08733
:1052000006E0606820B1E8606068C6F86401F4E711
:105210001020F3E730B5054608780C4620F00F0063
:10522000401C20F0F001103121700020607095F8D2
:10523000230030B104280FD0052811D0062814D03F
:10524000FFDF20780121B1EB101F04D295F8200078
:1052500000F01F00607030BD21F0F000203002E04F
:1052600021F0F00030302070EBE721F0F00040300A
:10527000F9E7F0B591B0022715460C4606463A46C6
:10528000ADF80870092103AB05F045F8049000283B
:1052900010D004208DF804008DF80170E0340996D8
:1052A00005948DF818500AA968460FF082F900B1EC
:1052B000FFDF012011B0F0BD10B588B00C460A998F
:1052C000ADF80000CBB11868CDF80200D3F80400A7
:1052D000CDF80600ADF80A20102203A809F063F803
:1052E00068460CF08BF903F0AFFF002803D1A17FD3
:1052F00041F01001A17708B010BD0020CDF80200E8
:10530000E6E72DE9F84F0646808A0D4680B28246D0
:10531000FEF799F804463078DFF8A48200274FF0B2
:105320000209A8F120080F2870D2DFE800F06FF220
:105330003708387D8CC8F1F0EFF35FF3F300A07FFE
:1053400000F00300022809D05FF0000080F00101A6
:1053500050460DF033FC050003D101E00120F5E7D4
:10536000FFDF98F85C10C90702D0D8F860000BE0A6
:10537000032105F11D0010F0CAFED5F81D0091496A
:10538000B0FBF1F201FB1200C5F81D007068686700
:10539000B068A8672078252800D0FFDFCAE0A07F8A
:1053A00000F00300022809D05FF0000080F0010146
:1053B00050460DF003FC060003D101E00120F5E7A3
:1053C000FFDF3078810702D52178252904D040F00D
:1053D00001003070BDE8F88F85F80090307F2871AB
:1053E00006F11D002D36C5E90206F3E7A07F00F0A7
:1053F0000300022808D0002080F0010150460DF083
:10540000DDFB040004D102E00120F5E7A7E1FFDFA6
:105410002078C10604D5072028703D346C60D9E798
:1054200040F008002070D5E7E07F000700D5FFDFDF
:10543000307CB28800F0010301B05046BDE8F04F67
:10544000092106F046B804B9FFDF716821B11022C6
:1054500004F1240008F0A7FF28212046FDF75AFE9A
:10546000A07F00F0030002280ED104F124000023E5
:1054700000901A4621465046FFF71EFF112807D01C
:1054800029212046FDF746FE307A84F82000A1E766
:10549000A07F000700D5FFDF14F81E0F40F00800C2
:1054A0002070E782A761E761C109607861F341007C
:1054B000014660F382016170307AE0708AE7A07F74
:1054C00000F00300022809D05FF0000080F0010125
:1054D00050460DF073FB040003D101E00120F5E715
:1054E000FFDF022104F1850010F011FE0420287076
:1054F00004F5B4706860B4F885002882304810382C
:105500007C346C61C5E9028064E703E024E15BE080
:105510002DE015E0A07F00F00300022807D0002056
:1055200080F0010150460DF049FB18B901E001205F
:10553000F6E7FFDF324621465046BDE8F84FE8E582
:1055400004B9FFDF20782128A1D93079012803D1BF
:10555000E07F40F00800E077324621465046FFF7F2
:10556000D8FD2046BDE8F84F2321FDF7D3BD3279A1
:10557000AA8005F108030921504604F0CCFEE8603A
:1055800010B10520287025E7A07F00F00300022855
:1055900008D0002080F0010150460DF00FFB040000
:1055A00003D101E00120F5E7FFDF04F162010223EE
:1055B0001022081F0DF089F907703179417009E751
:1055C0005402002040420F00A07F00F00300022898
:1055D00008D0002080F0010150460DF0EFFA0500E0
:1055E00003D101E00120F5E7FFDF95F8840000F02A
:1055F000030001287AD1A07F00F00307E07F10F0BC
:10560000010602D0022F04D133E095F8A000C007B4
:105610002BD0D5F8601121B395F88320087C62F374
:1056200087000874A17FCA09D5F8601162F34100B0
:105630000874D5F8601166F300000874AEB1D5F8AF
:105640006001102204F12401883508F0ACFE287EA8
:1056500040F001002876287820F0010005F888093C
:1056600000E016B1022F04D02DE095F88800C007A5
:1056700027D0D5F85C1121B395F88320087C62F31C
:1056800087000874A17FCA09D5F85C1162F3410054
:105690000874D5F85C1166F3000008748EB1D5F873
:1056A0005C01102204F12401883508F07CFE287882
:1056B00040F0010005F8180B287820F0010005F8EB
:1056C000A009022F44D0002000EB400005EBC000F1
:1056D00090F88800800709D595F87C00D5F86421FA
:1056E000400805F17D011032FDF77DFE8DF8009038
:1056F00095F884006A4600F003008DF8010095F8E3
:1057000088108DF8021095F8A0008DF8030021464E
:10571000504601F05FFA2078252805D0212807D0CF
:10572000FFDF2078222803D922212046FDF7F2FC52
:10573000A07F00F0030002280CD0002080F00101BF
:1057400050460DF04DFA00283FF44FAEFFDF41E622
:105750000120B9E70120F1E7706847703AE6FFDF02
:1057600038E670B5FE4C002584F85C5025660EF0D6
:10577000ECFE04F11001204603F000FF84F83050E5
:1057800070BD70B50D46FDF75EFE040000D1FFDF71
:105790004FF4B8720021284608F02FFE04F12400CF
:1057A0002861A07F00F00300022809D05FF001010A
:1057B00005F1E0000EF0CAFE002800D0FFDF70BD4A
:1057C0000221F5E70A46014602F1E0000EF0DFBED5
:1057D00070B50546406886B001780A2906D00D29C3
:1057E00033D00E292FD0FFDF06B070BD868830463B
:1057F000FDF729FE040000D1FFDF20782128F3D037
:1058000028281BD1686802210E3001F0D8F9A8B110
:1058100068680821801D01F0D2F978B104F12401F3
:1058200030460CF0B3F803F00FFD00B1FFDF06B017
:105830002046BDE870402921FDF76CBC06B0BDE8EC
:10584000704003F0E2BE012101726868C6883046EC
:10585000FDF7F9FD040000D1FFDFA07F00F0030198
:10586000022902D120F01000A077207821280AD048
:105870006868017A09B1007980B1A07F00F0030067
:10588000022862D0FFDFA07F00F003000228ABD126
:10589000FEF724F80028A7D0FFDFA5E703F0B5FE48
:1058A000A17F08062BD5E07FC00705D094F8200023
:1058B00000F01F00102820D05FF0050084F82300BE
:1058C000207829281DD02428DDD13146042010F06D
:1058D00005FF22212046FDF71DFCA07F00F00300FC
:1058E000022830D05FF0000080F0010130460DF05A
:1058F00077F90028C7D0FFDFC5E70620DEE70420E0
:10590000DCE701F00300022808D0002080F001014C
:1059100030460DF053F9050003D101E00120F5E711
:10592000FFDF25212046FDF7F5FB03208DF8000061
:10593000694605F1E0000EF021FE0228A3D0002800
:10594000A1D0FFDF9FE70120CEE703F05EFE9AE7DC
:105950002DE9F04387B09946164688460746FDF77D
:1059600072FD04004BD02078222848D3232846D04B
:10597000E07F000743D4A07F00F00300022809D095
:105980005FF0000080F0010138460DF017F90500C6
:1059900002D00CE00120F5E7A07F00F00300022810
:1059A00005D00121002238460DF0FFF80546694672
:1059B000284601F036F9009800B9FFDF45B100989C
:1059C000E03505612078222806D0242804D007E09D
:1059D00000990020086103E025212046FDF79AFB8D
:1059E0000098012141704762868001A9C0E90289BF
:1059F0000EF0DFFD022802D0002800D0FFDF07B044
:105A0000BDE8F08370B586B00546FDF71CFD017852
:105A100022291ED9807F00F00300022808D0002030
:105A200080F0010128460DF0C9F804002FD101E0F3
:105A30000120F5E7FFDF2AE0B4F85E0004F162061A
:105A400030440178427829B121462846FFF711FCFD
:105A5000B0B9C9E6ADF804200921284602AB04F02C
:105A60005AFC03900028F4D005208DF80000694608
:105A700004F1E0000EF082FD022801D000B1FFDF4A
:105A800002231022314604F15E000CF054FFB4F8FA
:105A900060000028D0D1A7E610B586B00446FDF717
:105AA000D2FC017822291BD9807F00F00300022854
:105AB00008D0002080F0010120460DF07FF804009E
:105AC00003D101E00120F5E7FFDF06208DF800009B
:105AD000694604F1E0000EF051FD002800D0FFDF20
:105AE00006B010BD2DE9F05F05460C460027007892
:105AF000904601093E4604F1080BBA4602297DD0C2
:105B0000072902D00A2909D146E0686801780A29E4
:105B100005D00D2930D00E292ED0FFDFBBE1142790
:105B20001C26002C6BD08088A080FDF78CFC5FEADF
:105B3000000900D1FFDF99F817005A46400809F123
:105B40001801FDF750FC6868C0892082696851F827
:105B5000060FC4F812004868C4F81600A07E01E0E1
:105B60003402002020F0060040F00100A07699F8F1
:105B70001E0040F020014DE01A270A26002CD1D04B
:105B8000C088A080FDF75FFC050000D1FFDF59460B
:105B90002846FFF73FFB7EE10CB1A88BA080287A56
:105BA0000B287DD006DC01287BD0022808D00328F2
:105BB00004D135E00D2875D00E2874D0FFDF6AE1DE
:105BC0001E270926002CADD0A088FDF73CFC5FEA1B
:105BD000000900D1FFDF287B00F003000128207AB4
:105BE0001BD020F001002072297B890861F341005D
:105BF0002072297BC90861F3820001E041E1F2E0F3
:105C00002072297B090961F3C300207299F81E00F4
:105C100040F0400189F81E103DE140F00100E2E74C
:105C200013270D26002CAAD0A088FDF70CFC814676
:105C3000807F00F00300022808D0002080F00101DE
:105C4000A0880CF0BBFF050003D101E00120F5E7BF
:105C5000FFDF99F81E0000F00302022A50D0686F9F
:105C6000817801F003010129217A4BD021F0010153
:105C7000217283789B0863F3410121728378DB08EA
:105C800063F38201217283781B0963F3C3012172DC
:105C9000037863F306112172437863F3C71103E0BD
:105CA00061E0A9E090E0A1E0217284F809A0C17848
:105CB000A172022A29D00279E17A62F30001E1722D
:105CC0000279520862F34101E1720279920862F3AB
:105CD0008201E1720279D20862F3C301E172427972
:105CE000217B62F3000121734279520862F3410182
:105CF00021734279920862F382012173407928E08E
:105D0000A86FADE741F00101B2E74279E17A62F3B1
:105D10000001E1724279520862F34101E172427975
:105D2000920862F38201E1724279D20862F3C30100
:105D3000E1720279217B62F300012173027952083A
:105D400062F3410121730279920862F382012173A7
:105D50000079C00860F3C301217399F8000023287B
:105D600031D9262140E018271026E4B3A088FDF79A
:105D70006AFB8346807F00F00300022809D00020E0
:105D800080F00101A0880CF019FF5FEA000903D13F
:105D900001E00120F4E7FFDFE868A06099F8000067
:105DA00040F0040189F8001099F80100800708D537
:105DB000012020739BF8000023286CD92721584626
:105DC00051E084F80CA066E015270F265CB1A0888E
:105DD000FDF739FB814606225946E86808F06CFB5E
:105DE0000120A073A0E041E048463CE016270926C8
:105DF000E4B3287B20724EE0287B19270E26ACB333
:105E0000C4F808A0A4F80CA0012807D0022805D0E7
:105E1000032805D0042803D0FFDF0DE0207207E03F
:105E2000697B042801F00F0141F0800121721ED02E
:105E3000607A20F003006072A088FDF704FB05463D
:105E40000078212827D0232800D0FFDFA87F00F08A
:105E50000300022813D0002080F00101A0880CF07C
:105E6000BFFE22212846FDF755F914E004E0607AD0
:105E700020F00300401CDEE7A8F8006010E00120DD
:105E8000EAE70CB16888A080287A68B301280AD0B4
:105E900002284FD0FFDFA8F800600CB12780668091
:105EA0000020BDE8F09F15270F26002CE4D0A08825
:105EB000FDF7C9FA807F00F00300022808D0002017
:105EC00080F00101A0880CF079FE050003D101E00B
:105ED0000120F5E7FFDFD5F81D000622594608F03E
:105EE000EBFA84F80EA0D6E717270926002CC3D0BA
:105EF000A088FDF7A8FA8146807F00F00300022801
:105F000008D0002080F00101A0880CF057FE0500A9
:105F100003D101E00120F5E7FFDF6878800701D5B4
:105F2000022000E00120207299F800002328B2D955
:105F3000272159E719270E26002C9DD0A088FDF7B0
:105F400082FA5FEA000900D1FFDFC4F808A0A4F8D4
:105F50000CA084F808A0A07A40F00300A07299F881
:105F60001E10C90961F38200A07299F81F2099F8E8
:105F70001E1012EAD11F05D099F8201001F01F0160
:105F800010292BD020F00800A07299F81F10607A19
:105F900061F3C3006072697A01F003010129A2D1A3
:105FA00040F00400607299F81E0000F0030002281F
:105FB000E87A16D0217B60F300012173AA7A607B16
:105FC00062F300006073EA7A520862F341012173C0
:105FD000A97A490861F3410060735CE740F008006A
:105FE000D2E7617B60F300016173AA7A207B62F3E0
:105FF00000002073EA7A520862F341016173A97AC2
:10600000490861F34100207345E710B5F74C30B102
:106010000146102204F1200008F0C5F9012084F89F
:10602000300010BD10B5044600F0EBFDEF492046EE
:106030001022BDE81040203108F0B5B970B5EB4D25
:1060400006004FF0000413D0FBF703F908B1102449
:106050000CE00621304608F016FA411C05D02866EF
:106060005FF0010085F85C0000E00724204670BD69
:106070000020F7E7007810F00F0204D0012A05D0C5
:10608000022A0CD110E0000909D10AE00009012818
:1060900007D0022805D0032803D0042801D0072008
:1060A00070470870002070470620704705282AD2E4
:1060B000DFE800F003070F171F00087820F0FF004B
:1060C0001EE0087820F00F00401C20F0F000103097
:1060D00016E0087820F00F00401C20F0F00020307F
:1060E0000EE0087820F00F00401C20F0F000303067
:1060F00006E0087820F00F00401C20F0F00040304F
:10610000087000207047072070472DE9F041804655
:1061100088B00D4600270846FBF7E8F8A8B94046C6
:10612000FDF791F9040003D02078222815D104E06E
:1061300043F2020008B0BDE8F08145B9A07F4106F6
:1061400003D500F00300022801D01020F2E7A07F61
:10615000C10601D4010702D50DB10820EAE7E17FAD
:10616000090701D50D20E5E700F0030002280DD155
:1061700065B12846FEF75EFF0700DBD1FBF732FB77
:1061800020B9E878800701D50620D3E7A07F00F08A
:106190000300022808D0002080F0010140460CF0E6
:1061A0000DFD060002D00FE00120F5E7A07F00F012
:1061B000030002280ED0002080F00101002240469A
:1061C0000CF0F3FC060007D0A07F00F003000228CB
:1061D00004D009E00120EFE70420ABE725B12A460F
:1061E00031462046FEF74AFF6946304600F019FD69
:1061F000009800B9FFDF0099022006F1E002487024
:10620000C1F824804A6100220A81A27F02F00302C1
:10621000022A1CD001200871287800F00102087EB3
:1062200062F3010008762A78520862F38200087649
:106230002A78920862F3C30008762A78D20862F3BB
:106240000410087624212046FCF764FF33E035B3C0
:106250000871301D88613078400908777078C0F384
:1062600040004877287800F00102887F62F301003F
:106270008877A27FD20962F382008877E27F62F397
:10628000C3008877727862F304108877A878C8779B
:1062900001F1210228462031FEF711FF03E003201F
:1062A00008710520087625212046FCF733FFA07FE2
:1062B00020F04000A07701A900980EF07AF902289A
:1062C00001D000B1FFDF384634E72DE9FF4F934698
:1062D000474A0D4699B09A4607CA0AAB002783E899
:1062E00007001998FDF7AFF8060006D03078262889
:1062F00006D008201DB0BDE8F08F43F20200F9E798
:10630000B07F00F00309B9F1020F11D04DB9584622
:10631000FEF790FE0028EDD1B07F00F003000228C8
:1063200006D0BBF1000F11D0FBF75CFA20B10DE0F5
:10633000BBF1000F4FD109E006200CF0E7FB28B1BC
:106340009BF80300800701D50620D3E7B07F00F05B
:106350000300022808D0002080F0010119980CF0F9
:106360002DFC040003D101E00120F5E7FFDF852DBE
:1063700027D007DCEDB1812D1DD0822D1DD0832DBE
:1063800008D11CE0862D1ED0882D1ED0892D1ED050
:106390008A2D1ED00F2020710F281CD003F032F957
:1063A000D8B101208DF83C00201D10902079B0B1AB
:1063B00056E10020EFE70120EDE70220EBE70320A4
:1063C000E9E70520E7E70620E5E70820E3E70920FD
:1063D000E1E70A20DFE707208CE711208AE7B9F11F
:1063E000020F07D0A56F07D1A06F06E0340200208E
:1063F00050550200656FF6E7606F80462DD04FF074
:10640000010001904FF0020000905A4621463046AC
:10641000FEF734FE9BF8000000F00101A87861F35C
:106420000100A870B17FC90961F38200A870F17FF3
:1064300061F3C300A870617861F30410A87020783C
:10644000400928706078C0F3400068709BF8020033
:10645000E87000206871287103E00220019001209B
:106460000090A87898F80210C0F3C000C1F3C001F2
:10647000084003902CD05046FAF7EBFEC0BBDAF888
:106480000C00FAF7E6FE98BBDAF81C00FAF7E1FE1A
:1064900070BBDAF80C00A060DAF81C00E0606078ED
:1064A00098F8012042EA500161F34100607098F8C9
:1064B0000210C0B200EA111161F300006070002008
:1064C0002077009906F11700022907D0012106E084
:1064D000607898F8012002EA5001E5E7002104EB1A
:1064E000810148610199701C022902D0012101E05B
:1064F00028E0002104EB81014861A87800F0030046
:10650000012857D198F8020000F00300012851D16A
:10651000B9F1020F04D02A1D691D5846FEF7CFFDC0
:10652000287998F8041008408DF83400697998F8B3
:10653000052011408DF8381008433BD05046FAF73B
:1065400088FE08B11020D5E60AF110018B46B9F19A
:10655000020F17D00846002104F18C03CDE9000397
:1065600004F5AE7202920DAB2046039AFEF7F0FDE1
:106570000028E8D1B9F1020F08D0504608D14FF0F9
:10658000010107E050464FF00101E5E75846F5E705
:106590004FF0000104F1A403CDE9000304F5B0724B
:1065A000029281F001010EAB2046039AFEF7D0FD66
:1065B0000028C8D16078800733D4A87898F80210F2
:1065C000C0F38000C1F3800108432AD0297898F8ED
:1065D00000000AAAB9F1020F06D032F811204300D8
:1065E000DA4002F003070AE032F810204B00DA40EC
:1065F00012F0030705D0012F0AD0022F0AD0032F73
:1066000006D0039A6AB1012906D0042904D008E013
:106610000227F6E70127F4E7012801D0042800D17A
:106620000427B07F40F08000B077F17F039860F3DB
:106630000001F1776078800705D50320A0710398E9
:1066400070B9002029E00220022F18D0012F18D0A5
:10665000042F2AD00020A071B07F20F08000B077F6
:1066600025213046FCF756FD0FA904F1E0000DF09E
:1066700085FF10B1022800D0FFDF00203AE6A071AC
:10668000DFE7A0710D22002104F1200007F0B5FE24
:10669000207840F00200207001208DF85C0017AADD
:1066A0003146199800F096FADAE70120A071D7E791
:1066B0002DE9F04387B09046894604460025FCF753
:1066C000C2FE060006D03078272806D0082007B082
:1066D000BDE8F08343F20200F9E7B07F00F0030069
:1066E000022809D05FF0000080F0010120460CF084
:1066F00065FA040003D101E00120F5E7FFDFA77987
:106700005FEA090005D0012821D0B9F1020F26D196
:1067100010E0B8F1000F22D1012F05D0022F05D0D3
:10672000032F05D0FFDF2EE00C252CE001252AE009
:10673000022528E04046FAF78CFDB0B9032F0ED1B0
:106740001022414604F11D0007F02DFE1BE0012F31
:1067500002D0022F03D104E0B8F1000F13D00720BC
:10676000B5E74046FAF775FD08B11020AFE71022F3
:10677000002104F11D0007F040FE0621404607F00D
:1067800082FEC4F81D002078252140F00200207010
:106790003046FCF7BFFC2078C10713D020F0010081
:1067A000207002208DF8000004F11D0002908DF889
:1067B00004506946C3300DF0E1FE022803D010B149
:1067C000FFDF00E02577002081E730B587B00D4678
:1067D0000446FCF738FE98B1807F00F003000228E1
:1067E00011D0002080F0010120460CF0E7F90400F0
:1067F0000ED02846FAF72DFD38B1102007B030BD75
:1068000043F20200FAE70120ECE72078400701D4C8
:106810000820F3E7294604F13D002022054607F051
:10682000C2FD207840F01000207001070FD520F045
:106830000800207007208DF80000694604F1E00090
:1068400001950DF09BFE022801D000B1FFDF002072
:10685000D4E770B50D460646FCF7F5FD18B1017892
:10686000272921D102E043F2020070BD807F00F0B1
:106870000300022808D0002080F0010130460CF00F
:106880009DF9040003D101E00120F5E7FFDFA079C5
:10689000022809D16078C00706D02A462146304632
:1068A000FEF7E7FC10B10FE0082070BDB4F86000FF
:1068B0000E280BD204F1620102231022081F0CF0F3
:1068C00004F8012101704570002070BD112070BDD9
:1068D00070B5064614460D460846FAF7BAFC18B9D4
:1068E0002046FAF7DCFC08B1102070BDA6F57F4009
:1068F000FF380ED03046FCF7A6FD38B1417822466D
:106900004B08811C1846FCF76EFD07E043F20200BD
:1069100070BD2046FDF790FD0028F9D11021E01D43
:106920000FF0F5FBE21D294604F1170000F089F98C
:10693000002070BD2DE9F04104468AB01546884616
:1069400000270846FAF7D2FC18B92846FAF7CEFC19
:1069500018B110200AB0BDE8F0812046FCF773FDA5
:10696000060003D0307827281BD102E043F2020052
:10697000F0E7B07F00F00300022809D05FF00000CC
:1069800080F0010120460CF019F9040003D101E068
:106990000120F5E7FFDF2078400702D56078800707
:1069A00001D40820D6E7B07F00F00300022803D00E
:1069B000A06F03D1A16F02E0606FFAE7616F4078CA
:1069C00000B19DB1487810B1B8F1000F0ED0ADB153
:1069D000EA1D06A8E16800F034F9102206A905F1C5
:1069E000170007F0B3FC18B1042707E00720B1E750
:1069F0001022E91D04F12D0007F0D5FCB8F1000FBD
:106A000006D0102208F1070104F11D0007F0CBFCAD
:106A10002078252140F0020020703046FCF77AFBF8
:106A20002078C10715D020F00100207002208DF8D9
:106A3000000004F11D000290103003908DF80470E6
:106A40006946B3300DF09AFD022803D010B1FFDF84
:106A500000E0277700207DE7F8B515460E4607468B
:106A6000FCF7F1FC040004D02078222804D0082090
:106A7000F8BD43F20200F8BDA07F00F00300022839
:106A800002D043F20500F8BD3046FAF7E2FB18B930
:106A90002846FAF7DEFB08B11020F8BD00953288D1
:106AA000B31C21463846FEF707FC112815D00028F4
:106AB000F3D1297C4A08A17F62F3C711A177297C11
:106AC000E27F61F30002E277297C890884F82010D4
:106AD000A17F21F04001A177F8BDA17F0907FBD478
:106AE000D6F80200C4F83600D6F80600C4F83A001A
:106AF0003088A0861022294604F1240007F053FCB8
:106B0000287C4108E07F61F34100E077297C61F354
:106B10008200E077287C800884F82100A07F40F084
:106B20000800A0770020D3E770B50D4606460BB1EC
:106B3000072070BDFCF787FC040007D020782228CE
:106B400002D3A07F800604D4082070BD43F2020067
:106B500070BDADB1294630460AF018FF02F074FB53
:106B6000297C4A08A17F62F3C711A177297CE27FC3
:106B700061F30002E277297C890884F8201004E0A0
:106B800030460AF026FF02F05FFBA17F21F02001D2
:106B9000A17770BD70B50D46FCF755FC040005D01B
:106BA0002846FAF77CFB20B1102070BD43F20200AA
:106BB00070BD29462046FEF72DFB002070BD04E085
:106BC00010F8012B0AB100207047491E89B2F7D294
:106BD0000120704770B51546064602F013FD04000B
:106BE00000D1FFDF207820F00F00801C20F0F000A3
:106BF0002030207066802868A060BDE8704002F0F8
:106C000004BD10B5134C94F83000002808D104F1ED
:106C10002001A1F110000DF0F3FC012084F83000F8
:106C200010BD10B190F8B9202AB10A4890F835008B
:106C300018B1002003E0B83001E0064834300860A5
:106C4000704708B50023009313460A460CF0B5F9C7
:106C500008BD00003402002018B18178012938D124
:106C600001E010207047018842F60112881A914213
:106C700031D018DC42F60102A1EB020091422AD089
:106C80000CDC41B3B1F5C05F25D06FF4C0500818DB
:106C900021D0A0F57060FF381BD11CE001281AD06C
:106CA00002280AD117E0B0F5807F14D008DC012853
:106CB00011D002280FD003280DD0FF2809D10AE0F7
:106CC000B0F5817F07D0A0F58070033803D001288C
:106CD00001D0002070470F2070470A281FD008DC21
:106CE0000A2818D2DFE800F0191B1F1F171F231DE9
:106CF0001F21102815D008DC0B2812D00C2810D02A
:106D00000D2816D00F2806D10DE011280BD08428AD
:106D10000BD087280FD00320704700207047052034
:106D20007047072070470F207047042070470620E7
:106D300070470C20704743F20200704738B50C468C
:106D4000050041D06946FFF795F9002819D19DF853
:106D50000010607861F3020060706946681CFFF7FC
:106D600089F900280DD19DF80010607861F3C50005
:106D70006070A978C1F34101012903D0022905D02F
:106D8000072038BD217821F0200102E0217841F070
:106D900020012170410704D0A978C90861F3861049
:106DA0006070607810F0380F07D0A978090961F396
:106DB000C710607010F0380F02D16078400603D51C
:106DC000207840F040002070002038BD70B50446A7
:106DD0000020088015466068FFF7B0FF002816D134
:106DE0002089A189884211D860688078C0070AD0BC
:106DF000B1F5007F0AD840F20120B1FBF0F200FBB0
:106E00001210288007E0B1F5FF7F01D90C2070BD7A
:106E100001F201212980002070BD10B5047813789B
:106E200064F3000313700478640864F3410313707F
:106E30000478A40864F3820313700478E40864F30C
:106E4000C30313700478240964F3041313700478E3
:106E5000640964F3451313700078800960F38613A6
:106E6000137031B10878C10701D1800701D5012025
:106E700000E0002060F3C713137010BD4278530781
:106E800002D002F0070306E012F0380F02D0C2F37E
:106E9000C20300E001234A7863F302024A7040789B
:106EA00010F0380F02D0C0F3C20005E0430702D053
:106EB00000F0070000E0012060F3C5024A7070474F
:106EC0002DE9F04F95B00D00824613D0122200211B
:106ED000284607F092FA4FF6FF7B05AA0121584693
:106EE00007F053F80024264637464FF420586FF435
:106EF000205972E0102015B0BDE8F08F9DF81E00FB
:106F000001280AD1BDF81C1041450BD011EB090036
:106F10000AD001280CD002280CD0042C0ED0052C4D
:106F20000FD10DE0012400E00224BDF81A6008E052
:106F3000032406E00424BDF81A7002E0052400E0F2
:106F40000624BDF81A10514547D12C74BEB34FF03A
:106F5000000810AA4FF0070ACDE90282CDE900A887
:106F60000DF13C091023CDF81090424631465846A9
:106F700007F0DBF808BBBDF83C002A46C0B210A9F8
:106F80000DF0B4FBC8B9AE81CFB1CDE900A80DF1C9
:106F9000080C0AAE40468CE8410213230022394611
:106FA000584607F0C2F840B9BDF83C00F11CC01EBD
:106FB000C0B22A1D0DF09AFB10B103209BE70AE036
:106FC000BDF82900E881062C05D19DF81E00A872A5
:106FD000BDF81C00288100208DE705A806F0E1FF20
:106FE00000288BD0FFF779FE85E72DE9F0471C4696
:106FF000DDE90978DDF8209015460E00824600D1C3
:10700000FFDF0CB1208818B1D5B11120BDE8F087A1
:10701000022D01D0012100E0002106F1140005F04D
:107020007DFEA8F8000002463B462946504603F084
:1070300072F9C9F8000008B9A41C3C600020E5E71B
:107040001320E3E7F0B41446DDE904528DB10023C8
:1070500014B1022C09D101E0012306E00D7CEE07FA
:1070600003D025F0010501230D742146F0BC04F086
:1070700030BA1A80F0BC70472DE9FE4F91461A884D
:107080001C468A468046FAB102AB494603F043F9F2
:10709000050019D04046A61C27880BF0D4FE3246C6
:1070A000072629463B4600960BF0E1FA2088234646
:1070B000CDE900504A4651464046FFF7C3FF002045
:1070C00020800120BDE8FE8F0020FBE72DE9F0477E
:1070D00086B082460EA8904690E8B000894604AA81
:1070E00005A903A88DE807001E462A4621465046FA
:1070F000FFF77BFF039901B101213970002818D1F6
:10710000FA4904F1140204AB0860039805998DE86C
:10711000070042464946504606F0B3F9A8B109288F
:1071200011D2DFE800F005080510100A0C0C0E0063
:10713000002006B06AE71120FBE70720F9E70820E6
:10714000F7E70D20F5E70320F3E7BDF810100398EB
:10715000CDE9000133462A4621465046FFF772FF2B
:10716000E6E72DE9F04389B01646DDE910870D46C4
:1071700081461C461422002103A807F03EF9012095
:1071800002218DF810108DF80C008DF81170ADF8FB
:10719000146064B1A278D20709D08DF81600E08897
:1071A000ADF81A00A088ADF81800A068079008A8EC
:1071B0000095CDE90110424603A948466B68FFF7E8
:1071C00085FF09B0BDE8F083F0B58BB0002406461A
:1071D000069407940727089405A80994019400973A
:1071E0000294CDE903400D4610232246304606F0B6
:1071F0009CFF78B90AA806A9019400970294CDE9EA
:107200000310BDF8143000222946304606F02BFD4D
:10721000002801D0FFF761FD0BB0F0BD06F0BCBB4C
:107220002DE9FC410C468046002602F0EBF90546AC
:1072300020780D287ED2DFE800F0BC0713B325BD0F
:1072400049496383AF959B00A848006820B1417805
:1072500041F010014170ADE0404602F003FAA9E0B0
:10726000042140460BF0AAFC070000D1FFDF07F124
:107270001401404605F0E7FCA5BB13214046FDF78D
:10728000C1FB97E0042140460BF098FC070000D1B9
:10729000FFDFE088ADF800000020B8819DF8000015
:1072A000010704D5C00602D5A088B88105E09DF885
:1072B000010040067ED5A088F88105B9FFDF22468F
:1072C0002946404601F0C0FC022673E0E188ADF893
:1072D00000109DF8011009060FD5072803D00628D5
:1072E0000AD00AE024E0042140460BF067FC0600C7
:1072F00000D1FFDFA088F0810226CDB9FFDF17E0C3
:10730000042140460BF05AFC070000D1FFDF07F1D3
:10731000140006F078FB90F0010F02D1E07900062E
:1073200048D5387C022640F00200387405B9FFDFEA
:10733000224600E03DE02946404601F085FC39E068
:10734000042140460BF03AFC017C002D01F00206BE
:10735000C1F340016171017C21F002010174E7D1A8
:10736000FFDFE5E702260121404602F0ADF921E00A
:10737000042140460BF022FC0546606800902089FD
:10738000ADF8040001226946404602F0BEF9287CAF
:1073900020F0020028740DE0002DC9D1FFDFC7E7FF
:1073A000022600214046FBF78DF8002DC0D1FFDFFB
:1073B000BEE7FFDF3046BDE8FC813EB50C0009D0DA
:1073C00001466B4601AA002006F034FF20B1FFF70A
:1073D00084FC3EBD10203EBD00202080A0709DF8A2
:1073E000050002A900F00700FEF760FE50B99DF805
:1073F000080020709DF8050002A9C0F3C200FEF746
:1074000055FE08B103203EBD9DF8080060709DF850
:107410000500C109A07861F30410A0709DF8051063
:10742000890961F3C300A0709DF80410890601D595
:10743000022100E0012161F342009DF8001061F398
:107440000000A07000203EBD70B5144606460D46F3
:1074500051EA040005D075B10846F9F73EFF78B946
:1074600001E0072070BD2946304606F04AFF10B102
:10747000BDE8704031E454B12046F9F72EFF08B161
:10748000102070BD21463046BDE8704095E70020D1
:1074900070BD2DE9FC5F0C4690460546002701783B
:1074A0000822007A3E46B2EB111F7DD104F10A0199
:1074B00000910A31821E4FF0020A04F1080B01917B
:1074C000092A72D2DFE802F0EDE005F528287BAA50
:1074D000CE00688804210BF071FB060000D1FFDFAD
:1074E000B08928B152270726C3E000009802002087
:1074F00051271026002C7DD06888A0800120A07123
:10750000A88900220099FFF79FFF002873D1A8895E
:107510002081288AE081D1E0B5F81290072824D193
:10752000E87B000621D5512709F1140086B2002C12
:10753000E1D0A88900220099FFF786FF00285AD1E0
:107540006888A08084F806A0A88920810120A07303
:10755000288A2082A4F81290A88A009068884B4656
:10756000A969019A01F04CFBA8E0502709F112002B
:1075700086B2002C3ED0A88900225946FFF764FF4E
:10758000002838D16888A080A889E080287A072858
:1075900013D002202073288AE081E87BC009607341
:1075A000A4F81090A88A01E085E082E00090688845
:1075B0004B4604F11202A969D4E70120EAE7B5F8C5
:1075C0001290512709F1140086B2002C66D0688809
:1075D00004210BF0F3FA83466888A080A889002272
:1075E0000099FFF731FF00286ED184F806A0A88922
:1075F000208101E052E067E00420A073288A208205
:10760000A4F81290A88A009068884B46A969019A4C
:1076100001F0F6FAA989ABF80E104FE06888FBF785
:1076200012FF0746688804210BF0C8FA064607B91E
:10763000FFDF06B9FFDF687BC00702D051271426A1
:1076400001E0502712264CB36888A080502F06D046
:1076500084F806A0287B594601F0E2FA2EE0287B48
:10766000A11DF9E7FE49A8894989814205D154271E
:1076700006269CB16888A08020E053270BE068882C
:10768000A080A889E08019E0688804210BF096FAB0
:1076900000B9FFDF55270826002CF0D1A8F80060BC
:1076A00011E056270726002CF8D06888A08000201B
:1076B00013E0FFDF02E0012808D0FFDFA8F8006038
:1076C0000CB1278066800020BDE8FC9F5727072665
:1076D000002CE3D06888A080687AA071EEE7401D96
:1076E00020F0030009B14143091D01EB4000704740
:1076F00013B5DB4A00201071009848B10024684699
:107700000BF079F8002C02D1D64A009911601CBD0B
:1077100001240020F4E770B50D461446064686B0F5
:107720005C220021284606F068FE04B9FFDFA0783D
:107730006874A2782188284601F09DFA0020A8816B
:10774000E881228805F11401304605F060FA6A46A6
:107750000121304606F019FC1AE000BF9DF8030035
:10776000000715D5BDF806103046FFF72DFD9DF832
:107770000300BDF8061040F010008DF80300BDF8BE
:107780000300ADF81400FF233046059A06F081FD92
:10779000684606F006FC0028E0D006B070BD10B5C3
:1077A0000C4601F1140005F06AFA0146627C20469D
:1077B000BDE8104001F094BA30B50446A84891B035
:1077C0004FF6FF75C18905AA284606F0DEFB30E0BA
:1077D0009DF81E00A0422AD001282AD1BDF81C0025
:1077E000B0F5205F03D042F60101884221D100208C
:1077F00002AB0AAA0CA9019083E8070007200090B9
:10780000BDF81A1010230022284606F08EFC38B965
:10781000BDF828000BAAC0B20CA90CF067FF10B18C
:10782000032011B030BD9DF82E00A04201D10020F0
:10783000F7E705A806F0B5FB0028C9D00520F0E75A
:1078400070B5054604210BF0B9F9040000D1FFDF43
:1078500004F114010C46284605F0F5F921462846A6
:10786000BDE8704005F0F6B970B58AB00C46064622
:10787000FBF7E9FD050014D02878222827D30CB1A6
:10788000A08890B101208DF80C0003208DF8100025
:1078900000208DF8110054B1A088ADF818002068C0
:1078A00007E043F202000AB070BD0920FBE7ADF823
:1078B00018000590042130460BF080F9040000D137
:1078C000FFDF04F1140005F0F0F9000701D40820EF
:1078D000E9E701F097FE60B108A802210094CDE924
:1078E000011095F8232003A930466368FFF7EEFBEB
:1078F000D9E71120D7E72DE9F04FB2F802A083466F
:1079000089B0154689465046FBF79DFD0746042180
:1079100050460BF053F90026044605964FF0020836
:107920000696ADF81C6007B9FFDF04B9FFDF4146DA
:10793000504603F035FF50B907AA06A905A88DE8FF
:1079400007004246214650466368FFF74EFB444815
:1079500007AB0660DDE9051204F11400CDF80090D4
:10796000CDE90320CDE9013197F82320594650464F
:107970006B6805F0E3F906000AD0022E04D0032E4E
:1079800014D0042E00D0FFDF09B03046BDE8F08FE0
:10799000BDF81C000028F7D00599CDE9001042463B
:1079A000214650466368FFF74DFBEDE7687840F0ED
:1079B00008006870E8E72DE9F04F99B004464FF0F1
:1079C00000082748ADF81C80ADF82080ADF8248071
:1079D000A0F80880ADF81480ADF81880ADF82C80C0
:1079E000ADF82880007916460D464746012808D094
:1079F000022806D0032804D0042802D0082019B099
:107A0000C4E72046F9F725FC70BB2846F9F721FCAE
:107A100050BB6068F9F76AFC30BB606848B16089A8
:107A20002189884202D8B1F5007F01D90C20E6E710
:107A300080460EAA06A92846FFF7C8F90028DED11D
:107A400068688078C0F34100022808D19DF81900C9
:107A500010F0380F03D02869F9F73FFC20B904E093
:107A6000980200201400002022E005A92069FFF7F9
:107A700065F90028C3D1206948B1607880079DF876
:107A8000150000F0380001D5F0B300E0E0BB9DF830
:107A9000140080060ED59DF8150010F0380F03D0A5
:107AA0006068F9F71AFC18B96068F9F71FFC08B1AB
:107AB0001020A4E70AA96069FFF740F900289ED1C9
:107AC000606940B19DF8290000F0070101293CD10F
:107AD00010F0380F39D00BA9A069FFF72FF9002853
:107AE0008DD19DF8280080062FD49DF82C008006AB
:107AF0002BD4A06950B19DF82D0000F00701012999
:107B000023D110F0380F00E01FE01ED0E06818B15C
:107B10000078D0B11C2818D20FAA611C2046FFF7AC
:107B20007CF90121384661F30F2082468DF852100E
:107B3000B94642F603000F46ADF850000DF13F0282
:107B400018A928680CF0F1FD08B1072057E79DF847
:107B5000600015A9CDF80090C01CCDE9019100F09E
:107B6000FF0B00230BF20122514614A806F038F94E
:107B7000F0BBBDF854000C90FE482A892969009298
:107B8000CDE901106B89BDF838202868069906F008
:107B900027F901007ED120784FF0020AC10601D4F6
:107BA00080062BD5CDF80C90606950B90AA906A8BB
:107BB000FFF764F99DF8290020F00700401C8DF8BC
:107BC00029009DF8280008A940F0C8008DF8280079
:107BD0008DF8527042F60210ADF8500003AACDF8AD
:107BE00000A0CDE90121002340F2032214A800E007
:107BF0001EE00A9906F0F4F801004BD1DD484D462D
:107C000008385B460089ADF83D000FA8CDE9029029
:107C1000CDF80490CDF810904FF007090022CDF870
:107C20000090BDF854104FF6FF7006F01CF810B12C
:107C3000FFF753F8E3E69DF83C00000624D52946FB
:107C4000012060F30F218DF852704FF424500395FA
:107C5000ADF8500062789DF80C00002362F300003C
:107C60008DF80C006278CDF800A0520862F3410054
:107C70008DF80C0003AACDE9012540F2032214A8D7
:107C800006F0AEF8010005D1606888B32069A8B994
:107C900005A900E084E006A8FFF7F0F86078800707
:107CA00006D49DF8150020F038008DF8150005E089
:107CB0009DF8140040F040008DF814008DF85270CB
:107CC00042F60110ADF85000208940F20121B0FBCE
:107CD000F1F201FB1202606809ABCDF80080CDE93A
:107CE0000103002314A8059906F07AF8010057D182
:107CF0002078C00728D00395A06950B90BA906A821
:107D0000FFF7BCF89DF82D0020F00700401C8DF80F
:107D10002D009DF82C008DF8527040F040008DF839
:107D20002C0042F60310ADF8500007A903AACDF8C5
:107D300000A0CDE90121002340F2032214A80B99F1
:107D400006F04EF801002BD1E06868B32946012007
:107D500060F30F218DF8527042F60410ADF8500018
:107D6000E068002302788DF8582040788DF859009B
:107D7000E06816AA4088ADF85A00E06800798DF8EE
:107D80005C00E068C088ADF85D00CDF80090CDE9FA
:107D900001254FF4027214A806F022F8010003D066
:107DA0000C9800F0C9FF2AE67248032108380171D7
:107DB00056B100893080BDF824007080BDF82000E5
:107DC000B080BDF81C00F080002018E670B50125D9
:107DD0008AB016460B46012802D0022816D104E0CC
:107DE0008DF80E504FF4205003E08DF80E5042F6FF
:107DF0000100ADF80C005BB10024601C60F30F249F
:107E000004AA08A918460CF090FC18B107204AE50E
:107E1000102048E504A99DF820205648CDE900210E
:107E2000801E02900023214603A802F2012205F0E1
:107E3000D7FF10B1FEF751FF35E54E4808380EB1B7
:107E4000C1883180057100202DE5F0B593B007465B
:107E500001268DF83E6041F60100ADF83C0012AA03
:107E60000FA93046FFF7B2FF002849D1414C002549
:107E7000083CEFB31C22002102A806F0BEFA9DF8D0
:107E800008008DF83E6040F020008DF8080042F6B2
:107E90000520ADF83C000E959DF83A00119520F0B4
:107EA0000600801C8DF83A009DF838006A4620F0E4
:107EB000FF008DF838009DF8390009A920F0FF0077
:107EC0008DF839000420ADF82C00ADF830000EA874
:107ED0000A9011A80D900FA80990ADF82E5002A895
:107EE000FFF769FD00280BD1BDF80000608100E0BC
:107EF00008E0BDF80400A081401CE081257100204D
:107F000013B0F0BD6581A581BDF84800F4E72DE907
:107F1000F74F1849A0B00024083917940A79A146F0
:107F2000012A04D0022A02D0082023B02EE5CA88F4
:107F3000824201D00620F8E721988A46824201D188
:107F40000720F2E70120214660F30F21ADF8480039
:107F50004FF6FF780691ADF84A808DF86E0042F634
:107F6000020B8DF872401CA9ADF86CB0ADF87040F2
:107F7000139101E0A0020020ADF8508012A806F095
:107F80003FF800252E462F460DAB072212A940468A
:107F900006F039F878B10A285DD195B38EB3ADF803
:107FA0006450ADF866609DF85E008DF8144019AC21
:107FB000012864D06BE09DF83A001FB3012859D125
:107FC000BDF8381059451FD118A809A90194029489
:107FD000CDE9031007200090BDF8361010230022D1
:107FE000404606F0A2F8B0BBBDF86000042801D0FE
:107FF00006284AD1BDF82410219881423AD10F2099
:1080000093E73AE0012835D1BDF83800B0F5205F9C
:1080100003D042F6010188422CD1BAF80600BDF81F
:108020003610884201D1012700E0002705B19EB13A
:10803000219881421ED118A809AA01940294CDE981
:108040000320072000900D4610230022404606F032
:108050006CF800B902E02DE04E460BE0BDF8600080
:10806000022801D0102810D1C0B217AA09A90CF01B
:108070003DFB50B9BDF8369086E7052055E705A9C8
:1080800017A8221D0CF051FB08B103204DE79DF805
:1080900014000023001DC2B28DF814202298009213
:1080A000CDE901401BA8069905F09AFE10B90222FD
:1080B0008AF80420FEF711FE37E710B50B46401E84
:1080C00088B084B205AA00211846FEF7A6FE00205B
:1080D0000DF1080C06AA05A901908CE807000720FD
:1080E00000900123002221464FF6FF7005F0BBFDF2
:1080F0000446BDF81800012800D0FFDF2046FEF737
:10810000ECFD08B010BDF0B5F74F044687B03879E4
:108110000E46032804D0042802D0082007B0F0BD82
:1081200004AA03A92046FEF751FE0500F6D16068B7
:108130008078C0F3410002280AD19DF80D0010F0AC
:10814000380F05D02069F9F7C8F808B11020E5E725
:10815000208905AA21698DE807006389BDF81020F0
:108160002068039905F03CFE10B1FEF7B6FDD5E797
:1081700016B1BDF814003080042038712846CDE7D0
:10818000F8B50C0006460CD001464FF6FF750023EB
:108190006A46284606F04EF828B100BFFEF79DFD5E
:1081A000F8BD1020F8BD69462046FEF7C7FD00283F
:1081B000F8D1A078314600F001032846009A06F075
:1081C00068F8EBE730B587B0144600220DF1080CD3
:1081D00005AD01928CE82C00072200920A46014668
:1081E00023884FF6FF7005F03EFDBDF81410218086
:1081F000FEF773FD07B030BD70B50D4604210AF0DF
:10820000DDFC040000D1FFDF294604F11400BDE8C5
:10821000704004F043BD70B50D4604210AF0CEFC59
:10822000040000D1FFDF294604F11400BDE87040CE
:1082300004F057BD70B50D4604210AF0BFFC0400E0
:1082400000D1FFDF294604F11400BDE8704004F0BE
:108250006FBD70B5054604210AF0B0FC040000D1E2
:10826000FFDF214628462368BDE870400122FEF763
:1082700003BF70B5064604210AF0A0FC040000D13B
:10828000FFDF04F1140004F0FAFC401D20F00305A8
:1082900011E0011D00880022431821463046FEF7F8
:1082A000EBFE00280BD0607CABB2684382B2A068C2
:1082B000011D0AF040FBA06841880029E9D170BD8A
:1082C00070B5054604210AF079FC040000D1FFDFF7
:1082D000214628466368BDE870400222FEF7CCBE06
:1082E00070B50E46054601F08DF9040000D1FFDFA0
:1082F0000120207266726580207820F00F00001D3A
:1083000020F0F00040302070BDE8704001F07DB9F1
:1083100010B50446012900D0FFDF2046BDE810401B
:108320000121FAF7CFB82DE9F04F97B04FF0000ACE
:108330000C008346ADF814A0D04619D0E06830B1E7
:10834000A068A8B10188ADF81410A0F800A05846A4
:10835000FBF779F8070043F2020961D03878222848
:108360005CD3042158460AF029FC050005D103E03E
:10837000102017B0BDE8F08FFFDF05F1140004F006
:108380007EFC401D20F00306A078012803D00228BF
:1083900001D00720EDE7218807AA584605F0F5FD32
:1083A00030BB07A805F0FDFD10BB07A805F0F9FDDF
:1083B00048B99DF82600012805D1BDF82400A0F594
:1083C0002451023902D04FF45050D2E7E068B0B1E6
:1083D000CDE902A00720009005AACDF804A00492E0
:1083E000A2882188BDF81430584605F03CFC10B135
:1083F000FEF773FCBDE7A168BDF8140008809DF886
:108400001F00C00602D543F20140B2E70B9838B115
:10841000A1780078012905D080071AD40820A8E7A0
:108420004846A6E7C007F9D002208DF83C00A868AE
:108430004FF00009A0B1697C4288714391420FD985
:108440008AB2B3B2011D0AF02CFA8046A0F800A04F
:1084500006E003208DF83C00D5F800804FF00109BC
:108460009DF8200010F0380F00D1FFDF9DF82000AC
:108470001E49C0F3C200084497F8231010F8010CFD
:10848000884201D90F2074E72088ADF8400014A974
:108490000095CDE90191434607220FA95846FEF702
:1084A00015FE002891D19DF8500050B9A078012800
:1084B00007D1687CB3B2704382B2A868011D0AF08C
:1084C00004FA002055E770B5064615460C460846E6
:1084D000FEF7C2FB002805D12A4621463046BDE8FA
:1084E000704073E470BD12E5980200205A550200F6
:1084F00070B51E4614460D0009D044B1616831B113
:1085000038B1FC49C988814203D0072070BD1020D2
:1085100070BD2068FEF7A0FB0028F9D13246214645
:108520002846BDE87040FFF746BA70B515460C0006
:1085300006D038B1EF490989814203D0072070BDC8
:10854000102070BD2068FEF787FB0028F9D129466E
:108550002046BDE87040D6E570B5064686B00D46AB
:1085600014461046F8F79BFED0BB6068F8F7BEFED5
:10857000B0BBA6F57F40FF3803D03046FAF763FF63
:1085800080B128466946FEF79BFC00280CD19DF877
:1085900010100F2008293DD2DFE801F0080606067A
:1085A000060A0A0843F2020006B070BD0320FBE78A
:1085B0009DF80210012908D1BDF80010B1F5C05F87
:1085C000F2D06FF4C052D142EED09DF806100129CE
:1085D0000DD1BDF80410A1F52851062907D200E0FD
:1085E00029E0DFE801F0030304030303DCE79DF85F
:1085F0000A1001290FD1BDF80810B1F5245FD3D0BE
:10860000A1F60211B1F50051CED00129CCD002293A
:1086100001D1C9E7FFDF606878B9002305AA2946C0
:10862000304605F007FE10B1FEF757FBBCE79DF89A
:108630001400800601D41020B6E76188224628463F
:108640006368FFF7BFFDAFE72DE9F043814687B0D0
:10865000884614461046F8F722FE18B1102007B0DD
:10866000BDE8F083002306AA4146484605F0E2FD36
:1086700018B100BFFEF731FBF1E79DF81800C00606
:1086800002D543F20140EAE70025072705A8019536
:1086900000970295CDE9035062884FF6FF7341467B
:1086A000484605F042FD060013D16068F8F7F7FD73
:1086B00060B960680195CDE9025000970495238860
:1086C00062884146484605F030FD0646BDF8140074
:1086D00020803046CEE739B1864B0A889B899A4282
:1086E00002D843F2030070471DE610B586B0814CF6
:1086F0000423ADF81430638943B1A4898C4201D2BC
:10870000914205D943F2030006B010BD0620FBE7F5
:10871000ADF81010002100910191ADF80030022158
:108720008DF8021005A9029104A90391ADF8122059
:108730006946FFF7F8FDE7E72DE9FC4781460D465E
:108740000846F8F786FD88BB4846FAF77CFE5FEAE4
:1087500000080AD098F80000222829D304214846AE
:108760000AF02CFA070005D103E043F20200BDE84D
:10877000FC87FFDF07F1140004F097FA064628781B
:10878000012803D0022804D00720F0E7B0070FD556
:1087900002E016F01C0F0BD0A8792C1DC00709D0E1
:1087A000E08838B1A068F8F754FD18B11020DEE772
:1087B0000820DCE721882A780720B1F5847F35D0AE
:1087C0001EDC40F20315A1F20313A94226D00EDCF1
:1087D000B1F5807FCBD003DCF9B1012926D1C6E702
:1087E000A1F58073013BC2D0012B1FD113E0012BF7
:1087F000BDD0022B1AD0032BB9D0042B16D112E016
:10880000A1F20912082A11D2DFE802F00B040410C9
:1088100010101004ABE7022AA9D007E0012AA6D065
:1088200004E0320700E0F206002AA0DACDB200F040
:10883000E9FE50B198F82300CDE90005FA892346F6
:1088400039464846FEF78DFC91E711208FE72DE968
:10885000F04F8BB01F4615460C4683460026FAF7AC
:10886000F2FD28B10078222805D208200BB081E55E
:1088700043F20200FAE7B80801D00720F6E7032F19
:1088800000D100274FF6FF79CCB1022D73D32046DB
:10889000F8F72CFD30B904EB0508A8F10100F8F752
:1088A00025FD08B11020E1E7AD1E38F8028CAAB210
:1088B0002146484605F012FE40455CD1ADB20D4957
:1088C000B80702D58889401C00E001201FFA80F813
:1088D000F80701D08F8900E04F4605AA4146584667
:1088E00005F053FB4FF0070A4FF00009DCB32046B8
:1088F0000BE0000098020020408810283BD8361D6D
:10890000304486B2AE4236D2A01902884245F3D333
:1089100051E000BF9DF8170002074CD594B304EB5B
:108920000608361DB8F80230B6B2102B23D89A19B3
:10893000AA4220D8B8F8002091421CD1C0061CD50C
:10894000CDE900A90DF1080C0AAAA11948468CE846
:108950000700B8F800100022584605F084F920B14D
:10896000FEF7BBF982E726E005E0B8F80200BDF8A3
:108970002810884201D00B2078E7B8F80200304474
:1089800086B207E0FFE7C00604D55846FEF71CFC98
:10899000002888D19DF81700BDF81A1020F01000AB
:1089A0008DF81700BDF81700ADF80000FF235846FA
:1089B000009A05F06EFC05A805F0F3FA18B9BDF8A9
:1089C0001A10B942A6D9042158460AF0F7F8040053
:1089D00000D1FFDFA2895AB1CDE900A94D4600239D
:1089E00021465846FEF7BDFB0028BBD1A5813DE7D7
:1089F00000203BE72DE9FF4F8BB01E4617000D46C8
:108A00004FF0000412D0B00802D007200FB0B1E43C
:108A1000032E00D100265DB10846F8F75EFC28B9A8
:108A20003888691E0844F8F758FC08B11020EDE7B3
:108A3000C74AB00701D5D18900E00121F0074FF600
:108A4000FF7802D0D089401E00E0404686B206AAD8
:108A50000B9805F09AFA4FF000094FF0070B0DF153
:108A6000140A38E09DF81B00000734D5CDF80490B7
:108A7000CDF800B0CDF80890CDE9039A4346002226
:108A80000B9805F052FB60BB05B3BDF814103A8893
:108A900021442819091D8A4230D3BDF81E2020F830
:108AA000022BBDF8142020F8022BCDE900B9CDE946
:108AB0000290CDF810A0BDF81E10BDF814300022B1
:108AC0000B9805F032FB08B103209FE7BDF81400B6
:108AD0002044001D84B206A805F063FA20B10A28DC
:108AE00006D0FEF7FAF891E7BDF81E10B142B9D9E9
:108AF00034B17DB13888A11C884203D20C2085E7AF
:108B0000052083E722462946404605F0E7FC01465A
:108B100028190180A41C3C80002077E710B504468A
:108B2000F8F7BDFB08B1102010BD8948C08920802E
:108B3000002010BDF0B58BB00D4606461422002172
:108B400003A805F05AFC01208DF80C008DF81000E8
:108B500000208DF81100ADF814503046FAF773FC80
:108B600048B10078222812D3042130460AF026F8B2
:108B7000040005D103E043F202000BB0F0BDFFDFBB
:108B800004F11400074604F090F8800601D4082090
:108B9000F3E7207C022140F00100207409A8009432
:108BA000CDE90110072203A930466368FEF78EFA6B
:108BB00020B1217C21F001012174DEE729463046F5
:108BC000F9F771FC08A9384604F05EF800B1FFDF40
:108BD000BDF82040172C01D2172000E02046A84203
:108BE00001D92C4602E0172C00D21724214630462A
:108BF000FFF711FB21463046F9F779F90020BCE771
:108C0000F8B51C4615460E46069F0AF00AF923469B
:108C1000FF1DBCB231462A46009409F0F4FCF8BDB1
:108C200070B50C4605460E220021204605F0E5FBF6
:108C3000002020802DB1012D01D0FFDF70BD062066
:108C400000E00520A07170BD10B54880087813467B
:108C500020F00F00001D20F0F00080300C4608705E
:108C60001422194604F1080005F09DFB00F0CDFC2C
:108C70003748046010BD2DE9F047DFF8D890491D52
:108C8000064621F0030117460C46D9F8000009F00A
:108C9000D0FD050000D1FFDF4FF000083560A5F8DA
:108CA00000802146D9F8000009F0C3FD050000D17D
:108CB000FFDF7560A5F800807FB104FB07F1091D97
:108CC0000BD0D9F8000009F0B4FD040000D1FFDF9B
:108CD000B460C4F80080BDE8F087C6F80880FAE701
:108CE0002DE9F0411746491D21F00302194D0646B2
:108CF00001681446286809F0C7FD22467168286893
:108D000009F0C2FD3FB104FB07F2121D03D0B168A8
:108D1000286809F0B9FD042009F0F8FE0446042093
:108D200009F0FCFE201A012804D12868BDE8F041B2
:108D300009F074BDBDE8F08110B50C4605F0F4F8FB
:108D400000B1FFDF2046BDE81040FDF7C6BF0000C0
:108D5000980200201400002038B50C468288817BE0
:108D600019B14189914200D90A462280C188121D59
:108D700090B26A4608F034FFBDF80000032800D323
:108D80000320C1B2208801F021F838BD38B50C4667
:108D90008288817B19B10189914200D90A462280DB
:108DA000C188121D90B26A4608F01AFFBDF8000093
:108DB000022800D30220C1B2208801F007F8401C2D
:108DC000C0B238BD2DE9FF5F82468B46FB48144692
:108DD0000BF10302D0E90110CDE9021022F00302E9
:108DE00001A84FF49071019209F005FDF44E002C9A
:108DF00002D1F449019A8A60019901440191B57F39
:108E000005F1010504D1E8B20BF008FC00B1FFDF69
:108E1000019800EB0510C01C20F0030101915CB922
:108E2000707AB27A1044C2B200200870308C80B2DE
:108E300004F0D9FE00B1FFDF0198316A08440190C7
:108E4000214601A800F085FF80460198C01C20F053
:108E500003000190B37AF27A717A04B1002009F02C
:108E6000C0FD019908440190214601A800F0B9FF16
:108E7000D34800273D4690F801900CE0284600F0CA
:108E80004BFF064681788088F9F7C8F871786D1C29
:108E900000FB0177EDB24D45F0D10198C01C20F0E8
:108EA0000300019004B100203946F9F7C2F8019996
:108EB000002708440190C2483D4690F801900CE01C
:108EC000284600F029FF0646C1788088FEF707FC97
:108ED00071786D1C00FB0177EDB24D45F0D1019822
:108EE000C01C20F00300019004B100203946FEF7B9
:108EF000FFFB01994FF0000908440190B0484D462E
:108F000047780EE0284600F007FF0646807B30B128
:108F100006F1080002F068F9727800FB02996D1CF6
:108F2000EDB2BD42EED10198C01C20F003000190CB
:108F300004B10020A3494A78494602F059F9019941
:108F400008440190214601A800F0B6FE0198C01D1A
:108F500020F007000190DAF80010814204D3A0EB62
:108F60000B01B1F5803F04DB4FF00408CAF80000A4
:108F700004E0CAF80000B8F1000F03D0404604B086
:108F8000BDE8F09F74BB90490020019A0DF03AFCB7
:108F9000FBF7EDF98A4C207F0090607F012823D0F9
:108FA000002318B30022864800211030F8F720FA79
:108FB00000B1FFDFE07FFEF748FF00B1FFDF804830
:108FC0004FF4F6720021403005F017FA7C48042176
:108FD000403080F8E91180F8EA11062180F8EB11A1
:108FE000032101710020CAE70123DAE702AADAE7C8
:108FF00070B5734C06464034207804EB4015E07899
:10900000083598B9A01990F8E80100280FD0A07889
:109010000F2800D3FFDF20220021284605F0EDF9BC
:10902000687866F3020068700120E070284670BD21
:109030002DE9F04105460C460027007805219046B1
:109040003E46B1EB101F00D0FFDF287A50B1012857
:109050000ED0FFDFA8F800600CB1278066800020EA
:10906000BDE8F0810127092674B16888A08008E076
:109070000227142644B16888A0802869E060A88A85
:109080002082287B2072E5E7A8F80060E7E730B58A
:109090004B4C01200021207061702072607203220D
:1090A000A272E072617721772173217405212183F7
:1090B0001F216183607445A161610A21A177E07776
:1090C000404D4FF4B06020626868C11C21F003017C
:1090D000814200D0FFDF6868606030BD30B5394C38
:1090E0001568636810339D4202D20420136030BDBE
:1090F000334B5D785A6802EB0512107051700320F3
:10910000D080172090800120D07090700020907344
:109110005878401C5870606810306060002030BD86
:1091200070B5064626480024457807E0204600F042
:10913000F3FD0178B14204D0641CE4B2AC42F5D135
:10914000002070BDF7B5074608780C4610B3FFF74E
:10915000E7FF0546A7F12006202F06D0052E19D2DD
:10916000DFE806F00F3838151A0000F0E0FD0DB109
:10917000697800E00021401AA17880B20844FF28F5
:1091800008D8A07830B1A088022831D202E06088E7
:1091900017282DD20720FEBD207A48B361881729F1
:1091A000F8D3A1881729F5D3A1790029F2D0E17964
:1091B0000029EFD0402811D9ECE7000060550200EB
:1091C000B403002018000020000000206E52463535
:1091D00078000000242F0BD1207A48B161884FF627
:1091E000FB70814202D8A188814201D90420FEBDD2
:1091F00065B9207802AA0121FFF770FF0028F6D197
:109200002078FFF78DFF050000D1FFDF052E18D273
:10921000DFE806F0030B0E081100A0786870A08844
:10922000E8800FE06088A8800CE0A078A87009E0D2
:10923000A078E87006E054F8020FA8606068E86063
:1092400000E0FFDF0020FEBD1A2835D00DDC13281A
:1092500032D2DFE800F01B31203131272723252DC2
:10926000313129313131312F0F00302802D003DC68
:109270001E2821D1072070473A3809281CD2DFE880
:1092800000F0151B0F1B1B1B1B1B0700002070474A
:1092900043F20400704743F2020070470420704715
:1092A0000D2070470F20704708207047112070472D
:1092B00013207047062070470320704710B50078D0
:1092C00000F0010008F07EFCBDE81040BCE710B5DE
:1092D000007800F0010008F07EFCBDE81040B3E724
:1092E0000EB5017801F001018DF80010417801F010
:1092F00001018DF801100178C1F340018DF80210D1
:109300004178C1F340018DF80310017889088DF888
:109310000410417889088DF8051081788DF80610C1
:10932000C1788DF8071000798DF80800684607F0BD
:109330000EFDFFF789FF0EBD2DE9F84FDFF8F8832A
:10934000FE4C00264FF490771FE0012000F08CFDCA
:109350000120FFF74DFE05463946D8F8080009F010
:1093600068FA686000B9FFDF686807F0BEFBB0B15B
:109370002846FAF748FB284600F07CFD28B93A4613
:109380006968D8F8080009F07FFA94F9E90104281F
:10939000DBDA022009F0BAFB07460025A5E03A46D1
:1093A0006968D8F8080009F06FFAF2E7B8F8021017
:1093B0004046491C89B2A8F80210B94201D30021E5
:1093C00041800221B8F8020009F0F8FB002864D0BF
:1093D000B8F80200694608F065FBFFF735FF00B1F9
:1093E000FFDF9DF8000078B1B8F8020009F02BFD0E
:1093F0005FEA000900D1FFDF484608F098FF18B186
:10940000B8F8020002F0BAF9B8F8020009F009FD54
:109410005FEA000900D1FFDF484608F080FFE0BBAB
:109420000321B8F8020009F0C9FB5FEA000B47D13D
:10943000FFDF45E0DBF8100010B10078FF2849D0CD
:10944000022000F011FD0220FFF7D2FD82464846BF
:1094500009F071F8CAF8040000B9FFDFDAF8040077
:1094600009F039F9002100900170B8F80210504657
:10947000AAF8021002F088F8484609F02EF900B95F
:10948000FFDF504600F0F6FC18B99AF8010000071B
:1094900004D50098CBF8100012E024E0DBF81000AF
:1094A00038B10178491C11F0FF01017008D1FFDFCC
:1094B00006E000221146484600F0FCFB00B9FFDF41
:1094C00094F9EA01022805DBB8F8020002F023F85B
:1094D0000028AFD194F9E901042804DB484609F0DB
:1094E00060F900B101266D1CEDB2BD4204D294F9C1
:1094F000EA010228BFF65AAF002E7FF422AFBDE882
:10950000F84F032000F0B0BC10B58B4CE060086849
:109510002061AFF2DB10F9F7C4FC607010BD874822
:1095200000214038017084480170854941607047CE
:1095300070B505464FF080500C46D0F8A410491C79
:1095400005D1D0F8A810C9430904090C0BD050F874
:10955000A01F01F001012970416821608068A0808E
:10956000287830B970BD062120460CF0D0FD0120CE
:109570002870607940F0C000607170BD70B54FF028
:1095800080540D46D4F88010491C0BD1D4F88410B7
:10959000491C07D1D4F88810491C03D1D4F88C1089
:1095A000491C0CD0D4F880100160D4F884104160BC
:1095B000D4F888108160D4F88C10C16002E01021CA
:1095C0000CF0A5FDD4F89000401C0BD1D4F8940009
:1095D000401C07D1D4F89800401C03D1D4F89C005B
:1095E000401C09D054F8900F286060686860A0683B
:1095F000A860E068E86070BD2846BDE870401021B2
:109600000CF085BD4D480079F2E470B54B4CE07824
:1096100030B3207804EB4010407A00F0070020447B
:1096200090F9E801002800DCFFDF2078002504EB3A
:109630004010407A00F00700011991F8E801401E3F
:1096400081F8E8012078401CC0B220700F2800D1BA
:109650002570A078401CA0700CF050FCE57070BD27
:10966000FFDF70BD3EB50546032109F0A7FA0446A9
:10967000284609F0D6FB054604B9FFDF206918B17A
:109680000078FF2800D1FFDF01AA6946284600F0D4
:1096900011FB60B9FFDF0AE0002202A9284600F0B2
:1096A00009FB00B9FFDF9DF8080000B1FFDF9DF85E
:1096B0000000411E8DF80010EED220690199884209
:1096C00001D1002020613EBD70B50546A0F57F4068
:1096D0000C46FF3800D1FFDF012C01D0FFDF70BD49
:1096E000FFF790FF040000D1FFDF207820F00F008B
:1096F000401D20F0F0005030207065800020207266
:1097000001202073BDE870407FE72DE9F041164647
:109710000D460746FFF776FF040000D1FFDF2078F3
:1097200020F00F00401D20F0F000503020706780C6
:1097300001202072286805E018000020F4030020B2
:10974000381400202061A888A0822673BDE8F0416B
:109750005BE77FB5FFF7E4FC040000D1FFDF02A95F
:109760002046FFF7F9FA054603A92046FFF70EFB4E
:109770008DF800508DF80100BDF80800001DADF80F
:109780000200BDF80C00001DADF80400E088ADF843
:109790000600684608F000FA002800D0FFDF7FBD11
:1097A0002DE9F05FF84E8146307810B10820BDE811
:1097B000F09F4846F7F773FD08B11020F7E7F34C28
:1097C000207808B9FFF763FCA17A607A4D46084417
:1097D000C4B200F0ACFAA04207D2201AC1B22A46A5
:1097E0000020FFF77BFC0028E1D17168E748C91C25
:1097F000002721F003017160B3463E463D46BA465C
:109800003C4690F801800AE0204600F085FA417855
:10981000807B0E4410FB0155641CE4B27F1C444560
:10982000F2D10AEB870000EBC600D84E00EB8500B2
:109830005C46F17A012200EB8100DBF80410451848
:1098400029464846FFF7BEFA070012D00020FFF76E
:1098500067FC05000BD005F11300616820F00300E0
:10986000884200D0FFDF7078401E70706560384617
:109870009DE7002229464846FFF7A4FA00B1FFDF22
:10988000D9F8000060604FF6FF7060800120207002
:1098900000208CE72DE9F0410446BB4817460E46F0
:1098A000007810B10820BDE8F0810846F7F7D1FC38
:1098B00008B11020F7E7B54D287808B9FFF7E7FBA6
:1098C000601E1E2807D8012C22D13078FE281FD810
:1098D000A8770020E7E7A4F120001F2805D8E0B210
:1098E0003A463146BDE8F0412CE4A4F140001F287F
:1098F00005D831462046BDE8F04100F0E3BAA4F1B6
:10990000A0001F2804D80020A02C03D0A12C06D032
:109910000720C8E7317801F00101E977C3E7316832
:109920000922F82901D38B0701D01046BBE76B7CD5
:1099300003F00303012B04D16B8BD7339CB28C4211
:10994000F3D82962AFE72DE9F04781460E46084675
:10995000F7F7A5FC48B94846F7F7BFFC28B909F165
:10996000030020F00301494502D01020BDE8F08734
:1099700086484FF0000A4030817869B141788046CE
:1099800000EB41140834378832460021204600F0AD
:109990007FFA050004D027E0A6F800A00520E5E73F
:1099A000B9F1000F24D03088B84201D90C251FE04E
:1099B000607800F00705284600F056FA08EB050726
:1099C000324697F8E8014946401C87F8E8012046EE
:1099D00007F5F47700F05CFA05463878401E3870D9
:1099E000032000F041FA2DB10C2D01D0A6F800A003
:1099F0002846BBE76078644E00F00701012923D0B8
:109A000002290CD0032934D0FFDF98F8011040461A
:109A1000491CC9B288F801100F2935D036E06168B9
:109A200021B1000702D46088FFF71CFE98F8EA0114
:109A30004746012802D17078F9F752FA97F9EA01FE
:109A40000428E2DBFFDFE0E7616821B14FF49072A8
:109A5000B06808F019FF98F8E9014746032802D1D9
:109A60007078F9F73DFA97F9E9010428CDDBFFDFBB
:109A7000CBE7C00602D56088FFF7F4FD98F9EB014B
:109A80000628C2DBFFDFC0E780F801A08178491E0D
:109A90008170617801F0070101EB080090F8E8118E
:109AA000491C80F8E811A3E770B50D460446F7F7A6
:109AB000D0FB18B92846F7F7F2FB08B1102070BDAB
:109AC00029462046BDE870400AF0E0BD70B5054665
:109AD0000AF0FFFDC4B22846F7F7FFFB08B11020DB
:109AE00070BD35B128782C7018B1A04201D0072084
:109AF00070BD2046FDF760FE052805D10AF0EDFD9A
:109B0000012801D0002070BD0F2070BD70B5044643
:109B100015460E460846F7F79CFB18B92846F7F796
:109B2000BEFB08B1102070BD022C03D0102C01D058
:109B3000092070BD2A46314620460AF0D7FD00288C
:109B4000F7D0052070BD70B514460D460646F7F7F0
:109B500080FB38B92846F7F7A2FB18B92046F7F77B
:109B6000BCFB08B1102070BD2246294630460AF0E1
:109B7000DCFD0028F7D0072070BD3EB50446F7F79E
:109B80008EFB28B110203EBD18000020B403002039
:109B9000684607F050F8FFF757FB0028F3D19DF80F
:109BA00006002070BDF808006080BDF80A00A080A3
:109BB0000020E8E770B505460C460846F7F78DFB30
:109BC00020B93CB12068F7F76AFB08B1102070BDDE
:109BD000A08828B121462846BDE87040FDF744BE64
:109BE000092070BD70B505460C460846F7F731FBF5
:109BF00030B9681E1E2814D82046F7F72AFB08B192
:109C0000102070BD032D01D9072070BD05B9FFDFFD
:109C1000FE4800EB850050F8041C2046BDE870406B
:109C20000847A5F120001F2805D821462846BDE891
:109C30007040FAF712BBF02D0AD0BF2DE4D1A07806
:109C4000218800F0010001F055FB68B1002070BDD3
:109C5000A068F7F7FEFA0028D2D1204608F001F8F4
:109C6000BDE87040FFF7F0BA082070BD70B504463B
:109C70000D460846F7F713FB30B9601E1E280FD8B3
:109C80002846F7F7E6FA08B1102070BD012C03D082
:109C9000022C01D0032C01D1062070BD072070BD1D
:109CA000A4F120001F28F9D829462046BDE87040BD
:109CB000FAF73DBB08F002BB7CB50446D448007BF4
:109CC00000F0010511BB04F0BAFB0DB1226800E001
:109CD0000022D0484178C06806F0E2FCCD48103040
:109CE000C0788DF8000010B1012802D004E00120F6
:109CF00000E000208DF80000684607F009F8C3482E
:109D000024380068019001A807F042FD002D02D020
:109D10002068283020607CBD30B5BD4D0446687891
:109D2000A04200D8FFDF686800EB041030BD70B5BA
:109D3000B74800252C46467807E02046FFF7ECFFA1
:109D40004078641C2844C5B2E4B2B442F5D1284638
:109D500070BD2DE9F0410C4607464FF0000800F0B9
:109D6000EDF80646FF2801D94FF013083868C01CEB
:109D700020F003023A6054EA080421D1A448F3B267
:109D8000072124300CF0D0FB09E0072C10D2DFE8CB
:109D900004F0060408080A0406009F4804E09F48EF
:109DA00002E09F4800E09F480CF0DEFB054600E023
:109DB000FFDFA54200D0FFDF641CE4B2072CE4D330
:109DC000386800EB0610386040466CE5021D5143D0
:109DD000452900D245210844C01CB0FBF2F0C0B2B6
:109DE00070472DE9FC5F064689484FF000088B4616
:109DF0004746444690F8019022E02046FFF78CFF4A
:109E0000050000D1FFDF687869463844C7B22846AC
:109E1000FEF7A2FF824601A92846FEF7B7FF0346D8
:109E2000BDF804005246001D81B2BDF80000001DBF
:109E300080B208F041FF6A78641C00FB0288E4B23B
:109E40004C45DAD13068C01C20F003003060BBF113
:109E5000000F00D000204246394608F03BFF316831
:109E600008443060BDE8FC9F69494031087100201A
:109E7000C870704766494031CA782AB10A7801EB48
:109E800042110831814201D0012070470020704703
:109E90002DE9F04106460078154600F00F04002039
:109EA0001080601E0F46052800D3FFDF57482A4662
:109EB000183800EB8400394650F8043C3046BDE8C1
:109EC000F04118472DE9F041514E0C46402806D08C
:109ED000412823D042282BD0432806D123E0A07864
:109EE00061780D18E178814201D90720DBE4207800
:109EF000012801D91320D6E4FF2D08D80AF080FDEF
:109F000007460BF0B3FF381A801EA84201DA122070
:109F1000C9E42068B060207930730DE0BDE8F041FD
:109F2000084600F036B808780228DED8307703E01B
:109F300008780228D9D870770020B4E42DE9F047DA
:109F4000DFF8CC900026344699F8090099F80A20E9
:109F500099F801700244D5B299F80B20104400F032
:109F6000FF0808E02046FFF7D7FE817B407811FB11
:109F70000066641CE4B2BC42F4D199F8091099F867
:109F80000A0029442944414400B1012008443044D6
:109F9000ECE438B50446407800F00300012803D013
:109FA00002280BD0072038BD606858B1F7F79EF93A
:109FB000D0B96068F7F791F920B915E06068F7F754
:109FC00048F988B969462046FCF754F80028EAD1D8
:109FD000607800F00300022808D19DF8000028B145
:109FE0006068F7F77AF908B1102038BD6189F8295F
:109FF0001CD82089884219D8607800F003020448F0
:10A00000012A15D1D73189B2026A0DE084550200C8
:10A01000B4030020180000205B41000011B30000D1
:10A02000B52F00000F4401008A4201D2092038BD3B
:10A0300094E80E0000F1100585E80E000AB9002131
:10A040000183002038BD00002DE9F0410746144689
:10A050008846084601F08AFD064608EB88001C2267
:10A06000796802EBC0000D18688C58B1414638463B
:10A0700001F08BFD014678680078C200082305F1E5
:10A0800020000CE0E88CA8B14146384601F084FD80
:10A090000146786808234078C20005F1240008F0E2
:10A0A0004AFC38B1062121726681D0E90010C4E96A
:10A0B000031009E0287809280BD00520207266815A
:10A0C0006868E060002028702046BDE8F04101F09B
:10A0D0002EBD072020726681F4E72DE9F041164677
:10A0E0000D460746406801EB85011C2202EBC101C9
:10A0F0004418204601F072FD40B10021708865F3DC
:10A100000F2160F31F4106200CF0E8FA09202070AF
:10A11000324629463846BDE8F04195E72DE9F04141
:10A120000E46074600241C21F07816E004EB840359
:10A13000726801EBC303D25C6AB1FFF763FA0500F2
:10A1400000D1FFDF6F802A4621463046FFF7C5FF6A
:10A150000120BDE8F081641CE4B2A042E6D80020F2
:10A16000F7E770B5064600241C21C0780AE000BF5E
:10A1700004EB8403726801EBC303D5182A782AB173
:10A18000641CE4B2A042F3D8402070BD2822002114
:10A19000284604F032F9706880892881204670BD15
:10A1A00070B5034600201C25DC780CE000EB80062F
:10A1B0005A6805EBC6063244167816B1128A8A42EE
:10A1C00004D0401CC0B28442F0D8402070BDF0B52D
:10A1D000044600201C26E5780EE000BF00EB800757
:10A1E000636806EBC7073B441F788F4202D15B7858
:10A1F000934204D0401CC0B28542EFD84020F0BD4D
:10A200000078032801D000207047012070470078B3
:10A21000022801D0002070470120704700780728ED
:10A2200001D000207047012070472DE9F04106461B
:10A2300088461078F1781546884200D3FFDF2C78E5
:10A240001C27641CF078E4B2A04201D8201AC4B2E2
:10A2500004EB8401706807EBC1010844017821B167
:10A260004146884708B12C7073E72878A042E8D1AE
:10A27000402028706DE770B514460B880122A2407B
:10A28000134207D113430B8001230A22011D08F05A
:10A290001CFB047070BD2DE9FF4F81B00878DDE92B
:10A2A0000E7B9A4691460E4640072CD4019808F042
:10A2B000CAFD040000D1FFDF07F1040820461FFAA1
:10A2C00088F107F007FF050000D1FFDF204629468F
:10A2D0006A4608F052F90098A0F80370A0F805A0AB
:10A2E000284608F0F8F9017869F306016BF3C71105
:10A2F000017020461FFA88F107F02FFF00B9FFDF39
:10A30000019806F03CF906EB0900017F491C017732
:10A3100005B0BDE8F08F2DE9F84F0E469A469146FC
:10A320000746032108F04AFC0446008DDFF8B88593
:10A33000002518B198F80000B0421ED1384608F048
:10A3400082FD070000D1FFDF09F10401384689B220
:10A3500007F0C0FE050010D0384629466A4608F0CE
:10A360000CF9009800210A460180817006F0C3F9BB
:10A370000098C01DCAF8000021E098F80000B04223
:10A3800016D104F1260734F8341F012000FA06F92B
:10A3900011EA090F00D0FFDF2088012340EA0900FD
:10A3A00020800A22391D384608F0AAFA067006E015
:10A3B000324604F1340104F12600FFF75CFF0A2164
:10A3C00088F800102846BDE8F88FFEB515460C4603
:10A3D000064602AB0C220621FFF79DFF002827D07E
:10A3E0000299607812220A70801C487008224A8004
:10A3F000A07002982988052381806988C180A98876
:10A400000181E988418100250C20CDE90005062263
:10A4100021463046FFF73FFF2946002266F31F41E1
:10A42000F02310460CF0B0F86078801C60700120BA
:10A43000FEBDFEB514460D460622064602AB114689
:10A44000FFF769FF002812D0029B1320002118702B
:10A45000A8785870022058809C800620CDE9000121
:10A460000246052329463046FFF715FF0120FEBDB1
:10A470002DE9FE430C46804644E002AB0E22072144
:10A480004046FFF748FF002841D060681C226778EB
:10A490008678BF1C06EB860102EBC10145180298C5
:10A4A0001421017047700A214180698A0181E98A7B
:10A4B0004181A9888180A9898181304601F056FBBC
:10A4C000029905230722C8806F7004202870002598
:10A4D0000E20CDE9000521464046FFF7DCFE294667
:10A4E00066F30F2168F31F41F023002206200CF0D1
:10A4F0004BF86078FD49801C607062682046921CB1
:10A50000FFF793FE606880784028B6D10120BDE84F
:10A51000FE83FEB50D46064638E002AB0E2207214B
:10A520003046FFF7F8FE002835D068681C23C17854
:10A5300001EB810203EBC20284180298152202701B
:10A54000627842700A224280A2894281A288828176
:10A55000084601F00BFB014602988180618AC180A8
:10A56000E18A0181A088B8B10020207000210E206E
:10A57000CDE900010523072229463046FFF78BFE6F
:10A580006A68DB492846D21CFFF74FFE6868C0782E
:10A590004028C2D10120FEBD0620E6E72DE9FE439A
:10A5A0000C46814644E0204601F002FBD0B302ABEA
:10A5B000082207214846FFF7AEFE0028A7D06068B2
:10A5C0001C2265780679AD1C06EB860102EBC10101
:10A5D00047180298B7F810800621017045700421D1
:10A5E0004180304601F0C2FA014602980523072255
:10A5F000C180A0F804807D70082038700025CDE966
:10A60000000521464846FFF746FE294666F30F211E
:10A6100069F31F41F023002206200BF0B5FF60789C
:10A62000801C60706268B3492046121DFFF7FDFD73
:10A63000606801794029B6D1012068E72DE9F34F20
:10A6400083B00D4691E0284601F0B2FA00287DD093
:10A6500068681C2290F806A00AEB8A0102EBC1018F
:10A6600044185146284601F097FAA178CB00696852
:10A670004978CA00014604F1240008F078F9074639
:10A680008188E08B4FF00009091A8EB208B1C846E4
:10A6900007E04FF00108504601F053FA08B9B61C24
:10A6A000B6B2208BB04200D80646B34602AB324663
:10A6B00007210398FFF72FFE060007D0B8F1000F1F
:10A6C0000BD0504601F03DFA10B106E000201FE625
:10A6D0000299B8884FF0020908800196E28B396828
:10A6E000ABEB09001FFA80F80A4403984E4600922B
:10A6F00008F0A9FBDDE90021F61D4346009607F0AE
:10A70000B6FFE08B404480B2E083B988884201D133
:10A71000012600E00026CDE900B6238A072229465B
:10A720000398FFF7B8FD504601F00BFA10B9E08925
:10A73000401EE08156B1A078401CA0706868E9789E
:10A74000427811FB02F1CAB2012300E007E08169FF
:10A750000E3008F0BAF880F800A00020E0836A68A4
:10A7600065492846921DFFF760FD68688179402998
:10A770007FF469AF0120CBE570B5064648680D4609
:10A7800014468179402910D104EB84011C2202EB8C
:10A79000C101084401F043FA002806D06868294640
:10A7A00084713046BDE8704048E770BDFEB50C4688
:10A7B0000746002645E0204601F0FAF9D8B3606864
:10A7C0001C22417901EB810102EBC1014518688926
:10A7D00000B9FFDF02AB082207213846FFF79BFDD7
:10A7E000002833D00299607816220A70801C4870C5
:10A7F000042048806068407901F0B8F90146029869
:10A800000523072281806989C1800820CDE90006DF
:10A8100021463846FFF73FFD6078801C6070A889AC
:10A8200069890844B0F5803F00D3FFDFA8896989B2
:10A830000844A8816E81626830492046521DFFF7A6
:10A84000F4FC606841794029B5D10120FEBD30B5E6
:10A85000438C458BC3F3C704002345B1838B641E2F
:10A86000ED1AC38A6D1E1D4495FBF3F3E4B22CB1BF
:10A87000008918B1A04200D8204603444FF6FF706B
:10A88000834200D3034613800C7030BD2DE9FC4198
:10A89000074616460D46486802EB86011C2202EB6D
:10A8A000C10144186A4601A92046FFF7D0FFA089DC
:10A8B000618901448AB2BDF80010914212D0081A91
:10A8C00000D5002060816868407940280AD1204680
:10A8D00001F09BF9002805D0686829464671384682
:10A8E000FFF764FFBDE8FC812C00002001A20000FE
:10A8F0000FA200001DA200001FBC00000BBC000046
:10A900002DE9FE4F0F46814615465088032108F079
:10A9100055F90190B9F8020001F01BF98246014691
:10A92000019801F045F9002824D001981C224168C3
:10A930000AEB8A0002EBC0000C18204601F04EF929
:10A94000002817D1B9F80000E18A88420ED8A18901
:10A9500061B1B8420ED100265146019801F015F9B7
:10A96000218C01EB0008608B30B114E0504601F0FF
:10A97000E8F8A0B3BDE8FE8F504601F0E2F808B158
:10A98000678308E0022FF5D3B9F804006083618A79
:10A99000884224D80226B81B87B2B8F80400A28BDC
:10A9A000801A002814DD874200DA38461FFA80FB3F
:10A9B000688869680291D8F800100A44009208F08B
:10A9C00030FAF61D009A5B460299009607F01BFECE
:10A9D000A08B384480B2A083618B884207D96888F5
:10A9E000019903B05246BDE8F04F01F035B91FD1CF
:10A9F0004FF009002872B9F802006881D8E9001008
:10AA0000C5E90410608BA881284601F090F85146F2
:10AA1000019801F0BAF801460198082340680078CF
:10AA2000C20004F1200007F086FF0020A0836083AD
:10AA3000504601F086F810B9A089401EA0816888B0
:10AA4000019903B00AF0FF02BDE8F04F1EE72DE9BF
:10AA5000F041064615460F461C461846F6F7F9FB28
:10AA600018B92068F6F71BFC10B11020BDE8F08182
:10AA70007168688C0978B0EBC10F01D31320F5E73A
:10AA80003946304601F081F80146706808230078A5
:10AA9000C20005F1200007F018FFD4E90012C0E958
:10AAA00000120020E2E710B50446032108F086F802
:10AAB0000146007800F00300022805D02046BDE8DA
:10AAC000104001F1140280E48A8A2046BDE810405B
:10AAD000AFE470B50446032108F070F8054601465E
:10AAE0002046FFF75BFD002816D029462046FFF7D9
:10AAF0005DFE002810D029462046FFF70AFD0028F9
:10AB00000AD029462046FFF7B3FC002804D0294686
:10AB10002046BDE8704091E570BD2DE9F0410C463E
:10AB200080461EE0E178427811FB02F1CAB28169E9
:10AB300001230E3007F0FFFE077860681C22C17900
:10AB4000491EC17107EB8701606802EBC10146181D
:10AB50003946204601F02CF818B1304601F037F89C
:10AB600020B16068C1790029DCD17FE7FEF74AFD9A
:10AB7000050000D1FFDF0A202872384600F0F6FFFA
:10AB800068813946204601F007F8014660680823CD
:10AB90004078C20006F1240007F0CDFED0E9001095
:10ABA000C5E90310A5F80280284600F0C0FFB07880
:10ABB00000B9FFDFB078401EB07057E770B50C46A3
:10ABC0000546032107F0FAFF01464068C279224496
:10ABD000C2712846BDE870409FE72DE9FE4F8246CE
:10ABE000507814460F464FF0000800284FD0012837
:10ABF00007D0022822D0FFDF2068B8606068F860C4
:10AC0000B8E602AB0E2208215046FFF784FB00286D
:10AC1000F2D00298152105230170217841700A2194
:10AC20004180C0F80480C0F80880A0F80C806288D9
:10AC300082810E20CDE90008082221E0A678304666
:10AC400000F094FF054606EB86012C22786802EBA3
:10AC5000C1010822465A02AB11465046FFF75BFB82
:10AC60000028C9D002980721017021784170042181
:10AC7000418008218580C680CDE9001805230A4659
:10AC800039465046FFF707FB87F8088072E6A6783A
:10AC9000022516B1022E13D0FFDF2A1D914602AB0A
:10ACA00008215046FFF737FB0028A5D00298012164
:10ACB000022E0170217841704580868002D005E027
:10ACC0000625EAE7A188C180E1880181CDE90098E5
:10ACD0000523082239465046D4E710B5044603211F
:10ACE00007F06CFF014600F108022046BDE8104065
:10ACF00073E72DE9F04F0F4605468DB01446508896
:10AD0000032107F05BFF4FF000088DF81480064622
:10AD1000ADF81680042F7BD36A78002A78D0287883
:10AD20004FF6FF794FF01C0A132834D008DC0128B5
:10AD300071D006284AD007286ED012280ED106E01E
:10AD400014286AD0152869D0162807D1AAE10C2F3B
:10AD500004D1307800F00301022907D0CDF8088033
:10AD6000CDF80C8068788DF808004CE040F00800C1
:10AD700030706878B07001208DF81400A888ADF8A4
:10AD80001800E888ADF81A002889ADF81C00688919
:10AD9000ADF81E0011E1B078904239D1307801074A
:10ADA00036D5062F34D120F0080030706088414637
:10ADB00060F31F4100200BF091FC02208DF814007D
:10ADC000ADF81890A888ADF81A00F6E0082F1FD14A
:10ADD000A888EF88814600F0BCFE804601463046D8
:10ADE00000F0E6FE18B1404600F0ABFEB8B1FC48FA
:10ADF000D0E90010CDE902106878ADF80C908DF81C
:10AE00000800ADF80E70608802AA3146FFF7E5FE33
:10AE10000DB0BDE8F08FB6E01EE041E0ECE07168F7
:10AE200008EB88002C2202EBC000085AB842EFD190
:10AE3000EB4802AAD0E90210CDE9021068788DF83B
:10AE4000080008F0FF058DF80A5060883146FFF7CA
:10AE5000C4FE224629461FE0082FD9D1B5F8048048
:10AE6000E88800F076FE07460146304600F0A0FE76
:10AE70000028CDD007EB870271680AEBC2000844B6
:10AE8000028A4245C4D101780829C1D14078697845
:10AE90008842BDD1F9B222463046FFF71EF9B7E726
:10AEA0000E2F7FF45BAFE9886F898B46B5F8089069
:10AEB0003046FFF775F9ABF14001402901D3092075
:10AEC0004AE0B9F1170F01D3172F01D20B2043E04D
:10AED00040280ED000EB800271680AEBC2000844E3
:10AEE0000178012903D140786978884290D00A20FE
:10AEF00032E03046FFF735F9014640282BD001EB10
:10AF0000810372680AEBC30002EB0008012288F893
:10AF100000206A7888F801207068AA884089B842C1
:10AF200000D93846AD8903232372A282E7812082AB
:10AF3000A4F80C906582084600F018FE6081A8F81D
:10AF40001490A8F81870A8F80E50A8F810B0204671
:10AF500000F0EDFD5CE7042005212172A4F80A80D1
:10AF6000E081012121739E49D1E90421CDE902212B
:10AF700069788DF80810ADF80A00608802AA314699
:10AF8000FFF72BFEE3E7062F89D3B07890421AD162
:10AF90003078010717D520F00800307060884146EE
:10AFA00060F31F4100200BF099FB02208DF8140084
:10AFB000A888ADF81800ADF81A906088224605A957
:10AFC000F9F7F7F824E704213046FFF700F90546C2
:10AFD0004028BFD0022083030090224629463046F5
:10AFE00000F003FE4146608865F30F2160F31F41C6
:10AFF00006200BF073FB0BE70E2FABD1042130467C
:10B00000FFF7E5F881464028A4D04146608869F3FF
:10B010000F2160F31F4106200BF060FBA8890B9005
:10B020006889099070682F894089B84200D93846EC
:10B030008346B5F80680A8880A90484600F096FD39
:10B0400060810B9818B1022000900B9B24E0B8F1AE
:10B05000170F1ED3172F1CD304202072099860826B
:10B06000E781A4F810B0A4F80C8009EB890271689C
:10B070000AEBC2000D18DDE90913A5F81480A5F844
:10B0800018B0E9812B82204600F051FD062028707F
:10B09000BEE601200B23009022464946304600F0D0
:10B0A000A4FDB5E6082F8DD1A9883046FFF778F8C2
:10B0B0000746402886D000F044FD00289BD107EBCE
:10B0C000870271680AEBC2000844804600F086FDE2
:10B0D000002890D1ED88B8F80E002844B0F5803FE4
:10B0E00005D360883A46314600F0B6FD90E6002D63
:10B0F000CED0A8F80E0060883A463146FFF73CFBF8
:10B1000008202072384600F031FD6081A5811EE7DD
:10B110002DE9F05F0C4601281FD0957992F8048044
:10B1200092F8056005EB85011F2202EBC10121F0B9
:10B13000030B08EB060111FB05F14FF6FF7202EA63
:10B14000C10909F1030115FB0611264F21F0031A6D
:10B15000BB6840B101283ED125E06168E57891F8EF
:10B1600000804E78DEE75946184607F062FB6060C3
:10B1700000B9FFDF5A460021606803F03EF9E57030
:10B180005146B86807F055FB6168486100B9FFDFB8
:10B190006068426902EB09018161606880F80080A3
:10B1A0006068467017E0606852464169184607F0CB
:10B1B0006BFB5A466168B86807F066FB032007F02E
:10B1C000A5FC0446032007F0A9FC201A012802D19F
:10B1D000B86807F023FB0BEB0A00BDE8F09F000006
:10B1E000905502002C0000200246002102208FE72B
:10B1F000F7B5FF4C0A2016462070009860B1002574
:10B200004FEA0D0007F0F7FA0021A1706670002DDB
:10B2100001D10099A160FEBD01250020F2E770B5C3
:10B220000C46154638220021204603F0E6F8012698
:10B2300066700A22002104F11C0003F0DEF805B953
:10B24000FFDF297A207861F301002070A8790028B7
:10B250002DD02A4621460020FFF75AFF6168402082
:10B26000E34A88706168C8706168087161684871F4
:10B270006168887161682888088161686888488188
:10B28000606886819078002811D061680620087770
:10B2900061682888C885616828884886606806854E
:10B2A000606869889288018681864685828570BD3E
:10B2B000C878002802D00022012029E7704770B525
:10B2C0000546002165F31F4100200BF007FA03211A
:10B2D000284607F073FC040000D1FFDF2146284612
:10B2E000FEF71CFF002804D0207840F010002070EA
:10B2F000012070BD70B505460C46032007F0F8FB31
:10B3000008B1002070BDBA4885708480012070BDEE
:10B310002DE9FF4180460E460F0CFEF773F905003C
:10B3200007D06F800321384607F048FC040008D19D
:10B3300006E004B03846BDE8F0411321F9F762BBDE
:10B34000FFDF5FEA080005D0B8F1060F18D0FFDF75
:10B35000BDE8FF8120782A4620F0080020700020F8
:10B36000ADF8020002208DF800004FF6FF70ADF836
:10B370000400ADF8060069463846F8F71AFFE7E71B
:10B38000C6F3072101EB81021C23606803EBC202B4
:10B39000805C042803D008280AD0FFDFD8E701200A
:10B3A00000904FF440432A46204600F01EFCCFE7B1
:10B3B00004B02A462046BDE8F041FEF78EBE2DE9D6
:10B3C000F05F05464089002790460C463E4682467F
:10B3D00000F0BFFB8146287AC01E08286BD2DFE848
:10B3E00000F00D04192058363C4772271026002C17
:10B3F0006CD0D5E90301C4E902015CE07027122694
:10B40000002C63D00A2205F10C0104F1080002F0BF
:10B41000CAFF50E071270C26002C57D0E868A060C6
:10B4200049E0742710269CB3D5E90301C4E9020161
:10B430006888032107F0C2FB8346FEF7E3F8024663
:10B440006888508049465846FEF7FEFD33E0752770
:10B450000A26ECB1A88920812DE076271426BCB1FC
:10B4600005F10C0004F1080307C883E8070022E097
:10B470007727102664B1D5E90301C4E90201688881
:10B48000032107F09BFB01466888FFF746FB12E0AB
:10B490001CE073270826CCB16888032107F08EFBD7
:10B4A00001460078C00606D56888FEF737FE10B959
:10B4B0006888F8F78CFAA8F800602CB12780A4F807
:10B4C00006A066806888A080002086E6A8F8006054
:10B4D000FAE72DE9FC410C461E461746804603213B
:10B4E00007F06CFB05460A2C0AD2DFE804F00505DC
:10B4F0000505050509090907042303E0062301E002
:10B50000FFDF0023CDE90076224629464046FEF7BC
:10B51000C2FEBDE8FC81F8B50546A0F57F40FF38C6
:10B520002BD0284607F07DFC040000D1FFDF204629
:10B5300007F001F8002821D001466A46204607F0AE
:10B540001CF800980321B0F80560284607F036FB88
:10B550000446052E13D0304600F0FBFA054601469E
:10B56000204600F025FB40B1606805EB85013E22D6
:10B5700002EBC101405A002800D00120F8BD007A3A
:10B580000028FAD00020F8BDF8B50446408807F03E
:10B5900048FC050000D1FFDF6A462846616800F0DC
:10B5A000C4FA01460098091F8BB230F8032F0280BD
:10B5B000428842800188994205D1042A08D0052A90
:10B5C00020D0062A16D022461946FFF799F9F8BD71
:10B5D000001D0E460546014622463046F6F74DFF51
:10B5E0000828F4D1224629463046FCF784F9F8BDF4
:10B5F0002C000020636864880A46011D2046FAF783
:10B60000A7F9F4E72246001DFFF773FBEFE770B5DB
:10B610000D460646032107F0D1FA040004D0207835
:10B62000000704D5112070BD43F2020070BD2A4608
:10B6300021463046FEF7C9FE18B92868606168687F
:10B64000A061207840F008002070002070BD70B527
:10B650000D460646032107F0B1FA040004D0207815
:10B66000000704D4082070BD43F2020070BD2A46D2
:10B6700021463046FEF7DDFE00B9A582207820F095
:10B6800008002070002070BD2DE9F04F0E4691B0EB
:10B690008046032107F092FA0446404607F0D3FBA8
:10B6A00007460020079008900990ADF830000A90F6
:10B6B00002900390049004B9FFDF0DF10809FFB96F
:10B6C000FFDF1DE038460BA9002206F0F7FD9DF8CC
:10B6D0002C0000F07F050A2D00D3FFDF6019017FE9
:10B6E000491E01779DF82C00000609D52A460CA9B1
:10B6F00007A8FEF7C0FD19F80510491C09F8051048
:10B70000761EF6B2DED204F13400F84D04F1260BB9
:10B71000DFF8DCA304F12A07069010E058460699EA
:10B7200000F08CFA064628700A2800D3FFDF5AF88A
:10B73000261040468847E08CC05DB04202D0208D84
:10B740000028EBD10A202870E94D4E4628350EE03E
:10B750000CA907A800F072FA0446375D55F82400DA
:10B7600000B9FFDF55F82420394640469047BDF820
:10B770001E000028ECD111B0BDE8F08F10B50321F8
:10B7800007F01CFA040000D1FFDF0A22002104F1B7
:10B790001C0002F032FE207840F00400207010BD42
:10B7A00010B50C46032107F009FA2044007F002859
:10B7B00000D0012010BD2DE9F84F8946154682467C
:10B7C000032107F0FBF9070004D02846F5F741FDF7
:10B7D00040B903E043F20200BDE8F88F4846F5F7B0
:10B7E0005EFD08B11020F7E7786828B16988008904
:10B7F000814201D90920EFE7B9F800001C2488B183
:10B8000000F0A7F980460146384600F0D1F988B12A
:10B8100008EB8800796804EBC000085C01280BD0B5
:10B820000820D9E73846FEF79CFC8046402807D11F
:10B830001320D1E70520CFE7FDF7E4FE06000BD08B
:10B8400008EB8800796804EBC0000C18B9F8000018
:10B8500020B1E88910B113E01120BDE7288817282E
:10B8600002D36888172801D20720B5E7686838B185
:10B870002B1D224641463846FFF7E9F80028ABD198
:10B8800004F10C0269462046FEF7E1FF2888608239
:10B890006888E082B9F8000030B102202070E889A1
:10B8A000A080E889A0B12BE003202070A889A080A7
:10B8B00078688178402905D180F802803946504661
:10B8C000FEF7D6FD404600F051F9A9F8000021E04E
:10B8D0007868218B4089884200D908462083A6F8E1
:10B8E00002A004203072B9F800007081E0897082F3
:10B8F000F181208B3082A08AB081304600F017F9A8
:10B900007868C178402905D180F8038039465046CF
:10B91000FEF7FFFD00205FE770B50D4606460321E8
:10B9200007F04CF904000ED0284600F012F9054645
:10B930000146204600F03CF918B1284600F001F914
:10B9400020B1052070BD43F2020070BD05EB8501FA
:10B950001C22606802EBC101084400F03FF908B105
:10B96000082070BD2A462146304600F075F90020B7
:10B9700070BD2DE9F0410C4617468046032107F0C3
:10B980001DF90546204600F0E4F8044695B101464D
:10B99000284600F00DF980B104EB84011C22686890
:10B9A00002EBC1014618304600F018F938B1082002
:10B9B000BDE8F08143F20200FAE70520F8E73B46D4
:10B9C000324621462846FFF742F80028F0D1E2B27D
:10B9D00029464046FEF75AFF708C0838082803D2E3
:10B9E00042484078F7F77CFA0020E1E72DE9F04182
:10B9F0000D4617468046032107F0E0F80446284626
:10BA000000F0A7F8064624B13846F5F722FC38B90D
:10BA100002E043F20200CBE73868F5F71AFC08B100
:10BA20001020C5E73146204600F0C2F860B106EBB1
:10BA300086011C22606802EBC1014518284600F00F
:10BA4000CDF818B10820B3E70520B1E7B888A98A76
:10BA5000884201D90C20ABE76168E88C4978B0EBEB
:10BA6000C10F01D31320A3E73146204600F094F81C
:10BA70000146606808234078C20005F1240006F002
:10BA800024FFD7E90012C0E90012F2B22146404675
:10BA9000FEF772FE00208BE72DE9F0470D461F46AA
:10BAA00090468146032107F089F80446284600F0B5
:10BAB00050F806463CB14DB13846F5F70EFC50B192
:10BAC0001020BDE8F08743F20200FAE7606858B141
:10BAD000A0F80C8027E03146204600F069F818B144
:10BAE000304600F02EF828B10520EAE72C000020AF
:10BAF000A855020006EB86011C22606802EBC1011A
:10BB00004518284600F06AF808B10820D9E7A5F8DA
:10BB10000880F2B221464846FEF7B8FE1FB1A88958
:10BB20006989084438800020CBE706F026BD0178FB
:10BB300021F00F01491C21F0F00110310170FDF7D7
:10BB400064BD20B94E48807808B1012070470020BC
:10BB500070474B498988884201D1002070474028AE
:10BB600001D2402000E0403880B2704710B5044652
:10BB7000402800D9FFDF2046FFF7E3FF10B140481F
:10BB8000808810BD4034A0B210BD40684269007882
:10BB9000484302EBC0007047C2784068037812FB4C
:10BBA00003F24378406901FB032100EBC1007047B9
:10BBB000C2788A4209D9406801EB81011C2202EB5C
:10BBC000C101405C08B10120704700207047007837
:10BBD000062801D901207047002070470078062808
:10BBE00001D00120704700207047F0B401EB8106BE
:10BBF0001C27446807EBC6063444049D05262670BE
:10BC0000E3802571F0BCFEF71FBA10B5418911B170
:10BC1000FFF7DDFF08B1002010BD012010BD10B5F9
:10BC2000C18C8278B1EBC20F04D9C18911B1FFF781
:10BC3000CEFF08B1002010BD012010BD10B50C468C
:10BC400001230A22011D06F076FE007821880122D8
:10BC500082409143218010BDF0B402EB82051C2686
:10BC60004C6806EBC505072363554B681C79402CCF
:10BC700003D11A71F0BCFEF791BCF0BC7047000014
:10BC80002C00002010B5EFF3108000F0010472B614
:10BC9000F8484178491C41704078012801D10AF0E8
:10BCA00055F9002C00D162B610BD70B5F14CA078EA
:10BCB00048B90125A570FFF7E5FF0AF058F920B152
:10BCC00000200AF022F9002070BD4FF08040E5709E
:10BCD000C0F80453F7E770B5EFF3108000F00105EA
:10BCE00072B6E44C607800B9FFDF6078401E607087
:10BCF000607808B90AF02EF9002D00D162B670BD47
:10BD0000DC4810B5817821B10021C1708170FFF746
:10BD1000E2FF002010BD10B504460AF028F9D5490D
:10BD20008978084000D001202060002010BD10B5A7
:10BD3000FFF7A8FF0AF01BF902220123CD4954079F
:10BD400028B1CD48026023610320087202E00A7224
:10BD5000C4F804330020887110BD2DE9F84FDFF8D6
:10BD600014934278817889F80420002689F8051018
:10BD7000074689F806600078DFF800B3354620B141
:10BD8000012811D0022811D0FFDF0AF002F94FF08C
:10BD9000804498B10AF004F9B0420FD130460AF05D
:10BDA00003F90028FAD042E00126EEE7FFF76AFF28
:10BDB00058460168C907FCD00226E6E70120E0608A
:10BDC000C4F80451AE490E600107D1F84412AC4AE0
:10BDD000C1F3423124321160A949343108604FF077
:10BDE000020AC4F804A3A060A6480168C94341F34D
:10BDF000001101F10108016841F01001016001E04A
:10BE000019F0D8F9D4F804010028F9D030460AF026
:10BE1000CBF80028FAD0B8F1000F04D19948016896
:10BE200021F010010160C4F808A3C4F8045199F886
:10BE300005004E4680B1387870B90AF098F880460F
:10BE40000AF030FA6FF00042B8F1000F02D0C6E9F4
:10BE5000032001E0C6E90302DBF80000C00701D0BF
:10BE60000AF081F8387810B13572BDE8F88F4FF0DC
:10BE70001808C4F808830127A7614FF42070ADF8B3
:10BE8000000000BFBDF80000411EADF80010F9D25F
:10BE9000C4F80C51C4F810517648C01D0AF096F849
:10BEA0003570FFF744FF67617549307920310860CC
:10BEB000C4F80483D9E770B5050000D1FFDF4FF067
:10BEC00080424FF0FF30C2F808030021C2F8001191
:10BED000C2F80411C2F80C11C2F81011654C61705F
:10BEE0000AF051F810B10120A0706070634800683A
:10BEF000C00701D00AF037F82846BDE870402CE7AB
:10BF00005C48007A002800D0012070472DE9FC5FD2
:10BF10005D48D0F800905C4A5C49083211608406A4
:10BF2000D4F8080100B10120D4F8001111B14FF08C
:10BF3000010801E04FF00008D4F8041101B101211B
:10BF40000191D4F80C1101B101210091D4F8101124
:10BF500001B10121474D8A4695F800B0002620B175
:10BF6000C4F80861012009F0D0FF4248C01D0AF062
:10BF700035F800B1FFDF0127B8F1000F10D0C4F889
:10BF80000873E87818B1EE70002009F0BEFF287A37
:10BF9000022805D103202872374802210160276159
:10BFA000019808B1C4F80461009850B1C4F80C615C
:10BFB000287A032800D0FFDF2F4806602F72FFF792
:10BFC0008AFEBAF1000F07D0C4F81061287A012860
:10BFD00001D100F05DF86761BBF1000F07D02E7052
:10BFE000287A012801D1FFF7A2FEFFF774FE21484D
:10BFF000C01D0AF009F82449091DC1F80090BDE8E8
:10C00000FC9F1C4810B5C01D09F0E8FF194940B15C
:10C01000012008704FF0E021C1F80002BDE8104097
:10C0200030E6087A012801D1FFF781FE1148BDE80A
:10C030001040C01D09F0E8BF70B50E4CA07808B9DB
:10C0400009F088FF01208507A861207A00260328CF
:10C050000AD100BFD5F80C0120B9002009F0A4FFD7
:10C060000028F7D1C5F80C6126724FF0FF30C5F8F3
:10C07000080370BD40000020340C00400C04004058
:10C080001805004010ED00E010050240010000011D
:10C0900070B5134C6079F0B1012803D0A179401E2E
:10C0A000814218DA09F063FF05460AF0FBF861796E
:10C0B000012902D9A179491CA1710DB1216900E0C2
:10C0C000E168411A022902DA11F1020FD1DC0DB147
:10C0D000206100E0E060BDE8704028E6C9E70000AC
:10C0E000400000200F4A12680D498A420CD11847BF
:10C0F0000C4A12680A4B9A4206D101B50AF0A4F81C
:10C100000AF077FBBDE8014007490968095808476C
:10C1100006480749054A064B70470000000000002A
:10C12000BEBAFECA5800002004000020B813002048
:10C13000B8130020F8B51D46DDE906470E000AD009
:10C1400006F081FE2346FF1DBCB231462A4600940C
:10C1500006F08DFAF8BDD0192246194602F023F9EF
:10C160002046F8BD70B50D4604461022002102F0AD
:10C1700044F9258117206081A07B40F00A00A0735C
:10C1800070BD4FF6FF720A80014602200AF0A6BA7F
:10C19000704700897047827BD30701D1920703D48F
:10C1A000808908800020704705207047827B9207B5
:10C1B00000D58181704701460020098841F6FE5272
:10C1C000114200D00120704700B50346807BC007B4
:10C1D00001D0052000BD59811846FFF7ECFFC007CC
:10C1E00003D0987B40F004009873987B40F00100E6
:10C1F0009873002000BD827B520700D509B14089A9
:10C20000704717207047827B61F3C30282737047C7
:10C210002DE9FC5F0E46044601789646012000FA9F
:10C2200001F14DF6FF5201EA020962684FF6FF7B09
:10C230001188594502D10920BDE8FC9FB9F1000FD2
:10C2400005D041F6FE55294201D00120F4E741EA2C
:10C25000090111801D0014D000232B7094F800C038
:10C26000052103221F464FF0020ABCF10E0F76D2C1
:10C27000DFE80CF0F909252F47646B77479193B4F9
:10C28000D1D80420D8E7616820898B7B9B0767D5CC
:10C2900017284AD30B89834247D38989172901D3A9
:10C2A000814242D185F800A0A5F801003280616882
:10C2B00088816068817B21F002018173C6E00420DF
:10C2C00028702089A5F801006089A5F80300318055
:10C2D000BCE0208A3188C01D1FFA80F8414524D374
:10C2E000062028702089A5F801006089A5F80300C0
:10C2F000A089A5F805000721208ACDE9000163691E
:10C3000041E00CF0FF00082810D008202870208998
:10C31000A5F801006089A5F8030031806A1D69460F
:10C3200004F10C0008F001FA10B15EE01020EDE716
:10C3300030889DF800100844308087E00A2028707B
:10C340002089A5F80100328044E00C202870208963
:10C35000A5F801006089A5F8030031803AE082E089
:10C3600064E02189338800EB41021FFA82F84345DB
:10C370003BD3B8F1050F38D30E222A700BEA4101E6
:10C38000CDE90010E36860882A467146FFF7D2FEC7
:10C39000A6F800805AE04020287060893188C01CCF
:10C3A0001FFA80F8414520D32878714620F03F00DD
:10C3B000123028702089A5F801006089CDE90002BB
:10C3C00060882A46E368FFF7B5FEA6F80080287863
:10C3D00040063BD461682089888037E0A089328894
:10C3E000401D1FFA80F8424501D204273DE0162087
:10C3F00028702089A5F801006089A5F80300A089AC
:10C40000CDE9000160882A4671462369FFF792FE54
:10C41000A6F80080DEE718202870207A6870A6F859
:10C4200000A013E061680A88920401D405271CE08B
:10C43000C9882289914201D0062716E01E21297061
:10C4400030806068018821F400510180B9F1000F4B
:10C450000BD061887823002202200AF095F86168E9
:10C460002078887006E0338003276068018821EA1D
:10C47000090101803846DFE62DE9FF4F85B01746F8
:10C48000129C0D001E461CD03078C10703D000F06E
:10C490003F00192801D9012100E000212046FFF7C3
:10C4A000AAFEA8420DD32088A0F57F41FF3908D00D
:10C4B0003078410601D4000605D5082009B0BDE852
:10C4C000F08F0720FAE700208DF800008DF80100BA
:10C4D00030786B1E00F03F0C0121A81E4FF0050ABA
:10C4E0004FF002094FF0030B9AB2BCF1200F75D246
:10C4F000DFE80CF08B10745E7468748C749C74B5F7
:10C5000074BA74C874D474E1747474F174EF74EE12
:10C5100074ED748B052D78D18DF80090A0788DF88E
:10C5200004007088ADF8060030798DF8010070784D
:10C5300000F03F000C2829D00ADCA0F102000928F5
:10C5400063D2DFE800F0126215621A621D622000F9
:10C55000122824D004DC0E281BD01028DBD11BE0CD
:10C5600016281FD01828D6D11FE02078800701E0B8
:10C5700020784007002848DAEEE020780007F9E745
:10C580002078C006F6E720788006F3E7207840069A
:10C59000F0E720780006EDE72088C005EAE720886C
:10C5A0004005E7E720880005E4E72088C004E1E7CC
:10C5B0002078800729D5032D27D18DF800B0B6F853
:10C5C000010081E0217849071FD5062D1DD381B2D6
:10C5D0007078012803D0022817D102E0C9E00220B8
:10C5E00000E0102004228DF8002072788DF80420DD
:10C5F000801CB1FBF0F2ADF8062092B242438A42B1
:10C6000003D10397ADF80890A6E079E02078000701
:10C6100076D598B282088DF800A0ADF80420B0EB72
:10C62000820F6DD10297ADF8061095E02178C9060A
:10C6300066D5022D64D381B206208DF80000707893
:10C6400002285DD3B1FBF0F28DF80400ADF80620AE
:10C6500092B242438A4253D1ADF808907BE02078F1
:10C6600080064DD5072003E0207840067FD50820BE
:10C670008DF80000A088ADF80400ADF80620ADF8F4
:10C68000081068E02078000671D50920ADF8042074
:10C690008DF80000ADF8061002975DE02188C9050D
:10C6A00065D5022D63D381B20A208DF80000707821
:10C6B00004285CD3C6E72088400558D5012D56D103
:10C6C0000B208DF80000A088ADF8040044E021E0C4
:10C6D00026E016E0FFE72088000548D5052D46D363
:10C6E0000C208DF80000A088ADF80400B6F8030017
:10C6F0006D1FADF80850ADF80600ADF80AA02AE0AD
:10C7000035E02088C00432D5012D30D10D208DF8C0
:10C71000000021E02088800429D4B6F80100E080E0
:10C72000A07B000723D5032D21D3307800F03F00F4
:10C730001B2818D00F208DF80000208840F40050EE
:10C74000A4F80000B6F80100ADF80400ED1EADF845
:10C750000650ADF808B0039769460598F5F7D6FB83
:10C76000050008D016E00E208DF80000EAE7072546
:10C7700010E008250EE0307800F03F001B2809D0BB
:10C780001D2807D00220059909F0A8FF208800F491
:10C7900000502080A07B400708D52046FFF70BFD06
:10C7A000C00703D1A07B20F00400A073284685E6D3
:10C7B0001FB5022806D101208DF8000088B2694615
:10C7C000F5F7A4FB1FBD0000F8B51D46DDE90647DF
:10C7D0000E000AD006F037FB2346FF1DBCB23146DF
:10C7E0002A46009405F043FFF8BDD01922461946A9
:10C7F00001F0D9FD2046F8BD2DE9FF4F8DB09B46D5
:10C80000DDE91B57DDF87CA00C46082B05D0E0695C
:10C8100001F0FEF850B11020D2E02888092140F044
:10C82000100028808AF80010022617E0E169012034
:10C830008871E2694FF420519180E1698872E06962
:10C8400042F601010181E0690021817328881121EC
:10C8500040F0200028808AF80010042638780A90DA
:10C860000A2038704FF0020904F118004D460C9070
:10C8700001F0C6FBB04681E0BBF1100F0ED1022DD6
:10C880000CD0A9EB0800801C80B20221CDE9001079
:10C8900005AB52461E990D98FFF796FFBDF816108E
:10C8A0001A98814203D9F74800790F9004E003D128
:10C8B0000A9808B138702FE04FF00201CDE9001955
:10C8C0000DF1160352461E990D98FFF77DFF1D9836
:10C8D0000088401B801B83B2C6F1FF00984200D243
:10C8E00003461E990BA8D9B15FF00002DDF878C0AD
:10C8F000CDE9032009EB060189B2CDE901C10F980A
:10C900000090BDF8161000220D9801F00EFC387052
:10C9100070B1C0B2832807D0BDF8160020833AE07A
:10C920000AEB09018A19E1E7022011B0BDE8F08F96
:10C93000BDF82C00811901F0FF08022D0DD09AF8E6
:10C940000120424506D1BDF82010814207D0B8F140
:10C95000FF0F04D09AF801801FE08AF80180C948CF
:10C9600000680178052902D1BDF81610818009EB15
:10C9700008001FFA80F905EB080085B2DDE90C100C
:10C9800005AB0F9A01F03FFB28B91D980088411BA9
:10C990004145BFF671AF022D13D0BBF1100F0CD182
:10C9A000A9EB0800801C81B20220CDE9000105AB93
:10C9B00052461E990D98FFF707FF1D98058000202D
:10C9C00038700020B1E72DE9F8439C46089E1346D5
:10C9D0000027B26B9AB3491F8CB2F18FA1F57F4546
:10C9E000FF3D05D05518AD882944891D8DB200E062
:10C9F00000252919B6F83C800831414520D82A4441
:10CA0000BCF8011022F8021BBCF8031022F8021B2C
:10CA1000984622F8024B914606F003FA4FF00C0CB0
:10CA200041464A462346CDF800C005F0ECFDF587A7
:10CA3000B16B00202944A41D2144088003E001E0DB
:10CA4000092700E083273846BDE8F88310B50B8836
:10CA5000848F9C420CD9846BE018048844B184888C
:10CA600024F40044A41D23440B801060002010BD5A
:10CA70000A2010BD2DE9F0478AB00025904689466E
:10CA80008246ADF8185007274BE005980688808845
:10CA9000000446D4A8F8006007A801950097029505
:10CAA000CDE903504FF4007300223146504601F0A7
:10CAB0003CFB04003CD1BDF81800ADF820000598FF
:10CAC00004888188B44216D10A0414D401950295D1
:10CAD000039521F400410097049541F48043428876
:10CAE0002146504601F0BFF804000BD1059881881B
:10CAF00041F40041818005AA08A94846FFF7A6FF36
:10CB00000400DCD0009705980295019503950495E3
:10CB10000188BDF81C300022504601F0A4F80A2C10
:10CB200006D105AA06A94846FFF790FF0400ACD03D
:10CB3000ADF8185004E00598818821F40041818007
:10CB400005AA06A94846FFF781FF0028F3D00A2C62
:10CB500003D020460AB0BDE8F0870020FAE710B500
:10CB60000C46896B86B051B10C218DF80010A18F55
:10CB7000ADF80810A16B01916946FAF751FB00204E
:10CB80004FF6FF71A063E187A08706B010BD2DE9C5
:10CB9000F0410D460746896B0020069E1446002989
:10CBA00011D0012B0FD1324629463846FFF762FFDC
:10CBB000002808D1002C06D0324629463846BDE868
:10CBC000F04100F034BFBDE8F0812DE9FC4114468E
:10CBD000DDE9087C0E46DDE90A15521DBCF800E0CF
:10CBE00092B2964502D20720BDE8FC81ACF8002045
:10CBF00017222A70A5F80160A5F803300522CDE9B7
:10CC000000423B462A46FFF7DFFD0020ECE770B507
:10CC10000C46154648220021204601F0EEFB04F1A7
:10CC2000080044F81C0F00204FF6FF71E06161849A
:10CC30002084A5841720E08494F82A0040F00A009C
:10CC400084F82A0070BD4FF6FF720A800146032067
:10CC500009F044BD30B585B00C460546FFF77FFFAF
:10CC6000A18E284629B101218DF800106946FAF7F6
:10CC7000D7FA0020E0622063606305B030BDB0F8F1
:10CC8000400070475C00002090F84620920703D4D3
:10CC9000408808800020F4E70620F2E790F846205C
:10CCA0009207EED5A0F84410EBE701460020098872
:10CCB0000A0700D5012011F0F00F01D040F002006A
:10CCC000CA0501D540F004008A0501D540F00800EE
:10CCD0004A0501D540F010000905D2D540F02000EA
:10CCE000CFE700B5034690F84600C00701D0062004
:10CCF00000BDA3F842101846FFF7D7FF10F03E0F13
:10CD000005D093F8460040F0040083F8460013F87D
:10CD1000460F40F001001870002000BD90F846203A
:10CD2000520700D511B1B0F84200AAE71720A8E7D2
:10CD300010F8462F61F3C3020270A2E72DE9FF4FFE
:10CD40009BB00E00DDE92B34DDE92978289D24D045
:10CD50002878C10703D000F03F00192801D901212C
:10CD600000E000212046FFF7D9FFB04215D3287814
:10CD7000410600F03F010CD41E290CD0218811F48B
:10CD80007F6F0AD13A8842B1A1F57F42FF3A04D0C1
:10CD900001E0122901D1000602D504201FB0C5E52B
:10CDA000FA491D984FF0000A08718DF818A08DF807
:10CDB0003CA00FAA0A60ADF81CA0ADF850A02978DD
:10CDC000994601F03F02701F5B1C04F1180C4FF0F4
:10CDD000060E4FF0040BCDF858C01F2A7ED2DFE8B4
:10CDE00002F07D7D107D267DAC7DF47DF37DF27DAE
:10CDF000F17DF47DF07D7D7DEF7DEE7D7D7D7D7D22
:10CE0000ED0094F84610B5F80100890701D5032E0E
:10CE100002D08DF818B01EE34FF40061ADF8501049
:10CE2000608003218DF83C10ADF84000D4E2052E5F
:10CE3000EFD1B5F801002083ADF81C00B5F8031060
:10CE4000618308B1884201D9012079E10020A072F4
:10CE500020814FF6FF702084169801F0D1F805204C
:10CE600089F800000220029083460AAB1D9A1699A9
:10CE70001B9801F0C8F890BB9DF82E00012804D043
:10CE8000022089F80100102003E0012089F8010048
:10CE900002200590002203A90BA807F046FCE8BB7E
:10CEA0009DF80C00059981423DD13988801CA1EB89
:10CEB0000B01814237DB02990220CDE900010DF11F
:10CEC0002A034A4641461B98FFF77EFC02980BF165
:10CED000020B801C81B217AA029101E09CE228E0BB
:10CEE00003A90BA807F021FC02999DF80C00CDE9DD
:10CEF000000117AB4A4641461B98FFF765FC9DF8B9
:10CF00000C000AAB0BEB00011FFA81FB02991D9A82
:10CF1000084480B2029016991B9800E003E001F0EB
:10CF200072F80028B6D0BBF1020F02D0A7F800B00B
:10CF30004FE20A208DF818004BE200210391072EE2
:10CF4000FFF467AFB5F801002083ADF81C00B5F819
:10CF50000320628300283FF477AF90423FF674AF1E
:10CF60000120A072B5F8050020810020A073E069BF
:10CF700000F04EFD78B9E16901208871E2694FF453
:10CF800020519180E1698872E16942F601000881CF
:10CF9000E06900218173F01F20841E9860620720E1
:10CFA0006084169801F02CF8072089F80000012011
:10CFB000049002900020ADF82A0028E019E29FE1D9
:10CFC00035E1E5E012E2A8E080E043E002980128C4
:10CFD00014D0E0698079012803D1BDF82800ADF8AC
:10CFE0000E00049803ABCDE900B04A4641461B98B9
:10CFF000FFF7EAFB0498001D80B20490BDF82A00F8
:10D00000ADF80C00ADF80E00059880B202900AABA6
:10D010001D9A16991B9800F0F6FF28B902983988D6
:10D02000001D05908142D1D20298012881D0E0698B
:10D030008079012803D1BDF82800ADF80E000498CE
:10D0400003ABCDE900B04A4641461B98FFF7BCFB55
:10D050000298BDE1072E02D0152E7FF4DAAEB5F8A6
:10D0600001102183ADF81C10B5F80320628300295C
:10D070003FF4EAAE91423FF6E7AE0121A1724FF0D4
:10D08000000BA4F808B084F80EB0052E07D0C0B28B
:10D09000691DE26907F02AFB00287FF44AAF4FF6CA
:10D0A000FF70208401A906AA14A8CDF800B081E879
:10D0B00085032878214600F03F031D9A1B98FFF74F
:10D0C0009BFB8246208BADF81C0082E10120032EE1
:10D0D000C3D14021ADF85010B5F801102183ADF84F
:10D0E0001C100AAAB8F1000F00D00023CDE90203FA
:10D0F00004921D98CDF80480009038880022401ECC
:10D1000083B21B9801F011F88DF8180090BB0B202A
:10D1100089F80000BDF8280035E04FF0010C052E1D
:10D120009BD18020ADF85000B5F801102183B5F8EF
:10D1300003002084ADF81C10B0F5007F03D9072050
:10D140008DF8180087E140F47C4222840CA8B8F1E5
:10D15000000F00D00023CDE90330CDE9018C1D98EC
:10D1600000903888401E83B21B9800F0DEFF8DF8D7
:10D17000180018B18328A8D10220BFE00D2189F83A
:10D180000010BDF83000401C22E100005C000020CF
:10D19000032E04D248067FF53CAE002018E1B5F816
:10D1A0000110ADF81C102878400602D58DF83CE03F
:10D1B00002E007208DF83C004FF000080320CDE985
:10D1C00002081E9BCDF810801D980193A6F1030B59
:10D1D00000901FFA8BF342461B9800F044FD8DF837
:10D1E00018008DF83C80297849060DD52088C005A7
:10D1F00006D5208BBDF81C10884201D1C4F82480CC
:10D2000040468DF81880E3E0832801D14FF0020AF0
:10D210004FF48070ADF85000BDF81C002083A4F8D6
:10D2200020B01E986062032060841321CDE0052E9B
:10D23000FFF4EFADB5F80110ADF81C10A28F6AB382
:10D24000A2F57F43FE3B29D008228DF83C2000BF89
:10D250004FF0000B0523CDE9023BDDF878C0CDF897
:10D2600010B01D9A80B2CDF804C040F40043009283
:10D27000B5F803201B9800F0F6FC8DF83CB04FF495
:10D2800000718DF81800ADF85010832810D0F8B157
:10D29000A18FA1F57F40FE3807D0DCE00B228DF88E
:10D2A0003C204FF6FE72A287D2E7A4F83CB0D2E051
:10D2B00000942B4631461E9A1B98FFF784FB8DF88D
:10D2C000180008B183284BD1BDF81C00208353E718
:10D2D00000942B4631461E9A1B98FFF774FB8DF87D
:10D2E0001800E8BBE18FA06B0844831D8DE888031C
:10D2F0004388828801881B98FFF767FC824668E0B4
:10D3000095F80180022E70D15FEA080002D0B8F1D2
:10D31000010F6AD109208DF83C0007A800908DF814
:10D3200040804346002221461B98FFF730FC8DF8D1
:10D3300042004FF0000B8DF843B050B9B8F1010F27
:10D3400012D0B8F1000F04D1A18FA1F57F40FF38B2
:10D350000AD0A08F40B18DF83CB04FF4806000E05F
:10D3600037E0ADF850000DE00FA91B98F9F758FF12
:10D3700082468DF83CB04FF48060ADF85000BAF1B1
:10D38000020F06D0FC480068C07928B18DF818005B
:10D3900027E0A4F8188044E0BAF1000F03D0812000
:10D3A0008DF818003DE007A8009043460122214671
:10D3B0001B98FFF7ECFB8DF8180021461B98FFF730
:10D3C000CEFB9DF8180020B9192189F80010012022
:10D3D00038809DF83C0020B10FA91B98F9F720FF79
:10D3E0008246BAF1000F33D01BE018E08DF818E048
:10D3F00031E02078000712D5012E10D10A208DF8D7
:10D400003C00E088ADF8400003201B9909F066F964
:10D410000820ADF85000C0E648067FF5FAAC4FF0A2
:10D42000040A2088BDF8501008432080BDF8500041
:10D4300080050BD5A18FA1F57F40FE3806D11E983F
:10D44000E06228982063A6864FF0030A5046A5E4C0
:10D450009DF8180078B1012089F80000297889F832
:10D460000110BDF81C10A9F802109DF8181089F8D9
:10D470000410052038802088BDF850108843208093
:10D48000E4E72DE9FF4F8846087895B001218140F7
:10D490004FF20900249C0140ADF820102088DDF8EF
:10D4A0008890A0F57F424FF0000AFF3A06D039B1CC
:10D4B000000705D5012019B0BDE8F08F0820FAE774
:10D4C000239E4FF0000B0EA886F800B018995D4619
:10D4D0000988ADF83410A8498DF81CB0179A0A7164
:10D4E0008DF838B0086098F8000001283BD0022879
:10D4F00009D003286FD1307820F03F001D30307004
:10D50000B8F80400E08098F800100320022904D144
:10D51000317821F03F011B31317094F84610090732
:10D5200059D505ABB9F1000F13D0002102AA82E84A
:10D530000B000720CDE90009BDF83400B8F804104D
:10D54000C01E83B20022159800F0EFFD0028D1D153
:10D5500001E0F11CEAE7B8F80400A6F80100BDF804
:10D560001400C01C04E198F805108DF81C1098F800
:10D570000400012806D04FF4007A02282CD003289A
:10D58000B8D16CE12188B8F8080011F40061ADF859
:10D59000201020D017281CD3B4F84010814218D393
:10D5A000B4F84410172901D3814212D1317821F007
:10D5B0003F01C91C3170A6F801000321ADF83410F9
:10D5C000A4F8440094F8460020F0020084F84600D5
:10D5D00065E105257EE177E1208808F1080700F480
:10D5E000FE60ADF8200010F0F00F1BD010F0C00F5F
:10D5F00003D03888228B9042EBD199B9B878C00714
:10D6000010D0B9680720CDE902B1CDF804B0009080
:10D61000CDF810B0FB88BA883988159800F023FB44
:10D620000028D6D12398BDF82010401C80294ED068
:10D6300006DC10290DD020290BD0402987D124E009
:10D64000B1F5807F6ED051457ED0B1F5806F97D116
:10D65000DEE0C80601D5082000E0102082460DA9B2
:10D6600007AA0520CDE902218DF83800ADF83CB0BD
:10D67000CDE9049608A93888CDE900015346072270
:10D6800021461598FFF7B8F8A8E09DF81C20012165
:10D690004FF00A0A002A9BD105ABB9F1000F00D068
:10D6A0000020CDE902100720CDE90009BDF83400C3
:10D6B0000493401E83B2218B0022159800F035FDA3
:10D6C0008DF81C000B203070BDF8140020E09DF890
:10D6D0001C2001214FF00C0A002A22D113ABB9F112
:10D6E000000F00D00020CDE902100720CDE900098D
:10D6F0000493BDF83400228C401E83B2218B159810
:10D7000000F013FD8DF81C000D203070BDF84C00AA
:10D71000401CADF8340005208DF83800208BADF8A2
:10D720003C00BCE03888218B88427FF452AF9DF8E2
:10D730001C004FF0120A00281CD1606AA8B1B8780A
:10D74000C0073FF446AF00E018E0BA680720CDE913
:10D7500002B2CDF804B00090CDF810B0FB88BA88C2
:10D76000159800F080FA8DF81C001320307001200D
:10D77000ADF8340093E000005C0000203988208B75
:10D780008142D2D19DF81C004FF0160A0028A06BF0
:10D7900008D0E0B34FF6FF7000215F46ADF808B047
:10D7A000019027E068B1B978C907BED1E18F0DAB10
:10D7B0000844821D03968DE80C0243888288018804
:10D7C00009E0B878C007BCD0BA680DAB03968DE805
:10D7D0000C02BB88FA881598FFF7F7F905005ED0B0
:10D7E000072D72D076E0019005AA02A92046FFF726
:10D7F0002DF90146E28FBDF80800824201D00029D0
:10D80000F1D0E08FA16B084407800198E08746E0E3
:10D810009DF81C004FF0180A40B1208BC8B1388821
:10D82000208321461598FFF79AF938E004F1180093
:10D830000090237E012221461598FFF7A8F98DF864
:10D840001C000028EDD1192030700120ADF8340003
:10D85000E7E7052521461598FFF781F93AE020888A
:10D8600000F40070ADF8200050452DD1A08FA0F538
:10D870007F41FE3901D006252CE0D8F808004FF092
:10D88000160A48B1A063B8F80C10A1874FF6FF71D3
:10D89000E187A0F800B002E04FF6FF70A087BDF866
:10D8A000200030F47F611AD07823002203201599DC
:10D8B00008F06AFE98F8000020712088BDF820105A
:10D8C000084320800EE000E007252088BDF82010E6
:10D8D00088432080208810F47F6F1CD03AE0218894
:10D8E000814321809DF8380020B10EA91598F9F7E1
:10D8F00097FC05469DF81C000028EBD086F801A097
:10D9000001203070208B70809DF81C003071052044
:10D91000ADF83400DEE7A18EE1B118980DAB0088B8
:10D92000ADF834002398CDE90304CDE90139206B2B
:10D930000090E36A179A1598FFF700FA0546012050
:10D940008DF838000EA91598F9F76AFC00B1054664
:10D95000A4F834B094F8460040070AD52046FFF7F3
:10D96000A4F910F03E0F04D114F8460F20F0040083
:10D9700020701898BDF83410018028469BE500B54A
:10D9800085B0032806D102208DF8000088B26946D0
:10D99000F9F746FC05B000BD10B5384C0B7822688D
:10D9A000012B02D0022B2AD111E013780BB1052BE9
:10D9B00001D10423137023688A889A802268CB8857
:10D9C000D38022680B891381498951810DE08B88AE
:10D9D00093802268CB88D38022680B8913814B897E
:10D9E00053818B899381096911612168F9F718FCCA
:10D9F000226800210228117003D0002800D0812065
:10DA000010BD832010BD806B002800D0012070471E
:10DA10008178012909D10088B0F5205F03D042F652
:10DA20000101884201D10020704707207047F0B5FE
:10DA300087B0002415460E460746ADF8184011E0A1
:10DA400005980088288005980194811DCDE9024140
:10DA5000072104940091838842880188384600F0A9
:10DA600002F930B905AA06A93046FEF7EFFF0028F3
:10DA7000E6D00A2800D1002007B0F0BD5C000020ED
:10DA800010B58B7883B102789A4205D10B885BB1CF
:10DA900002E08B79091D4BB18B789A42F9D1B0F82D
:10DAA00001300C88A342F4D1002010BD812010BDAC
:10DAB000072826D012B1012A27D103E0497801F0C6
:10DAC000070102E04978C1F3C20105291DD2DFE850
:10DAD00001F00318080C12000AB10320704702205D
:10DAE000704704280DD250B10DE0052809D2801EE0
:10DAF000022808D303E0062803D0032803D005201A
:10DB00007047002070470F20704781207047C0B2D7
:10DB100082060BD4000607D5FA48807A4143C01D1F
:10DB200001EBD00080B27047084670470020704774
:10DB300070B513880B800B781C0625D5F14CA47AA0
:10DB4000844204D843F010000870002070BD95682E
:10DB500000F0070605EBD0052D78F54065F30413BA
:10DB60000B701378D17803F0030341EA032140F2EC
:10DB70000123B1FBF3F503FB15119268E41D00FBD3
:10DB8000012000EBD40070BD906870BD37B514461D
:10DB9000BDF804101180117841F0040111709DF856
:10DBA00004100A061ED5D74AA368C1F30011927A61
:10DBB000824208D8FE2811D1D21DD2084942184607
:10DBC00000F01BFC0AE003EBD00200F00703012584
:10DBD00010789D40A843994008431070207820F0A9
:10DBE000100020703EBD2DE9F0410746C81C0E46CE
:10DBF00020F00300B04202D08620BDE8F081C14D84
:10DC0000002034462E60AF802881AA72E8801AE096
:10DC1000E988491CE980810614D4E17800F003000A
:10DC200041EA002040F20121B0FBF1F201FB1201B8
:10DC30002068FFF76CFF2989084480B22881381AD0
:10DC40003044A0600C3420784107E1D40020D4E7B0
:10DC5000AC4801220189C08800EB400002EB800043
:10DC6000084480B270472DE9FF4F89B01646DDE9C0
:10DC7000168A0F46994623F44045084600F054FBA7
:10DC8000040002D02078400703D401200DB0BDE885
:10DC9000F08F099804F058FF02902078000606D50E
:10DCA0009848817A0298814201D88720EEE722467F
:10DCB00001A90298FFF73CFF834600208DF80C0075
:10DCC0004046B8F1070F1AD001222146FFF7F0FEB7
:10DCD0000028DBD12078400611D502208DF80C00F9
:10DCE000ADF81070BDF80400ADF81200ADF8146086
:10DCF0001898ADF81650CDF81CA0ADF818005FEAE2
:10DD0000094004D500252E46A84601270CE02178BD
:10DD1000E07801F0030140EA012040F20121B0FB6C
:10DD2000F1F2804601FB12875FEA494009D5B84508
:10DD300007D1A178207901F0030140EA0120B04227
:10DD400001D3BE4201D90720A0E7A8191FFA80F924
:10DD5000B94501D90D2099E79DF80C0028B103A918
:10DD60000998F9F75BFA002890D1B84507D1A07857
:10DD70004FEA192161F30100A07084F804901A9809
:10DD800000B10580199850EA0A0027D0199830B1DF
:10DD90000BEB06002A46199900F005FB0EE00BEB91
:10DDA00006085746189E099805F03BF82B46F61DC5
:10DDB000B5B239464246009504F025FC224601A939
:10DDC0000298FFF7B5FE9DF80400224620F01000EF
:10DDD0008DF80400DDE90110FFF7D8FE002055E7BB
:10DDE0002DE9FF4FDFF81C91824685B0B9F8061087
:10DDF000D9F8000001EB410100EB810440F2012061
:10DE0000B2FBF0F1174600FB1175DDE9138B4E46AE
:10DE100029460698FFF77BFE0346FFF719FF1844D3
:10DE2000B1880C30884202D9842009B02FE70698C7
:10DE3000C6B2300603D5B00601D50620F5E7B9F81D
:10DE40000620521C92B2A9F80620BBF1000F01D0A7
:10DE5000ABF80020B00602D5C4F808800AE0B9F893
:10DE600008201A4492B2A9F80820D9F80000891AAB
:10DE70000844A0602246FE200699FFF787FEE7705F
:10DE800025712078390A61F301002A0AA17840F04F
:10DE9000040062F30101A17020709AF80200607121
:10DEA000BAF80000E08000252573300602D599F805
:10DEB0000A7000E00127B00601D54FF000084E4679
:10DEC00000244FF007090FE0CDE902580195CDF885
:10DED00000900495F1882046129B089AFFF7C3FE34
:10DEE0000028A2D1641CE4B2BC42EDD300209CE720
:10DEF00000B5FFF7ADFE03490C308A88904203D984
:10DF0000842000BD00060020CA88086802EB420396
:10DF100000EB8300521C037823F004030370CA80D3
:10DF2000002101730846ECE72DE9F047804600F038
:10DF3000FBF9070005D000264446F74D40F20129C1
:10DF400016E00120BDE8F087204600F0EDF90278E8
:10DF5000C17802F0030241EA0222B2FBF9F309FBA5
:10DF600013210068FFF7D3FD3044641C86B2A4B2CD
:10DF7000E988601E8142E7DCA8F10100E880288979
:10DF8000801B288100203870DCE710B5144631B1C1
:10DF9000491E218004F0D8FDA070002010BD012092
:10DFA00010BD70B50446DC48C188036801E0401C20
:10DFB00020802088884207D200EB400213EB8202C7
:10DFC00002D015786D07F2D580B2884216D2AAB178
:10DFD0005079A072D08820819178107901F00301E6
:10DFE00040EA0120A081A078E11CFFF7A1FD20619B
:10DFF0002088401C2080E080002070BD0A2070BD79
:10E000000121018270472DE9FF4F85B04FF6FF795E
:10E010008246A3F8009048681E460D4680788DF829
:10E02000060048680088ADF8040000208DF80A005A
:10E03000088A0C88A04200D304462C8251E038782C
:10E04000400708D4641C288AA4B2401C288208F126
:10E050000100C0B246E0288A401C2882781D696809
:10E06000FFF70EFDD8BB3188494501D1601E3080D5
:10E070003188A1EB080030806888A04238D3B87896
:10E08000397900F0030041EA002801A9781DFFF763
:10E09000F7FC20BB298949452ED000223946079834
:10E0A000FFF706FDD8B92989414518D1E9680391E0
:10E0B000B5F80AC0D7F808B05046CDF800C004F053
:10E0C000B0FEDDF800C05A460CF1070C1FFA8CFCBC
:10E0D00043460399CDF800C004F05FFA60B1641CB8
:10E0E000A4B200208046204600F01EF90700A6D109
:10E0F000641E2C820A2098E674807879B071F888C2
:10E10000B0803978F87801F0030140EA012070818D
:10E11000A6F80C80504604F017FD3A4606F10801B7
:10E12000FFF706FD306100207FE62DE9FF4F87B045
:10E1300081461C469246DDF860B0DDF854800898B0
:10E1400000F0F2F8050002D02878400702D4012040
:10E150000BB09CE5484604F0F7FC2978090605D584
:10E160006D49897A814201D88720F1E7CAF309060F
:10E170002A4601A9FFF7DCFC0746149807281CD0A3
:10E1800000222946FFF794FC0028E1D128784006B8
:10E1900013D501208DF808000898ADF80C00BDF8E3
:10E1A0000400ADF80E00ADF81060ADF8124002A901
:10E1B0004846F9F733F80028CAD12978E87801F001
:10E1C000030140EA0121AA78287902F0030240EA1B
:10E1D0000220564507D0B1F5007F04D9611E814267
:10E1E00001DD0B20B4E7864201D90720B0E7801B90
:10E1F00085B2A54200D92546BBF1000F01D0ABF88E
:10E200000050179818B1B9192A4600F0CCF8B8F1A7
:10E21000000F0DD03E4448464446169F04F013FEBE
:10E220002146FF1DBCB232462B46009404F01FFA73
:10E2300000208DE72DE9F04107461D4616460846A9
:10E2400000F072F8040002D02078400701D40120C9
:10E25000D3E4384604F078FC2178090605D52E4928
:10E26000897A814201D88720C7E422463146FFF7E8
:10E270005FFC65B12178E07801F0030140EA0120FC
:10E28000B0F5007F01D8012000E0002028700020B8
:10E29000B3E42DE9F04107461D461646084600F056
:10E2A00043F8040002D02078400701D40120A4E400
:10E2B000384604F049FC2178090605D51649897AC3
:10E2C000814201D8872098E422463146FFF75EFC60
:10E2D000FF2D14D02178E07801F0030240EA0220FB
:10E2E00040F20122B0FBF2F302FB130015B900F279
:10E2F000012080B2E070000A60F30101217000206B
:10E300007BE410B50C4600F00FF810B10178490716
:10E3100004D4012010BD000000060020C188218027
:10E320004079A0700020F5E70749CA88824209D3E6
:10E3300040B1096800EB40006FF00B0202EB800077
:10E3400008447047002070470006002070B504465E
:10E350000D4621462B460AB9002070BD01E0491C3C
:10E360005B1C501E021E03D008781E78B042F6D007
:10E3700008781E78801BF0E730B50C46014623462E
:10E38000051B954206D202E0521E9D5C8D54002A68
:10E39000FAD107E004E01D780D70491C5B1C521E89
:10E3A000002AF8D130BDF0B50E460146334680EA6A
:10E3B000030404F00304B4B906E002B9F0BD13F895
:10E3C000017B01F8017B521E01F00307002FF4D1FD
:10E3D0000C461D4602E080CD80C4121F042AFAD2EA
:10E3E00021462B4600BF04E013F8014B01F8014B16
:10E3F000521E002AF8D100BFE0E7F0B50C460146F6
:10E40000E6B204E002B9F0BD01F8016B521E01F062
:10E410000307002FF6D10B46E5B245EA052545EA8C
:10E42000054501E020C3121F042AFBD2194602E071
:10E4300001F8016B521E002AFAD100BFE3E710B5C4
:10E4400008F0CBFBF4F730FA08F042FABDE81040D0
:10E4500008F00ABB202834BF0120002070470123A8
:10E4600003FA00F04FF0A042002914BFC2F80C05D7
:10E47000C2F8080570474FF0A041012202FA00F0EF
:10E48000C1F81805704770B50346002002466FF0CA
:10E490002F050EE09C5CA4F130060A2E02D34FF04B
:10E4A000FF3070BD00EB800005EB4000521C2044A3
:10E4B000D2B28A42EED370BD30B50A230BE0B0FB76
:10E4C000F3F403FB1404B0FBF3F08D183034521E48
:10E4D00005F8014CD2B2002AF1D130BD30B500238D
:10E4E0004FF6FF7510E0040A44EA002084B2C85CCD
:10E4F0006040C0F30314604005EA00344440E0B2D9
:10E500005B1C84EA40109BB29342ECD330BD000008
:10E510002DE9F041FE4B0026012793F864501C784A
:10E5200093F868C0B8B183F89140A3F8921083F8CB
:10E53000902083F88E70BCF1000F0CBF83F89460BC
:10E5400083F89450F3488068008804F06AFCBDE8C2
:10E55000F04104F0FFB84FF6FF7083F89140A3F844
:10E56000920083F8902083F88E70BCF1000F14BFE6
:10E5700083F8945083F89460BDE8F0812DE9F04170
:10E58000E44D296891F89C200024012A23D091F8B9
:10E590009620012A30D091F86C301422DC4E0127ED
:10E5A000012B32D091F88E30012B4FD091F8A6205C
:10E5B000012A1CBF0020BDE8F08144701F2200F832
:10E5C000042B2222A731FFF7EEFE286880F8A64030
:10E5D0000120BDE8F08144701B220270D1F89D201B
:10E5E0004260D1F8A120826091F8A520027381F8E1
:10E5F0009C400120BDE8F081447007220270D1F8F0
:10E600009820426081F89640E2E78046447000F826
:10E61000042B20226E31FFF7C6FE88F808702868A8
:10E6200080F86C4090F86E000028D1D1B6F87000E8
:10E63000A6F89800A868417B86F89A1086F896702C
:10E64000008804F0EEFB04F094F8C1E791F86C3018
:10E65000012B0BD0447017220270D1F89020426039
:10E66000B1F89420028181F88E40B1E78046447071
:10E6700000F8042B20226E31FFF795FE88F8087011
:10E68000286880F86C4090F86E000028A0D1CDE793
:10E69000A048006890F86C10002914BFB0F8700012
:10E6A0004FF6FF70704770B59A4C064620680028F8
:10E6B00008BFFFDF0025206845706660002808BF9E
:10E6C000FFDF2068417800291CBFFFDF70BDCC222E
:10E6D0000021FFF792FE2068FF2101707F2180F862
:10E6E000371013214184282180F86910012180F816
:10E6F0005C1080F8615008F0C1FFBDE8704008F080
:10E7000014B984490968097881420CBF01200020AE
:10E7100070478048006890F82200C0F340007047BE
:10E720007C48006890F8220000F0010070477948AA
:10E73000006890F82200C0F3001070472DE9F04304
:10E740007448D0F800C09CF82400BCF82240C0F304
:10E750008001C0F34002114400F001000144C4F301
:10E760000010F0B1132C17D009DC102C02BF6A483E
:10E7700030F81100BDE8F083122C0DD008E0152C04
:10E7800008BF664809D01D2C04BF6548BDE8F0836A
:10E79000FFDF0020BDE8F083624830F81100BDE8DB
:10E7A000F0839CF85E209CF85F002E2600234FF437
:10E7B0007A774FF014084FF04009022A04BF4AF25A
:10E7C000D745B5FBF7F510D0012A04BF4AF22F75E3
:10E7D000B5FBF7F510D04AF62315B5FBF7F5082A77
:10E7E00008BF4E4613D0042A18D01E46082A0ED061
:10E7F000042A13D0022A49D003F12806042A0FD094
:10E80000082A1CBF4FF01908082204D00AE04FF074
:10E81000140806F5A8764FF0400203E006F5A87646
:10E820004FF0100218FB026212FB0152C1EB011102
:10E830003D4D01EB810105EB8101114414F0010F05
:10E840004FF4C8724FF4BF7504BFC4F34006002EE6
:10E850005DD0C4F3400601F5A571EEB1082804BFF0
:10E86000174640260CD0042804BF2F46102607D098
:10E87000022807BF03F11807042603F1280708261A
:10E8800006EB860808EB86163E441BE003F11806EB
:10E890004FF019080422C5E7082804BF1646402790
:10E8A0000CD0042804BF2E46102707D0022807BF2B
:10E8B00003F11806042703F12806082707EB87173A
:10E8C00006EB870631449C31082804BF16464027D2
:10E8D0000CD0042804BF2E46102707D0022807BFFB
:10E8E00003F11806042703F128060827C7EBC7071A
:10E8F00007EB470706EB47063144983114F0010F48
:10E9000027D0082808BF40201CD004280EE063E070
:10E910000C060020640000200C5602001456020071
:10E920008F89130004560200D4FEFFFF04BF2A465D
:10E93000102007D0022807BF03F11802042003F1BA
:10E940002802082000EB400303EB001010440144B0
:10E950003EE0082804BF144640260CD0042804BF1B
:10E960002C46102607D0022807BF03F118040426FE
:10E9700003F12804082606EB8616BCF840C004EB19
:10E9800086042144BCF1EB0F22D944F255240CF14A
:10E990000B0C0CFB04FC4FEA9C5C082807D00428F5
:10E9A00002D0022805D008E02A46102008E04020C6
:10E9B00006E003F11802042002E003F12802082017
:10E9C00000EB801002EB800000F5A5700CFB00113D
:10E9D00001F5B370BDE8F08301F5A574082804BF04
:10E9E000164640210CD0042804BF2E46102107D023
:10E9F000022807BF03F11806042103F128060821A5
:10EA000001EB8111BCF848C006EB81012144BCF147
:10EA1000EB0FDDD944F255240CF10B0C0CFB04FC7C
:10EA20004FEA9C5C0828C2D00428BDD00228C4D17B
:10EA3000BFE7FE4840F271210068806A4843704792
:10EA4000FA48006890F83600002818BF0120704787
:10EA500010B5F74C207B022818BF032808D1207D71
:10EA600004F115010DF0C9FB08281CBF012010BDE1
:10EA7000207B002816BF022800200120BDE810409E
:10EA800009F0FCB9EA4908737047E849096881F858
:10EA9000300070472DE9F047E44C2168087B0028DE
:10EAA00016BF022800200120487301F10E0109F071
:10EAB000CFF92168087B022816BF03280122002213
:10EAC00081F82F204FF0080081F82D00487B01F1DC
:10EAD0000E034FF001064FF00007012804BF5B79D9
:10EAE00013F0C00F0AD001F10E03012804D15879A8
:10EAF00000F0C000402801D0002000E0012081F893
:10EB00002E00002A04BF91F8220010F0040F07D055
:10EB1000087D01F115010DF070FB216881F82D00D1
:10EB20002068476006F0B2F92168C14D4FF0000936
:10EB3000886095F82D000DF07CFB804695F82F003D
:10EB4000002818BFB8F1000F04D095F82D000DF083
:10EB500035F968B195F8300000281CBF95F82E00F3
:10EB600000281DD0697B05F10E0001290ED012E0AE
:10EB70006E734A4605F10E01404609F0BFF995F85B
:10EB80002D1005F10E000DF04BFC09E0407900F06E
:10EB9000C000402831D0394605F10E0009F0E6F9F1
:10EBA0002068C77690F8220010F0040F08BFBDE877
:10EBB000F087002795F82D000DF0B6F9050008BF85
:10EBC000BDE8F08710210EF0B2F9002818BFBDE8AB
:10EBD000F08720683A4600F11C01C676284609F005
:10EBE0008DF9206800F11C0160680EF06BFC606814
:10EBF000BDE8F04701210EF080BC0DF04EFC4A4606
:10EC000005F10E0109F07AF9CAE7884A1268137B08
:10EC10000370D2F80E000860508A8880704778B57B
:10EC200083490446814D407B08732A682078107020
:10EC30006088ADF8000080B200F00101C0F340032D
:10EC400041EA4301C0F3800341EA8301C0F3C003FA
:10EC500041EAC301C0F3001341EA0311C0F34013BA
:10EC600041EA4311C0F3801041EA80105084E07DF6
:10EC7000012808BF012603D0022814BFFFDF0226A7
:10EC8000286880F85E60607E012808BF012603D0F6
:10EC9000022814BFFFDF0226286880F85F60217B0E
:10ECA00080F82410418C1D290CBF0021616881620D
:10ECB000617D80F83610A17B002916BF0229002152
:10ECC00001210175D4F80F10C0F81510B4F8131015
:10ECD000A0F81910A17E90F86B2061F3071280F85C
:10ECE0006B20E17E012918BF002180F8341000203C
:10ECF00078BD4E480068408CC0F3001131B1C0F3BC
:10ED00008000002804BF1F20704702E0C0F34001CC
:10ED100009B10020704710F0010F14BFEE20FF2052
:10ED2000704742480068408CC0F3001119B1C0F32D
:10ED3000800028B102E0C0F3400008B10020704715
:10ED4000012070473949002209684A664B8C1D2B07
:10ED50000CBF81F8682081F8680070470023334AAF
:10ED6000126882F85D30D164A2F85000012082F868
:10ED70005D0070472D4A0023126882F85C30A2F8CB
:10ED800058000120516582F85C00704727490968E6
:10ED900081F8350070472549096881F8610070479E
:10EDA0002248006890F9610070472048006890F898
:10EDB0002200C0F3401070471C48006890F8220001
:10EDC000C0F3C0007047012070471848006890F8F1
:10EDD0005F00704770B508F032FC08F011FC08F0D5
:10EDE000D2FA08F07FFB114C2068416E491C416645
:10EDF00090F83300002530B108F040FC07F095FD95
:10EE0000206880F833502068457090F8381021B1A0
:10EE1000BDE87040042009F0B6BC90F8681009B352
:10EE2000406E81421ED8042004E0000064000020EF
:10EE30000C06002009F0A7FC206890F8220010F0D2
:10EE4000010F07D0A06843220188BDE8704001206F
:10EE5000FFF75EBBBDE8704043224FF6FF71002014
:10EE6000FFF756BBBDE87040002009F08CBC2DE9CF
:10EE7000F04782B00F468246FE4E4FF000093068E0
:10EE8000458C15F0030F10D015F0010F05F00200AE
:10EE900005D0002808BF4FF0010906D004E0002883
:10EEA00018BF4FF0020900D1FFDF4FF000084446C1
:10EEB00015F0010F05F002000DD080B915F0040F18
:10EEC0000DD048F00800002F1CBF40F0010040F0BA
:10EED000020438D06EE010B115F0040F0DD015F01B
:10EEE000070F10D015F0010F05F002002ED00028FA
:10EEF00008BF15F0040F1FD035E0002F18BF48F0F1
:10EF0000090457D12CE02FB148F0080415F0200F68
:10EF10004CD04FE0306805F02001B0F848000843BD
:10EF200008BF48F0010445D048F0180415F0200F40
:10EF300008BF44F001043DE048F00800002F18BF6E
:10EF400040F0010436D140F0100433E0002818BF2F
:10EF500015F0040F07D0002F18BF48F00B0429D17B
:10EF600048F0180426E015F0030F22D115F0040F25
:10EF70001FD03FB128F0020040F0080415F0200F28
:10EF800014D017E0306805F02001B0F848000843BD
:10EF900008BF48F003040DD048F0180015F0200F0A
:10EFA00008BF40F0010040F0020403E024F0010437
:10EFB00000E0FFDF15F0400F12D07FB93068B0F8E5
:10EFC0004810002904BF408C10F0010F06D110F04A
:10EFD000020F04BF10F0200F15F0010F44F04004A1
:10EFE0007068A0F80080017821F0200101704FF0D6
:10EFF00007010EF033FA494670680EF026FC2146F0
:10F0000070680EF02EFC14F0010F0CD04FF00603C8
:10F010004FF00002984970680EF0FDFB3068417BAC
:10F0200070680EF05DFA14F0020F18D0D6E90010E7
:10F03000BAF1000F4FF006034FF0010207D01C3168
:10F040000EF0E9FB012170680EF057FA07E0153168
:10F050000EF0E1FB3068017D70680EF04EFA14F09E
:10F06000040F18BFFFDF14F0080F19D0CDF800808F
:10F070003068BDF800200223B0F86A1061F30B027B
:10F08000ADF8002090F86B00032201099DF8010003
:10F0900061F307108DF80100694670680EF0BBFB44
:10F0A000012F62D13068B0F84810E1B390F8220027
:10F0B000C0F34000B8BB70680EF0C3FB401CC7B281
:10F0C0003068C7F1FF05B0F84820B0F85A10511A5F
:10F0D000A942B8BF0D46AA423BD990F8220010F0D1
:10F0E000010F36D144F01004214670680EF0B9FBD0
:10F0F000F81CC0B2ED1E284482B23068B0F86A1025
:10F10000436EC1F30B0151FA83F190F860305B4F0D
:10F110001944BC460023E1FB07C31B096FF0240C14
:10F1200003FB0C1100E020E080F8601090F85F0015
:10F13000012101F007F90090BDF800009DF80210D0
:10F14000032340EA01400190042201A970680EF0F7
:10F1500062FB3068AAB2416C70680EF0B0FB306898
:10F16000B0F85A102944A0F85A1014F0400F06D0F5
:10F17000D6E900100123062261310EF04CFB14F099
:10F18000200F18BFFFDF0020002818BFFFDF02B0EC
:10F19000BDE8F0872DE9F043364C89B0206800289F
:10F1A00008BFFFDF20684178002936D10178FF29A8
:10F1B00033D0002680F83160A0F85A60867080F85D
:10F1C0003860304608F0AEF92D4802AD00F1240158
:10F1D00091E80E1085E80E10D0E90D10CDE906106B
:10F1E00002A808F08DF907F0F3FD206890F961009E
:10F1F00007F0BCFE234807F0BFFE234808F06CF977
:10F20000606808F092F9206890F8240010F0010F6F
:10F2100007D0252007F0B8FE0AE009B00C20BDE8B1
:10F22000F08310F0020F18BF262077D007F0ACFE55
:10F23000206890F85E10252007F096FD206880F881
:10F240002C6008F069F9206890F85E10002007F043
:10F2500095FF0F21052007F05DFE206890F82E1025
:10F26000002901BF90F82F10002990F8220010F01B
:10F27000040F0BE0640000201A06002053E4B36E74
:10F28000F855020000560200FD55020075D005F049
:10F29000FDFD054620682946806806F0E6FADFF89D
:10F2A0002C84074690FBF8F008FB1070414228467A
:10F2B00005F0D3FA2168886097FBF8F04A6810449B
:10F2C00048600CF097FF01462068426891426FD871
:10F2D000C0E90165FE4D4FF0010895F82D000CF0D6
:10F2E000A8FF814695F82F000127002818BFB9F123
:10F2F000000F04D095F82D000CF060FDA8B195F832
:10F30000300000281CBF95F82E00002825D0687B0F
:10F3100005F10E01012816D01AE0FFE710F0040FE6
:10F3200014BF2720FFDF81D182E73A466F7305F1D2
:10F330000E01484608F0E2FD95F82D1005F10E008B
:10F340000DF06EF809E0487900F0C000402815D0B3
:10F35000414605F10E0008F009FE206890F82200F1
:10F3600010F0040F24D095F82D000CF0DDFD050001
:10F370001ED010210DF0DBFD40B119E00DF08DF82D
:10F380003A4605F10E0108F0B9FDE6E720683A4675
:10F3900000F11C01C776284608F0B0FD206800F196
:10F3A0001C0160680EF08EF8012160680EF0A5F86F
:10F3B0002068417B0E3007F08FFD206890F85C10CC
:10F3C00061B3B0F85810A0F84810416D416490F84E
:10F3D0002210C1F30011F1B9B0F86A000221C0F3A4
:10F3E0000B05ADF80050684606F072FE28B1BDF876
:10F3F0000000C0F30B00A84204D1BDF80000401C7F
:10F40000ADF800002168BDF80000B1F86A2060F393
:10F410000B02A1F86A20206880F85C60206890F8F0
:10F420005D1039B1B0F85010A0F84010C16CC16344
:10F4300080F85D60B0F86A10426EC1F30B0151FABA
:10F4400082F190F86020DFF88CC2114463460022FC
:10F45000E1FB0C3212096FF0240302FB031180F868
:10F4600060100CF04AFF032160680CF0C9FF2168AE
:10F4700081F8330009B00020BDE8F0839649886028
:10F4800070472DE9F043944C83B0226892F83130F4
:10F490003BB1508C1D2808BFFFDF03B0BDE8F0432F
:10F4A00098E401260027F1B1054692F8600007F0C4
:10F4B0006BFD206890F85F10FF2007F055FC206876
:10F4C0004FF4A57190F85F20002007F01FFF20681F
:10F4D00090F8221011F0030F00F02C81002D00F0A5
:10F4E000238100F027B992F822108046D07EC1F324
:10F4F0000011002956D0054660680780017821F088
:10F5000020010170518C132937D01FDC102908BF4E
:10F51000022144D0122908BF062140D0FFDF6C4DE4
:10F52000606805F10E010DF0BFFF697B60680DF0AA
:10F53000D7FF2068418C1D2918BF152963D0B0F86A
:10F540004820416C60680DF0E4FF5CE0152918BFAD
:10F550001D29E3D14FF001010DF080FF60680178B3
:10F5600041F020010170216885B11C310DF0AAFF26
:10F57000012160680DF0C1FFD1E700210DF06EFFA1
:10F580006068017841F020010170C8E715310DF085
:10F5900099FF2068017D60680DF0AFFFBFE70DF0B7
:10F5A0005DFFBCE70021FFF762FC6068C17811F0E5
:10F5B0003F0F28D0017911F0100F24D00DF04CFF2F
:10F5C0002368024693F82410C1F38000C1F3400C75
:10F5D000604401F00101084493F82C10C1F3800C41
:10F5E000C1F34005AC4401F001016144401AC1B2CD
:10F5F00093F85E0000F0A6FE009003230422694603
:10F6000060680EF008F92068002590F8241090F842
:10F610002C0021EA000212F0010F18BF01250ED1C3
:10F6200011F0020F04D010F0020F08BF022506D01F
:10F6300011F0040F03D010F0040F08BF0425B8F137
:10F64000000F2BD0012D1BD0022D08BF26201BD070
:10F65000042D14BFFFDF272016D0206890F85E101D
:10F66000252007F081FB206890F82210C1F30011DB
:10F6700069B101224FF49671002007F047FE0DE0BA
:10F68000252007F081FCE8E707F07EFCE5E790F82D
:10F690005E204FF49671002007F038FE206890F845
:10F6A0002C10294380F82C1090F8242032EA010114
:10F6B0001CD04670418C13292BD026DC102904BFA6
:10F6C00003B0BDE8F083122923D007E040420F00C9
:10F6D0000C06002053E4B36E64000020C1F3001058
:10F6E000002818BFFFDF03B0BDE8F083418C1D295F
:10F6F00008BF80F82C70DCD0C1F30011002914BFC2
:10F7000080F8316080F83170D3E7152918BF1D29C2
:10F71000DBD190F85E2003B04FF00101BDE8F0436B
:10F72000084607F0E8BF00BF90F85F2001210846B7
:10F7300007F0E1FF2168002DC87E7CD04A8C3D4651
:10F74000C2F34000002808BF47F0080512F0400F40
:10F7500018BF45F04005002819BFD1F83C90B1F81A
:10F760004080D1F84490B1F8488060680721078054
:10F770000DF074FE002160680EF067F8294660689D
:10F780000EF06FF815F0080F17D02068BDF80010C4
:10F790000223B0F86A2062F30B01ADF8001090F874
:10F7A0006B00032201099DF8010061F307108DF839
:10F7B0000100694660680EF02EF860680DF00AFFDF
:10F7C0002168C0F1FE00B1F85A20A8EB0201814285
:10F7D000A8BF0146CFB2D019404544D245F0100130
:10F7E00060680EF03EF860680DF0F4FE2168C0F12C
:10F7F000FE00B1F85A10A8EB01018142A8BF0146F2
:10F80000CFB260680EF01DF83844421C2068B0F892
:10F810006A10436EC1F30B0151FA83F190F8603026
:10F82000F94D1944AC460023E1FB05C34FEA131C14
:10F830006FF0240300E03CE00CFB031180F8601043
:10F8400090F85F00012100F07DFD0090BDF8000000
:10F850009DF80210032340EA01400190042201A90F
:10F8600060680DF0D8FF216891F8220010F0400F79
:10F8700005D001230622613160680DF0CCFF2068BD
:10F880003A46B0F85A0000EB090160680EF017F82C
:10F890002068B0F85A103944A0F85A1008F009FA54
:10F8A000002818BFFFDF20684670867003B0BDE8EF
:10F8B000F0830121FFF7DBFAF0E7D44810B50068C8
:10F8C000417841B90078FF2805D000210846FFF7AC
:10F8D000D8FD002010BD07F0B2FE07F091FE07F042
:10F8E00052FD07F0FFFD0C2010BD2DE9F041C74D82
:10F8F0000446174628680E4690F86C00002818BF8A
:10F90000FFDF2868002F80F86E7018BFBDE8F08117
:10F910002188A0F870106188A0F88610A188A0F84E
:10F920008810E188A0F88A1094F88C1180F88C1067
:10F9300090F82F10002749B1427B00F10E01012AF7
:10F9400004D1497901F0C001402935D090F8301038
:10F9500041B1427B00F10E01012A04BF497911F047
:10F96000C00F29D000F17A0015F026FD6868FF2E3F
:10F970000178C1F380116176D0F80310C4F81A1031
:10F98000B0F80700E08328681ED0C0F88010E18B33
:10F99000A0F8841000F17402511E30460CF052FCA5
:10F9A000002808BFFFDF286890F8731041F00201BB
:10F9B00080F87310BDE8F081D0F80E10C0F87A100E
:10F9C000418AA0F87E10D1E7C0F88070A0F884705A
:10F9D000617E80F87310D4F81A104167E18BA0F8AB
:10F9E0007810BDE8F08170B5884C0125206890F84A
:10F9F0002200C0F3C00038B13C22FF21A068FFF70D
:10FA000074FF206880F86C50206890F8220010F095
:10FA1000010F1CBFA06801884FF03C0212BF0120FB
:10FA20004FF6FF710020FEF773FD206880F8385014
:10FA300070BD7649096881F8320070472DE9F041C0
:10FA4000002608F06CFE002800F0F7806F4C20685C
:10FA5000417800270125012906D0022901D0032978
:10FA60007BD0FFDFBDE8F081817802270029418C3F
:10FA700037D0C1F34002002A08BF11F0010F6DD04A
:10FA800090F85F204FF001014FF0000007F033FEC7
:10FA9000216891F82200C0F34000002814BF0C2018
:10FAA000222091F85F1007F05FF92068477090F806
:10FAB000330020B106F025FF402007F0CCFD206880
:10FAC00090F83400002818BF07F0F2FD00219620BE
:10FAD00007F05AFD08F0E4F8002818BFFFDFBDE882
:10FAE000F081C1F3001282B110293ED090F83300AA
:10FAF00020B106F006FF402007F0ADFD206890F829
:10FB0000221011F0040F35D042E090F8242090F834
:10FB10002C309A4229D1B0F84800002808BF11F0D3
:10FB2000010F05D111F0020F08BF11F0200F6FD0A7
:10FB30004FF001014FF00000FFF7A3FC2068418C5B
:10FB400011F0010F04BFC1F3400100290AD1B0F840
:10FB50005A10B0F84820914201E032E026E018BF88
:10FB6000BDE8F08180F83150B9E7BDE8F0410021EF
:10FB7000012086E490F83610012914BF03291026CD
:10FB800046F00E0190F85E204FF0000007F0B3FD44
:10FB9000206890F83400002818BF07F089FD002184
:10FBA000962007F0F1FC2068477098E7B0F85A10EB
:10FBB000B0F84800814240D0BDE8F041012108463C
:10FBC0005FE48178D9B1418C11F0010F21D080F828
:10FBD0006C5090F86E20B0F870100120FEF798FC81
:10FBE0002068477007F02BFD07F00AFD07F0CBFBFC
:10FBF00007F078FCBDE8F041032008F0C4BD81782F
:10FC0000BDE8F04101203CE453E4B36E6400002001
:10FC100013E011F0020F08BFFFDF3FF460AFB0F850
:10FC20005A10B0F84000814207D001210846FFF782
:10FC300028FC21680320487051E7BDE8F041FFF738
:10FC4000C9B8FFF7C7B810B5FE4C206890F834105B
:10FC500049B1373007F037FD18B921687F2081F8A6
:10FC6000370007F01BFD206890F8330018B107F04B
:10FC700005FD06F05AFE08F052FDA8B1206890F884
:10FC80002210C1F3001179B14078022818BFFFDFBC
:10FC900000210120FFF7F5FB2068417800291EBFF5
:10FCA00040780128FFDF10BDBDE81040FFF792B893
:10FCB0002DE9F047E34C0F4680462168B8F1030F69
:10FCC000488C08BFC0F3400508D000F0010591F84A
:10FCD0003200002818BF4FF0010901D14FF0000990
:10FCE00007F046F90646B8F1030F0CBF4FF00208C3
:10FCF0004FF0010835EA090008BFBDE8F087206829
:10FD000090F8330068B10CF0DBFA38700146FF2838
:10FD100007D06068C01C0CF0ACFA38780CF0DDFA43
:10FD2000064360680178C1F3801221680B7D9A4216
:10FD300008D10622C01C1531FEF708FB002808BFB9
:10FD4000012000D000203978FF2906D0C8B92068EA
:10FD500090F82D00884216D113E0A0B1616811F827
:10FD6000030BC0F380100CF048FA05460CF0A8FB1A
:10FD700038B128460CF0D8F818B110210DF0D7F89A
:10FD800008B1012000E00020216891F8221011F054
:10FD9000040F01D0F0B11AE0CEB9AB4890F83600AC
:10FDA000002818BF404515D1616811F8030BC0F356
:10FDB00080100CF022FA04460CF082FB38B1204689
:10FDC0000CF0B2F818B110210DF0B1F810B101200B
:10FDD000BDE8F0870020BDE8F0872DE9F04F994D90
:10FDE000044683B0286800264078022818BFFFDF49
:10FDF00028684FF07F0A90F8341049B1373007F087
:10FE000062FC002804BF286880F837A007F046FC91
:10FE100068680DF045FB8046002C00F0418207F039
:10FE200075F8002800F03C82012400274FF0FF09FC
:10FE3000B8F1050F1ED1686890F8240000F01F008B
:10FE4000102817D9286890F8350098B18DF80090DF
:10FE500069460520FFF72CFF002800F02182286862
:10FE600080F8A64069682222A730C91CFEF79BFAD9
:10FE700000F016BA68680DF09EFC002800F01082B1
:10FE80004046DFF8C4814FF0030B062880F01A8249
:10FE9000DFE800F0FCFCFC03FCFB8DF800906946F9
:10FEA0000320FFF705FF002800F0F180296891F892
:10FEB000340010B191F89C00D8B1286881780129EC
:10FEC0004DD06868042107800DF0C8FA08F10E01D2
:10FED00068680DF0E9FA98F80D1068680DF000FBFD
:10FEE0002868B0F84020C16B68680DF036FB00F060
:10FEF0005FB99DF8000081F89C400A7881F89D2048
:10FF0000FF280FD001F19F029E310CF09BF90028D1
:10FF100008BFFFDF286890F89E1041F0020180F8CA
:10FF20009E100DE068680278C2F3801281F89E206E
:10FF3000D0F80320C1F89F20B0F80700A1F8A30073
:10FF4000286800F1A50490F837007F2808BFFFDF7C
:10FF5000286890F83710217080F837A0ADE790F846
:10FF600022000721C0F3801938480479686869F3D2
:10FF7000861407800DF072FA002168680DF065FCA8
:10FF8000214668680DF06DFC0623002208F10E0181
:10FF900068680DF040FC2868417B68680DF0A0FAA5
:10FFA00068680DF017FB2968B1F84020C0F1FE0128
:10FFB0008A42B8BF1146CFB2BA423CD9F81EC7B286
:10FFC00044F0100A514668680DF04BFC68680DF06B
:10FFD00038FC384400F101082868B0F86A10426E15
:10FFE000C1F30B0151FA82F190F86020184C0A44D9
:10FFF000A4460023E2FB04C319096FF0240301FBAC
:020000040001F9
:10000000032180F8601090F85F004246012100F063
:1000100099F90190BDF804009DF80610032340EA09
:1000200001400290042202A968680DF0F4FB5146D9
:1000300068680DF016FCB9F1000F0FD0D5E900107B
:10004000012307E0640000200C060020F8550200A0
:1000500053E4B36E062261310DF0DDFB28683A46A9
:10006000C16B68680DF02BFC2868A0F85A70B0F8D6
:1000700040108F420CBF0121002180F8311007F0A1
:1000800018FE002818BFFFDF92E007E01AE1286899
:100090008078002840F0068100F002B98DF80090C9
:1000A00068680178C1F38019D0F803100191B0F8A5
:1000B0000700ADF8080069460520FFF7F9FD0028A4
:1000C000286879D08178002978D090F85FA0D5E9A8
:1000D0000104D0F80F10C4F80E10B0F813106182AC
:1000E000417D2175817D6175B0F81710E182B0F80E
:1000F00019106180B0F81B10A180B0F81D10E180CC
:1001000000F11F0104F1080015F05FF9686890F82C
:10011000241001F01F01217690F8240000214009ED
:1001200084F88C0184F864A084F865A004F13000A0
:100130000DF0D0FD2868002290F8691084F8661050
:1001400090F8610084F867009DF80010A868FFF738
:10015000CCFB022008F017FBA9480DF1040A082186
:100160000468686807800DF079F9002168680DF06F
:100170006CFB214668680DF074FB0623002208F131
:100180000E0168680DF047FB2868417B68680DF038
:10019000A7F9494668680DF0B0F9062301225146D7
:1001A00068680DF038FB07F084FD002818BFFFDFFA
:1001B000286880F801B077E06DE0FFE76868D5F85F
:1001C00008804FF00109027898F80D10C2F3401230
:1001D000114088F80D10D0F80F10C8F80E10B0F8C4
:1001E0001310A8F81210417D88F81410817D88F84A
:1001F0001510B0F81710A8F81610B0F81910A8F8D4
:100200000210B0F81B10A8F80410B0F81D10A8F8E0
:10021000061000F11F0108F1080015F0D6F8686813
:1002200090F8241001F01F0188F8181090F82400AD
:100230000021400988F88C0188F8649088F865905E
:1002400008F130000DF046FD2868002290F8691092
:1002500088F8661090F8610088F867009DF8001033
:10026000A868FFF742FB286880F86C4090F86E2081
:10027000B0F870100120FEF74BF92868477007F0BE
:10028000DEF907F0BDF907F07EF807F02BF9012041
:1002900008F079FA08E090F82200C0F3001008B1E5
:1002A000012601E0FEF796FD286890F8330018B1AA
:1002B00007F0E4F906F039FB66B100210120FFF7F1
:1002C000E0F810E0286890F82200C0F30010002841
:1002D000E8D0E5E728688178012904D190F85F101B
:1002E000FF2006F041FD28684178002919BF4178B8
:1002F000012903B0BDE8F08F4078032818BFFFDF65
:1003000003B0BDE8F08F70B53E4C06460D46206840
:10031000807858B106F08FFC21680346304691F88A
:100320005F202946BDE8704008F0D8BF06F083FC86
:1003300021680346304691F85E202946BDE87040AA
:1003400008F0CCBF78B50C4600210091082804BF06
:100350004FF4C87040210DD0042804BF4FF4BF7083
:10036000102107D0022807BF01F11800042101F174
:1003700028000821521D02FB010622489DF80010AA
:10038000006890F8602062F3050141F040058DF8A7
:10039000005090F85F00012804BF9DF8020020F093
:1003A000E0002AD0022818BFFFDF21D025F080000E
:1003B0008DF80000C4EB041000EB80001E2101EB5F
:1003C000800006FB04041048844228BFFFDF0F486A
:1003D000A0FB0410BDF80110000960F30C01ADF89A
:1003E0000110BDF800009DF8021040EA014078BD00
:1003F0009DF8020020F0E00020308DF80200D5E7E3
:10040000F855020064000020C4BF03008988888872
:100410000178406829B190F82C1190F88C0038B917
:1004200001E001F0BFBC19B1042901D001207047DF
:100430000020704770B50C460546062102F0BEFB51
:10044000606008B1002006E00721284602F0B6FBF4
:10045000606018B101202070002070BD022070BDC6
:100460002DE9FC470C4606466946FFF7E3FF0028E6
:100470007DD19DF8000050B1FEF70AF9B0427CD062
:10048000214630460AF0A5F8002873D12DE00DF082
:1004900049FDB04271D02146304612F021FD0028BE
:1004A00068D1019D95F8F00022E0012000E00020D5
:1004B000804695F839004FF0010A4FF00009F0B17D
:1004C00095F83A0080071AD584F8019084F800A0C6
:1004D00084F80490E68095F83B102172A98F618121
:1004E000E98FA18185F8399044E0019D95F82C01B0
:1004F00070350028DBD1287F0028D8D0D5E73046DA
:1005000002F0A1FC070000D1FFDF384601F0AFFE8A
:1005100040B184F801900F212170E680208184F899
:1005200004A027E0304602F07CFC070000D1FFDF8A
:10053000B8F1000F21D0384601F0F1FEB8B19DF8B6
:10054000000038B90198D0F818014188B14201D1B2
:1005500080F80090304607F0F9FB84F801900C21F8
:10056000217084F80490E680697F217200E004E045
:1005700085F81C900120BDE8FC870020FBE71CB536
:100580006946FFF757FF00B1FFDF684601F016FC30
:10059000FE4900208968A1F8F2001CBD2DE9FC414C
:1005A00004460E46062002F0B1FA0546072002F086
:1005B000ADFA2844C7B20025A8463E4417E020887B
:1005C000401C80B22080B04202D34046A4F8008094
:1005D00080B2B84204D3B04202D20020BDE8FC8110
:1005E0006946FFF727FF0028F8D06D1CEDB2AE4238
:1005F000E5D84FF6FF7020801220EFE738B54FF6B0
:10060000FF70ADF800000DE00621BDF8000002F01B
:10061000E7FA04460721BDF8000002F0E1FA0CB148
:1006200000B1FFDF00216846FFF7B8FF0028EBD0DC
:1006300038BD70B507F0F8FB0BF0C9FBD44C4FF692
:10064000FF76002526836683D2A025700168007995
:10065000A4F14002657042F8421FA11C1071601C99
:1006600012F05BFD1B2020814FF4A4716181A081F9
:10067000E181032121776177217404226274608211
:10068000A082A4F13E00E18205704680BF480C3094
:100690000570A4F110000570468084F8205070BDEC
:1006A00070B5BA4C16460D466060217007F034FBF9
:1006B000FFF7A4FFFFF7BDFF207810F090FAB748CE
:1006C0000DF076FD2178606812F0CCFC20780AF0FD
:1006D000EFFD284608F0DAFBB048FDF7E4FF21788B
:1006E00060680AF04FF83146207812F079FFBDE8D3
:1006F00070400BF06CBB10B501240AB1002010BD96
:1007000021B1012903D00024204610BD02210DF0A3
:1007100013F9F9E710B503780446002B4068134637
:100720000A46014608D00120F2F74FFC6168496A89
:10073000884203D9012010BD0020F5E7002010BD3C
:10074000887800B90320C97801B9032110701970A5
:100750000020704730B587B0044600886946FFF72F
:1007600069FE002806D1A08830B1012804D00228F3
:1007700002D0122007B030BD04AB03AA2146684660
:10078000FFF7DEFF0400F5D19DF8001001200025E1
:100790000029019906D081F8C501019991F810123C
:1007A00091BB29E081F82F01019991F8561139B9CF
:1007B000019991F82E1119B9019991F8971009B181
:1007C0003A2415E00695019981F82E01019A9DF8C9
:1007D0000C0082F83001019B9DF8102083F8312134
:1007E0008DF818008DF8192006AA00200CF043FDA2
:1007F000019880F82F5122E0019991F8C41119B99C
:10080000019991F8971009B13A2415E006950199DC
:1008100081F8C401019A9DF80C0082F8C601019B81
:100820009DF8102083F8C7218DF818008DF8192045
:1008300006AA01200CF01FFD019880F8C551204642
:1008400098E710B504460020A17801B90120E278AC
:100850000AB940F0020001F0C0FA002803D1204696
:10086000BDE8104076E710BD70B50D46044601891D
:10087000002380880CF0F4FC696A81421DD2401A82
:10088000401CA1884008091A8AB2A2802189081A4E
:100890002081668895F8641010460CF0BFFC8642F3
:1008A00000D230466080E68895F8651020890CF00B
:1008B000B5FC864200D23046E08070BDF0B585B010
:1008C0000D46064603A9FFF7B5FD00282DD19DF87A
:1008D0000C0060B300220499FB20B1F84E30FB2BD2
:1008E00000D30346B1F85040FB20FB2C00D3044654
:1008F000DFF8ACC09CE8811000900197CDF808C0EB
:10090000ADF80230ADF806406846FFF7ADFF6E80E7
:10091000BDF80400E880BDF808006881BDF8020059
:10092000A880BDF806002881002005B0F0BD012296
:10093000D1E72DE9F04186B0044600886946FFF70B
:1009400079FD00287ED12189E08801F060FA002835
:100950007FD1A188608801F05AFA002879D12189D5
:10096000E08801F04AFA002873D1A188608801F07C
:1009700044FA07006DD1208802A9FFF79FFF00B15C
:10098000FFDFBDF81010628809200BE07000002026
:1009900018080020FFFFFFFF1F000000D8060020FE
:1009A00034560200914254D3BDF80C10E2889142B3
:1009B0004FD3BDF81210BDF80E2023891144A28830
:1009C0001A44914245D39DF80010019D4FF0000854
:1009D000012640F6480041B185F8BB61019991F8C4
:1009E000FC1105F5DD7541B91AE085F8256101991D
:1009F00091F84A1105F5927509B13A2726E0E18888
:100A000069806188E9802189814200D30146A980FB
:100A1000A188814200D208462881012201990FE075
:100A2000E18869806188E9802189814200D301469B
:100A3000A980A188814200D208462881019900221C
:100A4000284600E005E0FFF70FFF2E7085F80180D3
:100A5000384606B0BDE8F0816BE770B504460DF08E
:100A600017FAB0B12078182811D1207901280ED1B9
:100A7000E088062102F0A2F8040008D0208807F0E0
:100A800065F92088062102F0ABF800B1FFDF0120F4
:100A900070BDF94D28780028FAD000266670142021
:100AA000207020223146201DFDF7A7FC0220207176
:100AB0002E70ECE710B50446FDF760FD002813D05A
:100AC000207817280FD1207968B1E088072102F03B
:100AD00075F840B1008807F039F9E088072102F085
:100AE0007FF800B1FFDF012010BD2DE9F0475FEA7C
:100AF000000800D1FFDFE04802211A308146FFF7ED
:100B00004DFD00B1FFDFDC4C0620678B01F0FEFFDE
:100B10000546072001F0FAFF2844C5B2681CC6B29A
:100B2000608BB04203D14046FFF7C4FF58B9608BD9
:100B3000A84203D14046FFF790FF20B9608B4146A1
:100B4000FFF78EFC38B1404601F06FF90028E7D17D
:100B50000120BDE8F08702214846FFF71FFD10B9CC
:100B6000608BB842DCD14046BDE8F04712F07DBD55
:100B700010B501F0BFF808B10C2010BD0BF07BF9E7
:100B8000002010BD10B50446007818B1012801D02E
:100B9000122010BD01F0BFF820B10BF01DFB08B111
:100BA0000C2010BD207801F07FF8E21D04F117033E
:100BB000611CBDE810400BF004BA10B5044601F00A
:100BC00099F808B10C2010BD207828B1012803D075
:100BD000FF280BD0122010BD01F066F8611C0BF04D
:100BE0000AF908B1002010BD072010BD01200BF04C
:100BF0003CF9F7E710B50BF0F2FA08B1002010BD90
:100C0000302010BD10B5044601F085F808B10C2065
:100C100010BD20460BF0DDFA002010BD10B501F02C
:100C20007AF820B10BF0D8FA08B10C2010BD0BF007
:100C30002DFA002010BDFF2181704FF6FF718180D9
:100C40008E4949680A7882718A880281498841817F
:100C500001214170002070471CB5002412F1080FDB
:100C600015D00CDC12F1280F11D012F1140F0ED098
:100C700012F1100F0BD012F10C0F0ED107E012F190
:100C8000040F04D01AB1032A01D0042A05D1012887
:100C900006D0022808D003280AD0122420461CBD02
:100CA0001046FEF778F8F9E710460DF07CFAF5E704
:100CB000084614466946FFF7BDFB08B10224EDE77C
:100CC0009DF80000019880F867400024E6E710B521
:100CD000134601220CF068F9002010BD10B504463F
:100CE00010F042FD052804D020460FF067FF0020D9
:100CF00010BD0C2010BD10B5044601F00CF808B171
:100D00000C2010BD2146002007F08FF8002010BDF8
:100D100010B504460FF0E1FF50B108F00DFB38B1FB
:100D2000207808F0BFF820780DF0FEFC002010BD00
:100D30000C2010BD10B5044600F0EDFF08B10C20EA
:100D400010BD2146012007F070F8002010BD38B515
:100D500004464FF6FF70ADF80000A079E1798842B3
:100D600016D02079FDF776FB90B16079FDF772FB24
:100D700070B10022A079114613F068F840B9002242
:100D8000E079114613F062F810B9207A072801D9EA
:100D9000122038BD08F0DDFA60B910F0E5FC48B962
:100DA00000216846FFF7FAFB20B1204605F0B5FFA9
:100DB000002038BD0C2038BD2DE9FC418178054666
:100DC0001A2925D00EDC16292ED2DFE801F02D2DB0
:100DD0002D2D2D212D2D2D2D2D2D2D2D2D2D2D2D4F
:100DE0002D2121212A291FD00BDCA1F11E010C2964
:100DF0001AD2DFE801F01919191919191919191955
:100E0000190D3A3904290FD2DFE801F00E020E0263
:100E10002888B0F5706F07D201276946FFF70AFBF3
:100E200020B10220BDE8FC811220FBE79DF8000004
:100E300000F041FF019C10B104F58A7401E004F553
:100E4000C8749DF8000000F036FF019E10B106F254
:100E5000151601E006F291166846FFF7D9FA08B1B7
:100E6000207808B10C20DDE72770A878307068463C
:100E700000F0A4FF0020D5E7180800207000002033
:100E80007CB50D466946FFF7D5FA002618B12E60ED
:100E90002E7102207CBD9DF8000000F00CFF019C2B
:100EA0009DF80000703400F006FF019884F842605D
:100EB00081682960017B297194F842100029F5D1DD
:100EC00000207CBD10B5044600F025FF20B10BF0DA
:100ED00083F908B10C2010BD207800F0E5FEE2791E
:100EE000611C0BF0FAFA08B1002010BD022010BD01
:100EF00010B5886E60B1002241F8682F0120CA71D8
:100F00008979884012F096FF002800D01F2010BD7C
:100F10000C2010BD1CB50C466946FFF78BFA002863
:100F200009D19DF8000000280198B0F8700000D0A9
:100F3000401C208000201CBD1CB50446008869466A
:100F4000FFF778FA08B102201CBD606828B1DDE91E
:100F50000001224600F0BDFF1CBDDDE90001FFF7E6
:100F6000C7FF1CBD2DE9F04104460078012804D0DC
:100F700018B1022801D003281ED1607828B10128B9
:100F800003D0022801D0032816D1E07B10B9A07845
:100F9000012811D1A07830F005020DD110F0050F15
:100FA0000AD0400801D0112054E5E078E688628933
:100FB0000F4618B1012801D012204BE5104600F071
:100FC000C6FF302558B13946304600F0CAFF30B16F
:100FD000A07B0028F0D00728EED800203AE528466C
:100FE00038E51FB5044600F07AFE10B10C2004B0BD
:100FF00010BD022104F10A0000F0BDFFA0788DF8B9
:101000000800A0788DF8000060788DF80400207842
:101010008DF80300A07B8DF80500E07B00B1012076
:101020008DF80600A078C0070CD0E078012812D017
:1010300098B100208DF80100E088ADF80A006089C1
:10104000ADF80C0002A80FF054FE0028CFD168467E
:101050000DF06FFBCBE70220ECE70120EAE710B5CB
:1010600004460121FFF77EFF002803D12046BDE89A
:101070001040B6E710BD0278012A01D0BAB118E0DD
:1010800042783AB1012A05D0022A12D189B1818869
:1010900079B100E059B1418849B1808838B101EB9C
:1010A0008101490000EB8000B1EB002F01D200204C
:1010B00070471220704770B5044600780D4601282D
:1010C00009D010F051FB052803D00FF022FD0028B5
:1010D00000D00C2070BD0DF020FA88B10DF032FA6E
:1010E0000DF007FB0028F5D125B160780DF0B8FAB6
:1010F0000028EFD1A1886088BDE870400FF014BED1
:10110000122070BD10B504460121FFF7B4FF00287E
:1011100004D12046BDE810400121CCE710BDF0B558
:10112000871FDDE9056540F67B44A74213D28F1F78
:10113000A74210D288420ED8B2F5FA7F0BD2A3F1A3
:101140000A00241FA04206D2521C4A43B2EB830F6E
:1011500001DAAE4201D90020F0BD0120F0BD2DE939
:10116000FC41477A8846044617F0050F73D0F8080B
:1011700071D1780701D5112054E694F83A0008B9E6
:10118000012F68D100252E46F8071BD088F00105F5
:10119000208A294600F0DBFE48B36089294600F02A
:1011A000E0FE20B3208A6189884254D8A18EE08D68
:1011B000CDE90001238D628CA18BE08AFFF7AFFFA0
:1011C000A8B10125B8070ED504EB4500828EC18D6C
:1011D000CDE90012038D428C818BC08AFFF79FFFFF
:1011E00028B12E466D1CB8F1000F02D023E030204C
:1011F00018E6228A012119E0B14203D004EB410034
:10120000008A024404EB4100C38A878ABB4222D190
:10121000838B478BBB421ED1438C078CBB421AD1B8
:10122000038DC08C834216D1491CC9B2A942E3D3B5
:10123000608990420FD3207810B101280BD102E0D1
:10124000A0780028F9D1607838B1012805D00228AB
:1012500003D0032801D01220E4E50020E2E50021BC
:101260007DE70178C90702D0406812F0D2B912F0C8
:101270009FB910B50078012800D00020FDF786FD49
:10128000002010BD2DE9F04788B00D46AFF6FC02F6
:10129000D2E90092014690462846FFF760FF06001B
:1012A0000CD100F01CFD40B9FE4F387828B90CF085
:1012B00039FEA0F57F41FF3902D00C2008B048E488
:1012C000032105F1100000F056FEF64801AA3E3851
:1012D0000190F5480290F34806211038039006A8C3
:1012E00001F03AFC040037D000210BF002FC04F1BD
:1012F00030017B8ABA8ACB830A84797C0091BA4612
:101300003B7CBA8A798A208801F014FD00B1FFDFA6
:10131000208806F01AFD218804F10E0000F005FD7A
:10132000E2A004F11207006800900321684604F06F
:10133000C5FE002069460A5C3A54401CC0B203282E
:10134000F9D3A88B6080688CA080288DE080687AB3
:10135000C10703D0012706E00920AFE7800701D5C8
:10136000022700E000273A46BAF8160011460FF0AF
:101370006FFD0146A06220460FF078FD3A462146F7
:1013800000200BF076FF00B90926C64A21461C3220
:1013900000200BF070FF002784F8767084F87770D7
:1013A000A87800F081FC6076D5F80300C4F81A0034
:1013B000B5F80700E083C4F8089084F80C80012099
:1013C00084F8200101468DF80070684604F076FE2E
:1013D0009DF8000000F00701C0F3C1021144C0F302
:1013E000401008448DF80000401D2076092801D2E5
:1013F00008302076012120460BF07BFB68780DF049
:1014000097F8E6BBA9782878EA1C0DF064F848B193
:101410000DF098F8A9782878EA1C0DF0FBF8060082
:1014200002D03AE0122638E0687A00F0010100208C
:10143000CA0700D00120890701D540F002000DF055
:1014400033F8060029D1214603200DF00DF90600DE
:1014500023D1687A00F001018DF81010C00705D083
:101460006889ADF81200288AADF8140004A80FF0BE
:1014700040FC064695F83A0000B1012000E00CE07F
:101480000DF024F84EB90DF034F9060005D1A98FFE
:1014900020460FF0CFFB060008D0208806F056FC4F
:1014A0002088062101F09CFB00B1FFDF304605E7F4
:1014B00001460020E6E638B57A48007878B910F0A1
:1014C00053F9052805D00CF02DFDA0F57F41FF391B
:1014D00005D068460FF06BFC040002D00CE00C2035
:1014E00038BD0098008806F031FC0098062100887D
:1014F00001F076FB00B1FFDF204638BD1CB58289C4
:101500004189CDE900120389C28881884088FFF7AC
:1015100006FE08B100201CBD30201CBD70B505467C
:10152000FFF7ECFF00280ED12888062101F046FBCA
:10153000040007D000F036FC20B1D4F8180101787F
:1015400031B901E0022070BDD4F86411097809B105
:101550003A2070BD05218171D4F81811002008814E
:10156000D4F81811A8884881D4F81811E88888811F
:10157000D4F818112889C881D4F818010289418942
:101580008A4204D88279082A01D88A4201D31220DB
:1015900070BD29884180D4F81811022008700020FD
:1015A00070BD3EB504460BF091FCB0B13D4801253D
:1015B000A0F140024570236842F8423F23790021A0
:1015C000137141706946062001F081FA00B1FFDF16
:1015D000684601F05AFA10B10EE012203EBDBDF887
:1015E0000440029880F82051684601F04EFA18B97C
:1015F000BDF80400A042F4D100203EBD70B5054600
:101600000088062101F0DAFA040007D000F0CAFBD6
:1016100020B1D4F81811087830B901E0022070BD6B
:10162000D4F86401007808B13A2070BDB020005DA4
:1016300010F0010F1BD0D5F802004860D5F8060065
:101640008860D4F81801698910228181D4F81801C2
:1016500005F10C010E3004F58C74FCF7A4FE216832
:1016600003200870216828884880002070BD0C2065
:1016700070BD38B504460078EF2854D86088ADF8BE
:101680000000009800F08AFCC0B36188080708D405
:10169000D4E90120824246D8202A44D3B0F5804FB5
:1016A00041D805E0180800207C00002011223300FA
:1016B000207B18B3072836D8607B28B1012803D0D7
:1016C000022801D003282ED14A0703D4022801D0D2
:1016D000032805D1A07B08B1012824D1480707D4ED
:1016E000607D28B1012803D0022801D003281AD137
:1016F000C806E07D03D5012815D110E013E00128CC
:1017000001D003280FD1C80609D4607E012803D078
:10171000022801D0032806D1A07E0F2803D8E07E3E
:1017200018B1012801D0122038BD002038BDF8B50D
:1017300015460E46044607F00CFE08B10C20F8BD15
:101740002046FFF796FF0028F9D1E07D03280BD053
:10175000A078C00602D4607E032805D0FDF720FBE8
:101760003070A07515B10CE01120F8BDFF208DF888
:10177000000069460020FDF7FDFA69460020FDF7EC
:10178000EDFA2046BDE8F840FDF749BA0022CEE761
:101790000078C10801D012207047FC4981F8200070
:1017A0000020704710B504460078C00704D1608857
:1017B00010B1FDF7B6FA80B12078618800F001021F
:1017C000607800F00FFC002806D1FDF792FA014680
:1017D0006088884203D9072010BD122010BD6168BF
:1017E000FDF7C8FA002010BD10B504460078C00708
:1017F00004D1608810B1FCF78CFF70B1207861884B
:1018000000F00102607800F0EDFB002804D1608850
:101810006168FDF7A3FA002010BD122010BD7CB551
:10182000044640784225012808D8A078FCF769FFD3
:1018300020B120781225012802D090B128467CBD25
:10184000FDF7BAFA20B1A0880028F7D08028F5D893
:10185000FDF7B9FA60B160780028EFD02078012850
:1018600008D006F095FB044607F06DFA00287FD0FB
:101870000C207CBDFDF7ECF810B9FDF796FA90B39B
:1018800007F067FD0028F3D1FCF702FFA0F57F41C8
:10189000FF39EDD1FDF7FEF8A68842F210704643FD
:1018A000A079FDF74FFAFCF73BFFF8B100220721C2
:1018B00001A801F051F9040058D0B5480021846016
:1018C00020460AF0D3FF2046FDF7D8FDAF4D04F1C6
:1018D00030006A8AA98AC2830184FCF728FF60B1BC
:1018E000E88A01210DE0FFE712207CBD314600208F
:1018F00007F0DBFA88B3FFDF44E0FDF766FA014644
:10190000E88A07F07DFB0146A0620022204606F02F
:1019100042FBFCF70CFF38B9FDF757FA02462146A7
:1019200001200BF0A6FCD0B1984A21461C320120C0
:101930000BF0A1FC687C00902B7CAA8A698A208825
:1019400001F0F8F900B1FFDF208806F0FEF931461A
:10195000204607F0AAFA00B1FFDF13E008E00721F4
:10196000BDF8040001F03CF900B1FFDF09207CBDA7
:1019700044B1208806F0EAF92088072101F030F907
:1019800000B1FFDF00207CBD002148E770B50D46A7
:10199000072101F013F9040003D094F8930110B16A
:1019A0000AE0022070BD94F87D00142801D01528AB
:1019B00002D194F8E00108B10C2070BD1022294634
:1019C00004F5CA70FCF7EFFC012084F893010020B5
:1019D00070BD10B5072101F0F1F818B190F893111E
:1019E00011B107E0022010BD90F87D10142903D03A
:1019F000152901D00C2010BD022180F89311002080
:101A000010BD2DE9FC410C464BF680321221944268
:101A10001CD8DCB16946FEF70DFD002815D19DF8F4
:101A2000000000F048F9019E9DF80000703600F0BB
:101A300042F9019DAD1C2F882246394630460AF0F6
:101A4000D0FE2888B842F6D1002005E4084603E419
:101A50007CB5044600886946FEF7ECFC002810D1EE
:101A60009DF8000000F027F9019D9DF800007035F9
:101A700000F021F90198A27890F82C10914201D140
:101A80000C207CBD7F212972A9720021E972E178C6
:101A900080F82D10217980F82E10A17880F82C1074
:101AA00000207CBD1CB50C466946FEF7C3FC00282F
:101AB0000AD19DF8000000F0FEF8019890F88C0023
:101AC00000B10120207000201CBD7CB50D461446DD
:101AD0006946FEF7AFFC002809D19DF8000000F030
:101AE000EAF8019890F82C00012801D00C207CBD68
:101AF0009DF8000000F0DFF8019890F87810297048
:101B000090F87900207000207CBD70B50D46164617
:101B1000072101F053F818B381880124C388428853
:101B200004EB4104AC4217D842F210746343A41092
:101B30006243B3FBF2F2521E94B24FF4FA72944233
:101B400000D91446A54200D22C46491C641CB4FBA3
:101B5000F1F24A43521E91B290F8CC211AB901E039
:101B6000022070BD01843180002070BD10B50C468C
:101B7000072101F023F868B180F8FF4024B190F804
:101B8000FD1009B107F052FA002010BD180800201E
:101B9000700000200220F8E7017889B1417879B11E
:101BA00041881B290CD381881B2909D3C1880229AC
:101BB00006D3F94902680A65406848650020704705
:101BC0001220704710B504460FF03EF9204607F08A
:101BD000E6F90020D9E710B507F0E4F90020D4E7D2
:101BE0002DE9F04115460F460646012211463846BA
:101BF0000FF02EF904460121384607F001FA84421D
:101C000000D204460121304600F05AF80646012170
:101C1000002000F055F83118012096318C4206D989
:101C200001F19600611AB1FBF0F0401C80B22880EF
:101C30000020BDE8F08110B5044600F06CF808B152
:101C40000C20A2E7601C0AF023FC207800F00100C1
:101C5000FCF71BFF207800F001000CF06EFC002068
:101C600093E710B50446072000F042FF08B10C20AE
:101C70008BE72078C00711D000226078114612F05F
:101C8000E5F808B1122080E7A06809F0ECF8607868
:101C9000D4F8041009F0F0F8002076E7002009F0ED
:101CA000E2F800210846F5E718B1022801D001202A
:101CB00070470020704708B100207047012070472E
:101CC00010B5012904D0022905D0FFDF20465CE7CA
:101CD000C000503001E080002C3084B2F6E710B52F
:101CE0000FF042FD042803D0052801D000204CE766
:101CF00001204AE710B5FFF7F2FF10B10CF0BDFC70
:101D000028B907F026FB20B1FCF79AFE08B10120A4
:101D10003BE7002039E710B5FFF7E1FF18B907F0FE
:101D200018FB002800D001202FE72DE9FE430025F5
:101D30000F4680460A260421404604F0E8F9404652
:101D40000BF0A0F8062000F0E1FE044615E069461D
:101D5000062000F0BCFE0AE0BDF80400B84206D040
:101D60000298042241460E30FCF7F0FA50B1684662
:101D700000F08BFE0500EFD0641E002C06DD002D68
:101D8000E5D005E040460BF086F8F5E705B9FFDF42
:101D9000D8F800000AF02FFD761E01D00028CAD026
:101DA000BDE8FE8390F8F01090F88C0020B919B1CE
:101DB000042901D0012070470020704701780029D4
:101DC0000AD0416891F8FD20002A05D0002281F850
:101DD000FD20406807F02AB9704770B514460546E3
:101DE000012200F013F9002806D121462846BDE85B
:101DF0007040002200F00AB970BDFB2803D840F6FD
:101E00004800814201D911207047002070471B38DB
:101E1000E12806D2B1F5A47F03D344F29020814299
:101E200001D912207047002070471FB55A49403130
:101E300091F82010CA0702D102781D2A0AD08A0719
:101E400002D402781C2A28D049073DD401781529EC
:101E500037D039E08088ADF8000002A9FEF7EAFA31
:101E600000B1FFDF9DF80800FFF725FF039810F889
:101E7000601F8DF8021040788DF803000020ADF847
:101E8000040001B9FFDF9DF8030000B9FFDF6846D9
:101E9000FEF7D7FCD8B1FFDF19E08088ADF800006D
:101EA00040F64801FB20ADF80410ADF80200ADF893
:101EB0000600ADF808106846FEF7CEFD38B1FFDF2A
:101EC00005E0807BC00702D0002004B05DE6012061
:101ED000FBE7F8B50746508915460C4640B1B0F50A
:101EE000004F05D20022A878114611F0AFFF08B1CB
:101EF0001220F8BDA06E04F1700630B1A97894F8F4
:101F00006E00814201D00C20F8BD012184F86F10D1
:101F1000A97884F86E106968A1666989A4F86C10C4
:101F20002889B084002184F86F1028886946FEF75C
:101F3000F1FFB08CBDF80010081A00B2002804DDD3
:101F400021463846FEF7D4FFDDE70020F8BD04281F
:101F500003D321B9B0F5804F01D90020704701208B
:101F60007047042803D321B9B0F5804F01D9002070
:101F700070470120704710B500224FF4C84408E0B4
:101F800030F81230A34200D9234620F81230521CF8
:101F9000D2B28A42F4D3F8E5D807002080B2C10655
:101FA0000BD401071CD481064FEAC07101D5B9B921
:101FB00000E099B1800713D410E0410610D48106E7
:101FC0000ED4C1074FEA807104D0002902DB40071C
:101FD00004D405E0010703D4400701D40120704771
:101FE0000020704770B50C460546FF2904D8FCF761
:101FF0009EFB18B11F2C01D9122070BD2846FCF79A
:1020000080FB08B1002070BD422070BD0AB10122E2
:1020100000E00222024202D1880802D109B1002068
:10202000704711207047000030B5058825F4004442
:1020300021448CB24FF4004194420AD2121B92B256
:102040001B339A4201D2A94307E005F40041214322
:1020500003E0A21A92B2A9431143018030BD0844A3
:10206000083050434A31084480B2704770B51D466D
:1020700016460B46044629463046049AFFF7EFFF02
:102080000646B34200D2FFDF282200212046FCF79B
:10209000B4F94FF6FF70A082283EB0B26577608039
:1020A000B0F5004F00D9FFDF618805F13C008142A7
:1020B00000D2FFDF60880835401B343880B22080B2
:1020C0001B2800D21B2020800020A07770BD8161DA
:1020D000886170472DE9F05F0D46C188044600F124
:1020E0002809008921F4004620F4004800F063FB31
:1020F00010B10020BDE8F09F4FF0000A4FF0010B37
